:1000000060440020E51200008FAF0000D112000014
:10001000D1120000D1120000D1120000D112000054
:10002000000000000000000000000000511400006B
:10003000D112000000000000E9130000D1120000FE
:10004000E5150000E5150000E5150000E5150000C8
:10005000E5150000E5150000E5150000E5150000B8
:10006000E5150000E5150000E5150000E5150000A8
:10007000E5150000E5150000E5150000E515000098
:10008000E5150000E5150000E5150000E515000088
:10009000E5150000E5150000E5150000E515000078
:1000A000E5150000E5150000E5150000E515000068
:1000B000E5150000E5150000E5150000E515000058
:1000C000E5150000E5150000E5150000E515000048
:1000D000E5150000E5150000E5150000E515000038
:1000E000E5150000E5150000E5150000E515000028
:1000F000E5150000E5150000E5150000E515000018
:10010000E5150000E5150000E5150000E515000007
:10011000E5150000E5150000E5150000E5150000F7
:10012000E5150000E5150000E5150000E5150000E7
:10013000E5150000E5150000E5150000E5150000D7
:10014000E5150000E5150000E5150000E5150000C7
:10015000E515000010F8012B11F8013B012A28BF1A
:100160009A42F7D0D01A7047034611F8012B03F8D2
:10017000012B002AF9D1704770B50D46044603F0F3
:1001800025F9224601462B780248BDE870400AF066
:1001900086BB00BF74E4000030B555489DB00AF03E
:1001A0007EFB54480AF07BFB002002F041FB014635
:1001B00028B151480AF073FB00201DB030BD4F48F4
:1001C0004F4C0AF06CFB4F480AF069FB22464E493F
:1001D0004E4803F021F9054608B10146E9E74748D2
:1001E0000AF05DFB4A480AF05AFB009549492B4644
:1001F000012220680BF025FA01460028D9D13F489A
:100200000AF04DFB44480AF04AFB4449206803F0D9
:10021000F5F901460028CCD138480AF040FB4048A7
:100220000AF03DFB3F49206803F028F90146002809
:10023000BFD132480AF033FB3B480AF030FB20685C
:100240000BF0A5FA01460028B3D12C480AF027FB91
:1002500036480AF024FB20680BF01DFA01460028FE
:10026000A7D126480AF01BFB31480AF018FB314998
:1002700020680BF0A4F9014600289AD11F480AF023
:100280000EFB206812A902F0A5FD9DF8483007ACCE
:10029000032B27D8DFE803F002202224264920463A
:1002A000FFF762FF9DF849301E2104939DF84A3004
:1002B000224A03939DF84B30059402939DF84C30ED
:1002C0000AA801939DF84D3000939DF84E3009F037
:1002D00007FE1B480AA96DE71A49E0E71A49DEE75D
:1002E0001A49DCE70A212046194A09F0F9FDD9E745
:1002F0008FE40000B4E40000D0E40000E1E400007A
:10030000780D0020EAE4000074E0000060E00000E6
:1003100004E5000080E000001CE50000F000002083
:1003200031E5000058E0000054E5000062E50000FF
:1003300081E50000AC250020A0E50000C9E5000033
:10034000ECE50000A7E50000AEE50000B8E5000020
:10035000C2E50000014B1B68184700BFF8000020F1
:10036000014B1860704700BFF800002030B585B021
:1003700004460D461022002168460DF056FB02236C
:100380008DF80230044B2A4621466846019309F055
:10039000D3FD05B030BD00BF5503000080B5054654
:1003A0000E461746984606F02BFA03460DF0E2FB80
:1003B0000446DFF81890424649F800303946304686
:1003C000A84754F8090000F0F9FF00BF080000003A
:1003D0002DE9F047058B04462807904611D40229E1
:1003E00005F0070540F0CC8020460AF072FA78B19B
:1003F0000138218B042811D8DFE800F0C2106D8588
:10040000950001290CBF45F0100545F02005258316
:1004100088F31188BFF36F8FBDE8F08701F0070AFA
:10042000AA4500F0A5800027B9463E46A368002BE8
:1004300000F0BC8041F00801218388F31188BFF3EC
:100440006F8FA168002900F0BA800D68002900F0C4
:10045000B680334652462046D1F80480C047002D6E
:1004600076D02B6829461D46F0E701F007035A1F96
:10047000012A1BD8002221F00701062B276889B228
:10048000C4E9002209D13B4603E0628B013262835A
:100490001B68002BF9D141F00201204621830AF0AC
:1004A00018FA00287AD041F0200176E0042B0AD116
:1004B00021F0070189B2204621830AF00AFA10B11F
:1004C00041F020012183218B01F0070AAA454FD07A
:1004D0000027B946AAE7236921F0070141F0060188
:1004E000062DD3F8009021832DD1B9F1000F3FD014
:1004F00041F00801218388F31188BFF36F8F2046F4
:100500003949C84729E021F00701236941F0040176
:1005100089B2042DD3F804902183E6D000274FF050
:10052000040A3E4682E721F00701236941F00501F4
:1005300089B2052DD3F808902183D6D000274FF03B
:10054000050A3E4672E700274FF0060A3E466DE771
:100550002B4687E7B9F1000FD1D1EFF311882023A3
:1005600083F31288BFF36F8F238B23F00803238359
:10057000258BEA062ED525F01003238305F0070509
:100580006669218B002EBFF670AF00232768C4E98F
:10059000003321F0070141F001012183218B4FF04D
:1005A000000901F0070AAA457FF440AF002F9CD054
:1005B00041F00801218388F31188BFF36F8F002F6A
:1005C000C8D03D6839463346524620460AF0ADF958
:1005D0002F46F4E7AB067FF51BAF25F020032383FE
:1005E00005F0070500E700BF57A90000034A13689C
:1005F0000BB9526813600020704700BFFC00002058
:1006000030B50C460E4985B00291D0F8D41105469C
:10061000CDE9003100F1F0014FF0FF33204604F046
:1006200099FE50B9012384F86C30D5F8D03123B14C
:10063000204605B0BDE83040184705B030BD00BFCA
:1006400099AC000038B50C46114605460AF026FB69
:10065000034638B9284604490AF020FB0346002027
:10066000236038BD0120FBE7EDEA00002DE9F04FE3
:10067000012381460569466891B005F56B77D7E897
:10068000EF2F002A03D1C7E8E13F0029F7D10CBFC3
:100690001A46002240F0BD80B368B16A05F5F878CB
:1006A0001C1F10460AF081FB84427BD8013A00F0FF
:1006B000AA80B2FA82F24FF00044D4407268204619
:1006C000073222F00302C5F83C22B16A0AF06DFB42
:1006D000C5F84002B36A40466343033323F0030383
:1006E00002EB4302230103EB4403093323F003032A
:1006F00003EBC403C5F834221A440832C5F830228B
:100700007368C5F83842C5F82C32434BC5E9AD6370
:10071000316800F0F3F90446002841D1D9F810B04F
:10072000D9F804A0D9F800300BF53479CDE90600EA
:1007300005934846DAE90734012B08BF103C0CF05A
:10074000FCFEDAF82400354905AB009301EB80216B
:10075000234648464FF4806205F0AAFC2021DAF8CF
:1007600024302F4A0DEB010009F0BAFB08A94846D6
:1007700005F01AFD2B490BF530700CF097FEDAE905
:10078000050183685C684CB15B46274AA047044674
:1007900030B9DAE9050183681B692BB96FF057049A
:1007A000002129E001327CE7012298470446002815
:1007B000F6D11E4B2846C5F8D0311D4BC5F8D431B3
:1007C0001C4B0393D5F840320293D5F83C32CDE967
:1007D000008305F51173B26AD5F8A81300F056F935
:1007E00004460028DCD105F1F00004F059FE002891
:1007F000C5F8B0030ADB022138460AF083FA204626
:1008000011B0BDE8F08F6FF00B04C9E76FF015046D
:10081000C6E76FF07704F2E7EFAC0000C0270020D6
:100820002DE60000D5AC0000C9AC0000390800007E
:1008300081AE000035AD000013B5044640B1002381
:100840000122CDE90032074BD0E9091204F056FD30
:10085000236F1B6823B1606F02B0BDE810401847DA
:1008600002B010BDEDEA000013B504460846216948
:1008700001F56B71D1E8AF1F022910D193B1A0B17E
:100880000121CDE900311346D0E9091204F036FD0B
:10089000074B984208BF6FF00B0002B010BD6FF01D
:1008A0000F00FAE76FF04C00F7E76FF00100F4E794
:1008B0002EF8FFFF2DE9F34789461546066906F530
:1008C0006B73D3E8AF3F022B64D1136823B96FF089
:1008D000150002B0BDE8F0871B78002BF7D0D6F8E2
:1008E000A8A3BAF1000F36D106F5EC774FF0FF322E
:1008F0004FF0FF33384605F03DF930462A6801A92C
:10090000FFF7A0FE019C80461CB938460AF0F8F9B2
:10091000DDE705F108032367AB6984F86CA0636722
:10092000646460B138460AF0EBF921463046A36EA4
:100930002A68FFF765FE0020C9F80040C9E71F22BA
:10094000296804F148000DF09AF8384684F8678069
:100950000AF0D6F9EFE7304610490AF09FF904464D
:100960000028B4D0002705F108030367AB6980F8BD
:100970006C70436740641F22296848300DF07FF88F
:1009800022460121304684F8677000F061F80028A3
:10099000D1D09CE76FF00F009BE700BFEDEA0000AD
:1009A00010B50C46006900F56B73D3E8AF3F022B1E
:1009B0000FD189B10A4900F530700CF0A3FD204633
:1009C0000CF0C2F87822002120460DF02EF800200D
:1009D00010BD6FF00F00FBE76FF00100F8E700BFFC
:1009E0007C0D00202DE9F04F05460E46904600276D
:1009F000D0F8C4A085B0AAF5BE7421463046FFF7F2
:100A0000A9FBE0B9114BA4F1480B0293DAF81030BE
:100A10003246CDE9008329464FF0FF335846AAF508
:100A2000E27904F097FC60B97823012203FB079375
:100A300083F86C20DAF80C300BB1584698477834BC
:100A400017B105B0BDE8F08F0127D6E7AFAE0000C3
:100A50001FB5144690B18AB1012912D10A4B00F199
:100A6000F0010293D0F8D431483201934FF0FF33B4
:100A70002046009304F06EFC04B010BD6FF015002A
:100A8000FAE70020F8E700BFAFAE00002DE9F04321
:100A900087B00E46DDE90E811446DDE910251F46BC
:100AA00030B329B3DFF850C000F1F009002D08BFC2
:100AB00065469EB9CDE9034400F5E27420460596EB
:100AC0000CF0DAFA03ABCDE900432A463B46414637
:100AD000484604F05FFD07B0BDE8F08300224146C0
:100AE0000E9248462A4607B0BDE8F04304F0A8BE7F
:100AF0006FF01500EFE700BFE5090000F0B5044610
:100B00002B4A87B004AB0E4692E8030083E803004B
:100B1000002C49D0184604F0F7FA0546B0B94FF05A
:100B2000FF33E16C04F15407A163CDE901000093A8
:100B30003846236D04F138020BF0B6FCA06C0AF0C5
:100B4000E5F9C4F8BC0020B96FF00B05284607B0E2
:100B5000F0BDA06C0AF0DAF9C4F8C0000028F3D0A8
:100B6000236CD4F8BC10C4F890300423C4F894303B
:100B7000C4F8AC300223E3620E4BB4F84820C4F84A
:100B80008C10616C236204F18C03C4F8A070A4F88B
:100B90009820C4F8B870C4F8A810A4F8B020C4F81D
:100BA000A400A6612363D1E76FF01505CEE700BF6F
:100BB00030E00000B8E00000014B03600020704707
:100BC000E4E0000008B5044809F069FE034809F0B4
:100BD00066FE002008BD00BF39E600006EE600009A
:100BE000014806F057BC00BFE4E0000038B50446F9
:100BF00018B90F4B0F485B6898476168B1F5683FBB
:100C000010D0B1F5680F0DD00B4DA9420AD011F4E8
:100C10006861206807D0014608480CF0E5FA002317
:100C20002360656038BD14220CF0FFFEF9E700BFB9
:100C3000C00200209CE600002C5F5CA9A4120020EA
:100C400008B560B34368B3F5683F0ED0B3F5680FDD
:100C500018D0144A934220D000684FF0FF324FF072
:100C6000FF3304F087FF58B115E001220368D3E891
:100C7000EF1F002903D1C3E8E02F0028F7D10AD1E4
:100C8000002008BD0368084A1B7803F5807352F8FA
:100C90002330002BF4D00548F3E70548F1E76FF463
:100CA000E040EEE72C5F5CA900000350E98FFFFFF6
:100CB000EA8FFFFF08B520B34368B3F5683F09D05A
:100CC000B3F5680F13D0114A93421DD0006804F0A9
:100CD000C9FF14E000220368D3E8EF1F012903D104
:100CE000C3E8E02F0028F7D109D0094808BD00214A
:100CF0000368084A1B7803F5807342F8231000202C
:100D0000F4E76FF4E040F1E70348EFE72C5F5CA9FC
:100D1000E98FFFFF00000350EA8FFFFF10B5044684
:100D200018B91D4B1D485B6898476368B3F5683F69
:100D30002FD0B3F5680F2CD0194A934219D12368EC
:100D400003BB4FF0FF324FF0FF332146154804F04C
:100D5000E3FE08B923681BB90F4B13485B6898473B
:100D60001422002120680CF060FE4FF46863636079
:100D700008E0B3F5683F0DD83A2B03D040F6BA62CD
:100D80009342DED120680CF07AFA636843F03A03AC
:100D9000636010BD054AF3E7C00200209CE6000036
:100DA0002C5F5CA9A4120020C2E600003A00003AC1
:100DB00008B506494023142205480CF007FABDE89F
:100DC00008400449044806F029BC00BFA40D0020D7
:100DD000A4120020ECE0000000E1000008B5034888
:100DE000034A0021121A0AF0CAF808BD780400204C
:100DF000BC270020074808B5074A0849121A0AF01C
:100E0000C0F8BDE808400648064A0749121A0AF029
:100E1000B8B800BF000000207404002044EE0000B9
:100E2000000000200000002044EE000038B5054618
:100E30000C4699B1D1E901230F48096809F02FFD4B
:100E4000D4E90423E1680D4809F029FDE1690C4863
:100E500009F025FDA1690B4809F021FD012D05D1FF
:100E6000EFF305810848103909F019FD214628469D
:100E7000BDE8384004F0FABCEFE600001FE70000D0
:100E80004FE700005FE700008EE7000030BFFFF78C
:100E9000FDBF00BF2DE9F04105460B4EDFF82C8069
:100EA000324606EB0807CC1B204609490CF096FD9C
:100EB000A01942460021083C0CF0B7FDC5F8A84037
:100EC00007F10800BDE8F081000000000400000008
:100ED00024E00000054B5A699B689A421FBF044AF0
:100EE000536843F080535360704700BF04150020DF
:100EF00000ED00E010B5204C204809F0D0FCA36ABA
:100F0000990137D51E4809F0CAFC1E20A36ADA01F0
:100F100003D51C4809F0C3FC1F20174CA36ADB0251
:100F200003D5194809F0BBFC0220A36A1C0303D5B2
:100F3000164809F0B4FC21200F4CA36A590303D5CD
:100F4000134809F0ACFC2220A36A9A0303D5114888
:100F500009F0A5FC2320084CA36ADB0303D50E4847
:100F600009F09DFC2420A36A6FEA03436FEA134350
:100F7000A36210BD1D20C9E700ED00E0A2E700005C
:100F8000BBE70000CFE70000EAE7000015E800003B
:100F900034E800005AE8000075E8000070B5244C01
:100FA000064624480D4609F07AFCA36AD90435D5D3
:100FB000214809F074FC1720A36A1A0503D51F48BD
:100FC00009F06DFC18201A4CA36A9B050FD51C482C
:100FD00009F065FCA16BA36A180407D5194809F04C
:100FE0005EFC1EB1A36A23F40043A3621920104CD7
:100FF000A36A590503D5144809F051FC1A20A36AC5
:10100000DA050DD5114809F04AFC1B20084A936AFD
:1010100043F47F43936200232B7070BD1620CBE70F
:10102000A36A9B04F2D50A4809F039FC1C20EDE7BD
:1010300000ED00E0A1E80000B8E80000CAE8000008
:10104000DEE80000F8E800000EE900002AE90000F0
:1010500043E9000070B5264C064626480D4609F0C7
:101060001EFCA36AD80640D5234809F018FC1120BD
:10107000A36A190703D5214809F011FC12201C4C62
:10108000A36A9A070FD51E4809F009FC616BA36A91
:101090001B0607D51B4809F002FC1EB1A36A23F00A
:1010A0008003A3621320124CA36ADE0703D51648FF
:1010B00009F0F5FB1420A36A9C0603D5134809F038
:1010C000EEFB15200A4B9A6AD10658BF9A6A9A6AB3
:1010D000920642BF5A6A22F400525A629A6A42F059
:1010E000FF029A6200232B7070BD1020C0E700BF82
:1010F00000ED00E073E900008AE90000CAE80000A2
:10110000BEE90000D7E90000EEE9000043E9000075
:101110002DE9F0415B4B04465F6800258AB0C7F3B8
:10112000080685F31188BFF36F8F02F07F43B3F198
:101130007F4F06D102F00C03082B13D1524809F05F
:10114000AEFB00252C464FF00008F31E8DF80780FB
:10115000092B00F28580DFE803F00A797D7583832F
:101160008383838110074CBF0C460125EBE747487A
:10117000444E09F094FB8DF80780F36A9A0704D572
:10118000434809F08CFB00232FE0F36A002B01DABF
:101190004048F6E7F36A5B00F5D53F4809F07FFB6E
:1011A0007369A26943F480737361BFF34F8FBFF318
:1011B0006F8F736932F8022C23F480737361BFF36D
:1011C0004F8FBFF36F8F4DF602739A4208D0B36A08
:1011D000DBB24BB301200DF10701FFF73BFF33E01A
:1011E00021682E4809F05BFB23689DF80720C2B9EF
:1011F00002AE04F12007324620686168083403C259
:10120000BC421646F7D1099AB5B3C2F3080121B919
:101210006FEA52226FEA42220992184602A9FFF7AA
:1012200005FE0AB0BDE8F081B36A13F47F4F05D024
:1012300001200DF10701FFF7B1FE05E0B36AB3F538
:10124000803FA0D3FFF756FE0346CEE700200DF106
:101250000701C2E700200DF10701ECE7104890E715
:10126000104B17F4F87F1049104818BF1946A6F123
:10127000100209F014FB86E722F4FF7222F001024B
:10128000CAE700BF00ED00E03CEA000068EA0000A9
:1012900080EA0000A2EA0000B1EA0000D1EA000002
:1012A000EEEA000023EA00000EEA000013EB000063
:1012B000064B5A6942F010025A615A6942F4806240
:1012C0005A615A6922F008025A61704700ED00E045
:1012D000EFF30880EFF3098101B57246FFF718FFBD
:1012E00001BD00BF002080F31488BFF36F8F002082
:1012F00080F30A8880F30B88104880F30888002068
:101300000F49087003F0ACF900200E490860BFF3E4
:101310004F8F00F02DF8202080F311880A484FF4F9
:101320000061401880F30988EFF31480022108431C
:1013300080F31488BFF36F8F00F0F0F86044002052
:10134000B927002094ED00E0203300200023184648
:101350000649D1F89020C2F30722934200DB704780
:10136000C1F89830C1F8A0000133F6E700ED00E0C5
:1013700010B572B6002484F31388FFF7E7FF234605
:101380004FF0FF300C4A03F120010133102B42F8DB
:101390002100F8D100234FF0FF30074A03F160012C
:1013A0000133102B42F82100F8D162B6BFF34F8F02
:1013B000BFF36F8F10BD00BF00E100E0084B9B68DA
:1013C00083420BD1EFF3058343B1064B5A6842F0D9
:1013D00080525A605A6A22F400425A6205F016BAE4
:1013E0000415002000ED00E016498A684FF0300037
:1013F0001044EFF3098C80E8F01F202080F312885E
:10140000BFF36F8F104F4FF000664A698A603E60ED
:10141000D2F8A8000D4C2060D2F8AC000023C2F82E
:10142000AC3080F3118802F1300090E8F01F8CF3AB
:10143000098802F1000004B509F0B4FDBDE80440DC
:10144000704700000415002004ED00E0C0120020E9
:101450001EF0040F0CBFEFF30880EFF309808169E1
:1014600011F8021C0229FFD001B5724609F08BFD6C
:1014700001BD00BF40B2002807DB01234109034A38
:1014800000F01F00834042F82130704700E100E087
:1014900040B200280CDB01220649430900F01F007E
:1014A0008240203341F82320BFF34F8FBFF36F8F6B
:1014B000704700BF00E100E0054B420953F82220CD
:1014C000012300F01F0003FA00F01040704700BF36
:1014D00000E100E040B2002801F10101ACBF00F1E1
:1014E0006040064B4FEA4111C9B2ABBF00F5614005
:1014F00000F00F0080F800131954704714ED00E05D
:10150000044B054A23F07F039360BFF34F8FBFF373
:101510006F8F70470000000000ED00E008B5FFF796
:10152000EFFF074AD2F8883023F47003C2F88830FE
:10153000FFF754FCFFF75EFC00F048F804F060FA97
:1015400000ED00E042F8203C009B0B4942F81C3CB7
:10155000019B21F0010142F8183C029B42F8081C53
:1015600042F8143C4FF0807342F8043C0023203AC8
:101570000265C0F8AC3070479D03000000B50E4B0B
:1015800015469860D0F8A8200C4B0E461A60D0F88B
:10159000983083F30B882C4686F309880020044B8F
:1015A00098472046002100220023024C20470000DB
:1015B000B5AF00009D03000004150020C0120020FC
:1015C0001022014B1A61704700ED00E0002320213A
:1015D0000348C2180133452B82F80013F9D1704734
:1015E00000E100E008B5EFF30583064A103B02EB8B
:1015F000C30152F8330049688847BDE80840FFF747
:1016000069BC00BF44DD00001FB5094C094A2346F0
:101610000121094800F0FAF800230393074B012148
:10162000E41A01A80193029400F0FAF804B010BD86
:10163000000007200000002010E1000078040020D6
:1016400010B50C7A0B6804F01F0223F01F031A4335
:10165000CB68640923F01F03054943EA440343F0C0
:101660000103C1F89800C1F89C20C1F8A03010BD5A
:1016700000ED00E010B5074BD3F89030C3F307231B
:10168000013B984202D8FFF7DBFF10BD6FF0150059
:10169000FBE700BF00ED00E02DE9F04F0F461446D8
:1016A00006464FF000084D4D85B0B84580F2928057
:1016B000D6F80490B9F1000F36D0B9F11F0F40F2FF
:1016C000878019F01F0F40F08380D6F800A01AF031
:1016D0001F0F7DD1504609F0A9FC834609EB0A0093
:1016E000013809F0A3FC834572D11BF1160F6FD0AE
:1016F0005C456DDDC5F898B0D5F89C10C5F898B07C
:10170000D5F8A03021F01F0143F01F0AD6E90032BE
:101710001A44994202F1FF391ED1CA4508D1314617
:101720005FFA8BF009F08BFC08F101080C36BCE77E
:101730003146C5F898B0D5F89C3022F01F0203F06E
:101740001F031343C5F89C30E0B209F078FC10F198
:10175000160F3DD0441CE7E7C5F898B0D5F8A02097
:10176000013B23F01F0302F01F021343CA45314619
:10177000E0B2C5F8A030E8D009F061FC10F1160F16
:1017800026D0C5F898B0D5F89C209DF808300AF10D
:10179000FF3A62F304038DF80830D5F8A0309DF8C5
:1017A00008205B0863F347128DF80820D6E9003261
:1017B0001344009323F01F035344A3EB09030130A8
:1017C00023F01F036946C0B20393FFF753FFBEE740
:1017D0006FF01504204605B0BDE8F08F00ED00E085
:1017E0000522044BC3F89420BFF34F8FBFF36F8FD4
:1017F000704700BF00ED00E0BFF35F8F0022024B97
:10180000C3F89420704700BF00ED00E010B5034C12
:101810002278FFF741FF207010BD00BFB0250020E7
:101820002DE9F74F294D8A4606464FF00008AB4692
:10183000274FD0451BDAD6F80490B9F1000F3FD0FE
:1018400031680846019109F0F1FB0199044609EB62
:101850000100013809F0EAFB84424FF014021D4BED
:1018600008D002FB08F36FF015024BF8032003B019
:10187000BDE8F08F14F1160F2C60F8D01978A14252
:10188000F5DD02FB08B0C7F89840C7F89840D7F8D4
:101890009C4000F10801007B64F304000871D7F854
:1018A000A0000C79400860F347140C71D7F89C1025
:1018B00021F01F016960D7F8A01021F01F012961F4
:1018C00008F1010814350C36B3E700BFC41200203C
:1018D00000ED00E0B0250020F0B55249524CD1F89F
:1018E00090302568C3F307239D4287B000F29680AD
:1018F0000020FFF781FF4D4BC1F8C030854216D163
:101900004B4C01A82570FFF757F900250646494FB3
:10191000AE4213D1002023784249D1F89020C2F37F
:101920000722934274DBFFF75BFF002043E061680E
:1019300001EB0011FFF784FE0130DFE70199280178
:1019400001EB0513DA683A40B2F5800F42D007D8B0
:10195000B2F5801F15D0B2F5001F2ED00135D7E7A4
:10196000B2F1006F43D0B2F1805FF7D15A689B6843
:101970000958013B22F01F00034423F01F030120FC
:1019800032E05A689B680958013B22F01F0003446B
:101990000120844623F01F0340EA4C10CDE90221C8
:1019A0008DF8100002A920780593FFF763FE002848
:1019B0002ADA6FF0150007B0F0BD5A689B68095825
:1019C000013B22F01F0003444FF0020C012023F0E2
:1019D0001F03E1E75A689B680958013B22F01F008A
:1019E0000344062023F01F034FF0000CD4E75A688D
:1019F0009B680958013B22F01F0003444FF0030C81
:101A0000012023F01F03C7E7237801332370A5E7E4
:101A1000C1F89830C1F8A00001337EE74FF0FF30E5
:101A2000C9E700BF00ED00E01CE10000AAFF440090
:101A3000B02500200000F0FF08B5024808F030FA99
:101A4000FEE700BF36EB000008B5024B1B68984765
:101A5000002008BDD8120020034B044A1860937878
:101A600043F0020393707047D81200205801002001
:101A700008B50649064821F00701C1F1005202F5F8
:101A8000E02208F0B2FE002008BD00BF7F5F00200A
:101A9000DC12002070B541690446867A0A4D59B1BE
:101AA000437ADB0706D42C2303FB06535B6A1B68CF
:101AB0009B689847002363612C20214606FB005059
:101AC000BDE870400BF083BCC40300202C22024B05
:101AD00002FB0030704700BFC40300202C21827A33
:101AE000054B01FB02339A6A1B7F801A1B3323F0DC
:101AF0000303B0FBF3F07047C403002038B52C2477
:101B0000827A064B04FB02335B6AD3E901240C6042
:101B10001568FFF7E3FF04FB005038BDC403002045
:101B20002DE9F04385B00546684690461C46039172
:101B30000BF03FFEDDE90067EFF31189202383F30B
:101B40001288BFF36F8F6B8B002B41D02A8B9A4288
:101B500025D900220023284604F0D4F80446F0B129
:101B600089F31188BFF36F8F039B002B41D032465E
:101B70003B4668460BF042FE2C21A27A254B2046BC
:101B800001FB02335B6A03A91B681D68DDE90023C2
:101B9000A847606170BB2046FFF77CFF24E0698B9B
:101BA0004B1E6B8389F31188BFF36F8F2B7F2A8BBA
:101BB000AC6A1B3323F00303521A02FB0344154B98
:101BC000154AEB1A9B105343A3722B7FE372CBE7AA
:101BD00089F31188BFF36F8F23464246284604F0ED
:101BE00091F804460028BFD10024204605B0BDE886
:101BF000F0836361012300252381039B29466382CF
:101C0000E27A656004F118000BF00FFF636925822A
:101C1000E360EAE7C4030020A38B2EBA70B52C253D
:101C20000C4C00B970BD037A4668002BFAD0013B1A
:101C3000DBB20372002BF5D1C3604360837A05FBEE
:101C400003431B6A13B198473046EAE7FFF722FFC8
:101C5000FAE700BFC4030020054B03EB8000D0F877
:101C6000003223F0E04343F04053C0F800327047A5
:101C700000258450052370B5144D154E2C78013481
:101C8000B4FBF3F303EB8303E41A0AF04BF8114AB5
:101C9000137823B156F82430C01A072814D94FF00E
:101CA0005023D3F8141141B10021C3F81411D3F813
:101CB00014312C700CB9012313702C780AF032F80F
:101CC00046F82400012070BD0020FCE7B22500206A
:101CD000E8120020B1250020012208B50B4B0C4969
:101CE000C3F8002502230020C1F8D036FFF7B4FF67
:101CF0001046FFF7B1FFC1F80427C1F80429C1F865
:101D0000002BBDE8084000F09DB800BF0010005057
:101D10000040005007B500220D4B0E49C3F8A82122
:101D2000C3F8AC204FF48062C3F8B8254FF40062CA
:101D30000948C3F83C250DF107020AF04EF80028C7
:101D400003DB9DF8070002F081FD03B05DF804FBA2
:101D500000A002502CA0025028A1025048B1054B0F
:101D6000054A1B68B3FBF2F35843044B43F00103ED
:101D7000184770476402002040420F0050E0000006
:101D8000002170B5104C114D114E000714F8013BA5
:101D900003F01F025B090FD0012B0FD1334603EB79
:101DA0008203D3F80022013122F0E04202430829E5
:101DB000C3F80022EAD170BD2B46F0E70023803241
:101DC00053F82230FFDE00BF3FEB000000258450B7
:101DD000002884502DE9F041064601200D46FFF70A
:101DE000CFFF4FF47F03D3F83021D3F83431072AE3
:101DF00020D1023B032B02D8114AD35CD3B14FF060
:101E000050244FF0010800270520C4F81886C4F8B4
:101E1000147609F0ADFF4046C4F8148609F0A8FF17
:101E2000C4F81476C4F8187630462B46BDE8F04165
:101E3000002118474FF050230022C3F81426F3E77F
:101E40003BEB00000149024808F092BD54E100005C
:101E5000FC1200201FB578B10023019303930123E6
:101E600069460848029308F096FD029B9B0700D143
:101E7000039B05B05DF804FB024805B05DF804EB78
:101E800008F0E0BDFC12002008B54FF0FF323F2300
:101E90000348C0E9002302F0C5FC002008BD00BFD4
:101EA0001813002008B504480BF03CF900280CBFBB
:101EB0006FF01200002008BDB8DC000010B509F07A
:101EC0009DF90BF053FB0B4C18B1D4E8AF3F63B94D
:101ED00010BD04F0A1FBD4E8AF3F1BB9BDE8104032
:101EE00004F0AEBB0A209847F8E70A20BDE810408E
:101EF000184700BF2013002038B50446084809F0F1
:101F0000C2F8054648B1631EDBB21F2B96BF054AD7
:101F10000021D15C0C3009F0FCF8284638BD00BF28
:101F20001C0400205AEB00000E38012810B50AD816
:101F3000094809F0A8F8044618B104210C3009F04A
:101F4000E8F8204610BD09B10448F2E70220BDE8D8
:101F50001040FFF7D1BF00BF48040020C403002099
:101F600010B50024084B86B0039303AB00934FF4E5
:101F70002C724FF0FF3305490548CDE9044404F0C5
:101F800097F8204606B010BD7AEB0000C02B002069
:101F900030080020054BD3E8AF2F02F00B02D3E846
:101FA000EF1FC3E8E02F0028F9D170478800002018
:101FB00010B5012104460C3009F0D6F82146BDE8E1
:101FC00010400023014A007809F03FB9DCE100002D
:101FD00010B5012104460C3009F0C6F82146BDE8D1
:101FE00010400223014A007809F02FB9CCE100002B
:101FF00010B5012104460C3009F0B6F82146BDE8C1
:1020000010400023014A007809F01FB9B4E1000034
:102010002DE9F04788461646824600286AD00023FC
:10202000DFF8D490D9E8EF4FC9E8E23F002AF9D1B0
:10203000002C5FD02046FFF751FD0C232F4D274683
:1020400003FB0050438853450DD0D9E8EF3FC9E862
:10205000E27F002AF9D1002B4CD01F463846BDE85C
:10206000F047FFF7DBBDA64208D0204609F006F88E
:10207000328AF16804F10C0009F042F82046FFF7BB
:102080002DFD0C2606FB00504368ABB1B8F1000FE4
:1020900012D12046FFF722FD012106FB00504268C5
:1020A000D2E90003127A03F01F06B1405B09DAB1EE
:1020B00000EB830009F0BAF82046FFF70FFD0C266D
:1020C00006FB00508368002BC8D02046FFF706FDB2
:1020D000704305F800802046FFF700FD06FB005521
:1020E000A86803F041FEB9E7C94300EB830009F09B
:1020F000C3F8E1E7BDE8F087C80000202413002002
:102100002DE9F8430C4604F087FAE268218A137837
:10211000042B6DD1022908D82046FFF77FFD00244B
:1021200004F08EFA2046BDE8F88353783E2B08D1A0
:102130000329F1D0D378012B01D00A2B49D10327F1
:1021400005E0052BFBD00E3B012B42D8012704F103
:102150000C06304609F018F8012105463046B4F85F
:10216000109008F0F9FF0221304608F0FDFF0378D7
:1021700080463E2B07D1E3681B78012B01D00A2B48
:1021800006D1032614E0052BFBD00E3B012B29D9E9
:1021900041F27B13194A1A491A4808F08DFB0023B3
:1021A00083F31188BFF36F8F0323184602DF0226E3
:1021B000154A0323214698F8000009F046F8B207B3
:1021C00012D56369A4F8109013FA85F5E560BB0792
:1021D000A5D521460D4808F05AFF0D490D480BF0D2
:1021E00081F99CE70126E3E72046FFF717FDEEE7BC
:1021F0002046FFF713FD6FF0150491E78AEB00000E
:10220000BEEB0000D7EB00009CE10000CC000020FA
:10221000080200200809002038B51C4808F04CFFCF
:10222000044688B300F10C05284608F0A5FF0428F1
:102230001DD12846022108F097FF037805460E3B82
:10224000012B0ED840F6B243114A1249124808F049
:1022500033FB002383F31188BFF36F8F03231846EA
:1022600002DF032321460D4A287808F0EEFF2046BE
:10227000FFF7D4FC0A4BD3F8CC302BB1BDE8384083
:10228000084909480BF02EB938BD00BFCC0000202A
:102290008AEB0000F4EB0000D7EB0000B4E1000093
:1022A00000000020080200200809002010B5C1E944
:1022B00000239DF808300C460B72FFF70FFC0C2230
:1022C000024B02FB00335C6010BD00BF24130020F2
:1022D000F8B502460B46104808F0D5FE0446C0B1DA
:1022E00004210C3008F002FF2046FFF7F7FB0C2713
:1022F00000260A4D07FB005046802046FFF7EEFB04
:1023000007FB005086602046FFF7E8FB07FB0055FF
:102310006E602046F8BD00BFF003002024130020AB
:10232000034B0146D3F8EC0082689268104700BF67
:10233000000000200421014808F078BF8800002038
:10234000014902480BF0CEB8F80100203008002007
:1023500070B505460C4659B94FF0FF304FF0FF31CC
:10236000FFF7B6FF044618B96FF06805284670BD40
:102370002046FFF7B3FB0C22154BA61802FB0033D7
:1023800030465D8008F000FF03280BD9032130465A
:1023900008F0D1FE0580238A0121033B837030467B
:1023A00008F0D1FE40F635439D4208D12046FFF7A4
:1023B000B7FF054648B12046FFF730FCD6E7214677
:1023C00004480AF0F9FFFFF7BBFF0025CEE700BF86
:1023D00024130020D40000202DE9F04306461746C0
:1023E0000C4687B069B94FF0FF304FF0FF31FFF76F
:1023F0006FFF044658B96FF06805284607B0BDE87E
:10240000F083887AFFF762FB304B834258D1012278
:10241000002168460AF0E5FF2046FFF75FFB0C232A
:10242000DFF8AC9003FB0090C0F808D0204608F01D
:1024300059FE01463046FFF78BFF054618B120468E
:10244000FFF7ECFBD9E74FF4A0220023684603F026
:10245000C5FC804690B14FF4FD731E4A1E491F48CB
:1024600008F02AFA424631461D4808F025FA85F35D
:102470001188BFF36F8F0323184602DF2046FFF752
:102480002DFB0C23584319F80060AEB12046093EDD
:10249000FFF7C4FB092E0CD8DFE806F0150B0B087C
:1024A000050B0B0B0B126FF00B05A6E76FF00C057D
:1024B000A3E76FF00405A0E7002FC0D03C609CE7C5
:1024C0006FF0150599E76FF06E0596E7F0030020B1
:1024D000241300208AEB000022EC0000D7EB000060
:1024E0002BEC0000F7B5144B054693F94F300C4622
:1024F000002B1DDA14B9204603B0F0BD082C4FF0B4
:10250000000142F2180001AA264628BF0826FFF75C
:1025100063FF0028F0D1019F3246F9682846013157
:102520000BF05CFA3846FFF779FB3544A41BE1E772
:102530006FF08500E0E700BF00000020F7B5002243
:1025400040F603401146FFF747FF0446002855D1E7
:10255000FFF720FD214641F2030001AAFFF73CFFEF
:10256000044600284AD1019AAE4DD16805F12C03EA
:10257000D1F80100D1F8051003C31046FFF74EFB58
:10258000214641F2010001AAFFF726FF0446002878
:1025900034D10198C3685A7885F824205A88EA848F
:1025A0001A7985F82520B3F807202A85B3F8053075
:1025B0006B85FFF733FB214641F2020001AAFFF7CA
:1025C0000BFF0446D0B9019F05F13406FA68531C8D
:1025D0004132344618685968083303C4934226468A
:1025E000F7D13846FFF71AFB09F080F8044628B9FE
:1025F00095F830305F0604D46FF01204204603B023
:10260000F0BD014601AA42F20300FFF7E5FE0446D1
:102610000028F3D1019A844BD168D1F80100D1F898
:10262000051003C31046FFF7F9FA214642F23A00BB
:1026300001AAFFF7D1FE0446002840F0C2800198AD
:10264000C368B3F80130A5F8A030FFF7E7FA95F8B2
:10265000306016F0200619D14FF0FF304FF0FF31F7
:10266000FFF736FE0446002800F0C18002210C303E
:1026700008F040FD0123214603704670324640F6C3
:102680006D40FFF7A9FE04460028B7D195F85030F9
:10269000180712D5002142F21C0001AAFFF79CFE88
:1026A00004460028AAD10198C368D3F80120D3F8C2
:1026B0000530C5E92623FFF7B1FA95F8923013F0FB
:1026C000180F01D1190604D500F078FF0446002840
:1026D00094D14FF0FF304FF0FF31FFF7F9FD044682
:1026E000002800F0848008210C3008F003FD10233E
:1026F0000022437002270723214607708370C270AF
:10270000027142718271C27142F20100FFF764FEF0
:10271000044600287FF472AF4FF0FF304FF0FF31D6
:10272000FFF7D6FD0646002861D008210C3008F0DE
:10273000E1FC802343702023047084700471447191
:1027400084712246C770C371314640F60140FFF7DD
:1027500043FE044600287FF451AF014601AA4FF61C
:102760000140FFF739FE044620BB0198FFF756FAF7
:1027700021464FF6024001AAFFF72EFE0446C8B9D3
:102780000198C368B3F80130A5F87530FFF746FA31
:1027900095F875305A070DD521464FF6034001AA2A
:1027A000FFF71AFE30B90198C3685B7885F874307A
:1027B000FFF734FAEB795BB903B0BDE8F04000F005
:1027C00025BB461D7FF41AAF1F23A5F8A0303EE7B6
:1027D0002E78002EF0D195F875309B061ED54FF05F
:1027E000FF304FF0FF31FFF773FD044610B96FF073
:1027F000680403E706210C3008F07CFCD5F80130B2
:1028000021460360094B32469B8883804FF6064081
:10281000FFF7E2FD04460028CED0EFE66FF0850416
:10282000ECE600BF00000020900000200100002026
:1028300073B5264D0646D5F8EC000AF073FC002867
:102840003CD06FF0020105F1880008F015FD012170
:1028500008F0ECFC10EA010433D11D4B1E600A465F
:1028600005F1B0000AF0BDFD05F1D4000AF098FDB5
:1028700018480AF062FE6FF007034FF4966216499B
:102880001448009403F014FC1449124803F08CFC23
:10289000D5F8EC00124983681B689847044628B9AC
:1028A0003EB9FFF74BFE78B9FFF744FD204602B072
:1028B00070BD05F1780003F0F5FBF7E76FF0120447
:1028C000F4E76FF07704F1E70446EFE7000000203B
:1028D0003013002008090020702E002070EC00004A
:1028E0000121000010B5FFF729FE044608B9FFF7E3
:1028F00021FD044B1B681BB12046BDE81040184762
:1029000010BD00BF3013002038B5044603210C3041
:1029100008F02AFCE3680578197840F63543B0F8EA
:10292000010098420AD02246FFF772FB35B10448F5
:1029300003F01AFABDE83840FFF702BD38BD00BF0A
:10294000B000002038B503F067FE274DD5F8D4302D
:10295000002B44D00022002305F1B00003F03EFA22
:1029600000283CD10022002305F1D40003F0CAF96D
:10297000044668B940F6C2431C4A1D491D4807F089
:102980009BFF84F31188BFF36F8F0323184602DF88
:10299000D5F8C80020B1FFF741F90023C5F8C830C9
:1029A000204608F09FFBC5F8C8002046FFF7B8FC9A
:1029B00098B1114803F0D8F92046FFF78FF80C22A0
:1029C0000E4B1F2102FB003022464088FFF720FB00
:1029D0002046FFF723F9FFF7B3FCFFF7B1FCBDE892
:1029E000384003F02DBE00BF000000208AEB00003D
:1029F00079EC0000D7EB0000B00000202413002089
:102A000038B5042104460C3008F0AEFB4578017857
:102A100022464088FFF7FCFA35B1044803F0A4F9D8
:102A2000BDE83840FFF78CBC38BD00BFB0000020C7
:102A3000F8B506460024094DEF79E3B29F4202D86B
:102A40006FF0010007E02946304608F01DFC07350D
:102A5000631C08B12046F8BD1C46EEE700000020CC
:102A600070B5144E0622314604460AF0E6FFD8B18E
:102A70004FF0FF304FF0FF31FFF72AFC0546A8B1B9
:102A8000062221460C3008F03BFB0022294642F288
:102A90000500FFF7A1FC40B93346226843F81D2921
:102AA000A288B28001221A77002070BD6FF0680002
:102AB000FBE700BF1D00002037B504460D4689B175
:102AC0002846184908F0E0FB60B9174A2968C4EBAA
:102AD000C4041151A318AA889A80AA799A71002077
:102AE00003B030BD684608F06CFB0028F8D168469A
:102AF000FFF79EFF0028F5DA0B4A0098C4EBC404E8
:102B000010519DF80610BDF80400A3189880997123
:102B1000002DE4D012592A609A88AA809B79AB7163
:102B2000DDE700BF47EB00000000002070B5044661
:102B300011B16FF0150070BDF0B1224908F0A4FB8F
:102B4000D0B92046FFF774FF002835DA237863B93F
:102B50001D4AD37983BB20681060A179A088917148
:102B600001219080D1711846E5E7012BE1D1A379CD
:102B700003F0C003C02BDCD1134DEB79012B1ED029
:102B800005F18803D3E8AF3FDB0707D4002CD0D092
:102B900020460C4908F078FB0028CAD1EE7921467E
:102BA000731C3046EB71FFF787FF08B93046C2E768
:102BB000EB79013BEB71BEE76FF07700BBE76FF09D
:102BC0000B00B8E747EB0000000000202DE9F341BF
:102BD0000446D8B1002141F2090001AAFFF7FCFB2D
:102BE000054698B9019E0622D6F80C80104908F1D6
:102BF000010738460AF021FF28B1062238460D4960
:102C00000AF01BFF30B93046FFF708F8002002B089
:102C1000BDE8F081D8F801303046C4F80130BB88F7
:102C20002570A4F80530FEF7F9FF0120EFE700BF9B
:102C300054EB00004EEB000007B56846FFF7C6FFF7
:102C4000044BD87118B169460020FFF735FF03B077
:102C50005DF804FB00000020F0B5294D89B0EE7945
:102C6000002E46D195F87630DB0722D56A463146EC
:102C70004FF60940FFF7B0FBD8B9DDF800C0DCF82B
:102C80000C406378012B1E4628BF012673B1A31C9C
:102C900002AA1234174618685968083303C7A342BA
:102CA0003A46F7D1186838609B88BB806046FEF7CB
:102CB000B5FFEE71002416260127EB79E0B28342BE
:102CC00002D8B3B1002012E008AB06FB003353F882
:102CD000182C33F8143C6946CDF80120ADF80530C6
:102CE0008DF80070FFF7E8FE01340028E5D009B048
:102CF000F0BD0021084609B0BDE8F040FFF716BF5F
:102D0000000000202DE9F0410D4617461C460646FE
:102D1000002856D0002B54D00A03037808D56D073D
:102D20004FD408F00FFB002849D1012323700CE099
:102D3000A9072CD026480FB1AA0608D4C3EBC302BA
:102D4000825C012A12D002B92270002037E090F88C
:102D50009020510638D5C3EBC302825C012A05D00E
:102D600002B92270237843F00203DFE74FF0010835
:102D7000072111FB03810144304608F092FAF0B9B3
:102D800084F80080002FE0D0AB06DED5EAE76A07C2
:102D900011D50F49C3EBC3028E5C012E08D1072267
:102DA00012FB0363194408F07CFA40B92670EBE784
:102DB000002EE9D1FAE708F0C5FA01232370BDE837
:102DC000F0816FF01500FAE76FF08500F7E700BFBC
:102DD0000000002090B189B10B4AD2E8AF3F5B07F9
:102DE0000FD50378883AC3EBC3039818D3580B6008
:102DF00083888B80837900208B7170476FF015007A
:102E000070476FF00A0070478800002010B50A4C28
:102E1000E3790BB1002010BDFFF70EFF0028FAD1B7
:102E2000E379002BF6D1FFF717FF0028F3D1601CE0
:102E3000BDE81040FFF714BE00000020F0B5274B9E
:102E4000064693F891300D469B0687B03DD518B9DC
:102E50006FF0150007B0F0BD00F118070F213846DC
:102E600008F091FA0028F3D00E21384608F08BFACA
:102E7000A8422DD04FF0FF304FF0FF31FFF728FA76
:102E8000044640B302210C3008F034F900220280DD
:102E900072780346427055B1012210210270384603
:102EA00008F071FA18B11A7842F002021A703A4624
:102EB000204603A90E230095FFF7F8F900222146CA
:102EC0004FF40150FFF788FAC4E76FF08500C1E7BF
:102ED0006FF07700BEE76FF06800BBE700000020EE
:102EE00000232DE9F04F074615461C468BB0019193
:102EF00051688B4214D1FB2C1AD9082107F1180014
:102F000008F041FA002840F0CA80664BB3F8A030C0
:102F10009C427FD96FF0200420460BB0BDE8F08FB3
:102F20002A6802EBC3025278013302321444E0E70C
:102F30005C4BB3F8A0309C42ECD80B2107F1180091
:102F400008F021FA10B91F2C28BF1F244FF0FF30C2
:102F50004FF0FF31FFF7BCF904F104098046002867
:102F600055D049460C3008F0C5F84FF0000B064626
:102F70004A46D94600210AF058FDD5F800A0331D75
:102F80006A6893450FD386F803907B7800223370EC
:102F900003234146737001230198B3700BB0BDE861
:102FA000F04FFFF719BA9AF8012009F102008118D1
:102FB0008C429AF800C008D2BCF1090FA4EB0002C1
:102FC0001FD1002A1DDD4FF0080CD1B20291013152
:102FD00003F8091009F10101C9B203F801C0DAF8D8
:102FE000041053FA80F003930AF0F8FC029B0BF1F3
:102FF000010B9A1C4A44039B5FFA82F90AF1080A02
:10300000BEE74046FEF70AFE6FF0150484E76FF056
:10301000680481E7294604A808F024FA0446002839
:103020007FF47AAF4FF001090546099A002A3FF470
:1030300073AFFB2A28BFFB224FF0FF304FF0FF3168
:103040009246161DFFF744F9804620B331460C30F6
:1030500008F050F87B78064603708570011D5FFA12
:103060008AF204A808F0A0F9099BF070B9F1000FEA
:103070000CD0002B0CBF03230123002241460198F2
:103080007370FFF7A9F940B98146CEE7B3FA83F32D
:103090005B095B00F1E76FF0680004463CE76FF006
:1030A0000A0439E700000020F8B5046906464568BF
:1030B00044B140F203432B403BD005F48263B3F5A7
:1030C000806F36D015F4806302D115F4F84F30D1FB
:1030D000194F3078FB7983422BD9C0EBC00007220F
:1030E000164938440AF0A9FCA8B115F0030306D12B
:1030F00097F82420082A02D8B2689F2A19D915F017
:10310000300F09D0ACB1EA060AD405F46035B5F544
:10311000603018BF0120F8BDEB0601D4002CF4D1BB
:10312000D6E902239A4204D81F2A02D9B3F5804F68
:10313000EBD90020EFE700BF0000002047EB0000C4
:1031400038B50D4DD5E8AF4F14F0010412D1A5F1FB
:1031500018031846582221460AF067FC0346D5E8B2
:10316000EF2F42F00102C5E8E12F0029F7D1184600
:103170005C7038BD0020FCE7F80900202DE9F3471A
:10318000D1F810900D4649689046B9F1000218BF79
:10319000012201650DF103030646FFF7B3FD044666
:1031A000002840F0EA8006F10F03B9F1000F00F0AB
:1031B00089802A6911684FF0FF30C6F80F10918896
:1031C000998092794FF0FF319A71FFF781F882462A
:1031D000002800F0F58019210C3007F08BFF044621
:1031E000002119220AF021FC73782370AB68E37088
:1031F000C3F307221B0C22716371EB68A371C3F345
:1032000007221B0C2372E2716A6812F4004F0CBF94
:1032100007230623D10348BF03F00503920348BFE9
:1032200003F0FB0363729DF80330A3727F23E37402
:10323000012323756B6803F44063B3F5806F14BFFB
:1032400001230223A3756B68DF0442BF03232375A8
:10325000A3756A6882F48063C3F3802350044FEA45
:10326000031348BF43F04003910444BF43F02003DD
:103270009BB2D70544BF012222766A6812F0030F81
:1032800002F4007100F0898043F00107BFB2B9F188
:10329000000F1ED0C1B143F003039BB2D1062969D0
:1032A00048BF43F00402086858BF43F00C02C4F85A
:1032B0000B00888892B2A4F80F0089791F466174C8
:1032C000134612E0404A75E7B8F1000FE3D13B46E0
:1032D000E4E7500555D521B143F003039BB21F46E7
:1032E00003E03B46B8F1000F53D16A785146E275CE
:1032F000AA7842F236006275A4F8013001AAFFF7FD
:103300006BF80446002838D1019806F11808C36804
:1033100093F90130B370FEF781FC0121404608F0BB
:10332000D6F86FF0100108F034F8C2063FD46A688E
:10333000092112F0030218BF0122404608F0B4F838
:103340000A214046C7F3400208F0AEF86A680C2133
:103350004046C2F3800208F0A7F86A680B21404695
:10336000C2F3802208F0A0F89DF803200321531E29
:103370005A4240465A4108F097F8204602B0BDE84C
:10338000F08743F003039BB20029A8D1B8F1000FE6
:10339000A5D043F002039BB204E00029F9D1B8F1B3
:1033A000000FF6D1B9F1000F7FF478AF97E7304600
:1033B00006F1090107F075FF0028B8D00446DCE7E4
:1033C0006FF06804D9E700BF47EB0000034BC01A59
:1033D000034BC0105843C0B2704700BFE009002043
:1033E000A38B2EBA20B90448D0E8AF3FDB0701D445
:1033F0000020704718387047F809002010B5054CB8
:10340000A06930B16FF00101183007F0C2FF00234E
:10341000A36110BD00000020F8B504460F46164613
:10342000154BD3E8AF3F5B071CD5F2B1FFF73CFE6D
:10343000D8B1FFF785FE0546D0B123782146037049
:1034400063780022C3704760FFF798FE044638B1E6
:103450006FF0010105F1180007F09BFF2046F8BD51
:103460003560FBE76FF00A04F8E76FF01504F5E745
:103470006FF00B04F2E700BF88000020F8B5354B71
:10348000074693F891200C46900603D46FF085050B
:103490002846F8BD17B96FF01505F9E707F11806CA
:1034A0000A21304607F06FFF0028F4D10921304689
:1034B00007F069FF0028EED10B21304607F063FFCB
:1034C0000028E8D02288052AE5D961889142E2D314
:1034D00093F89430D90602D463685A07D6D44FF0D3
:1034E000FF304FF0FF31FEF7F3FE054678B30721BA
:1034F0000C3007F0FFFD00220260C0F803207B784B
:10350000294603702388A0F801306388A0F80330AF
:103510006368C3F340039B01A0F8053042F23E000C
:10352000FEF75AFF05460028B2D163685B0708D54D
:103530001021304607F0CBFF0F21304607F0C7FFC0
:10354000A6E76FF48031304607F023FFF4E76FF011
:1035500068059DE70000002073B5C6687078FFF726
:1035600041FF044628B304F1180508F025F86FF46C
:103570008071284607F00DFF6FF08001284607F0A4
:1035800008FF03060CD5204607F0F3FE63683BB145
:103590001B682BB13279204601A98DF80420984789
:1035A000054B9B699C4204D102B0BDE87040FFF717
:1035B00025BF02B070BD00BF000000202DE9F3411F
:1035C000002142F2580001AAFEF706FF044670B936
:1035D0000198C3685F789D7893F803801E79FEF7A1
:1035E0001DFB054B83F802801F70DE705D70204666
:1035F00002B0BDE8F08100BFB32500202DE9F843FB
:103600003D4A804692F892300C461D0770D500F175
:103610001806D6E8AF3F98070AD5D6E8AF3F59035A
:1036200006D46378022B07D192F892309B0624D4FB
:103630006FF01500BDE8F883042B23D192F8923087
:1036400013F0200FF4D0E378023B492BF0D86368E5
:10365000002BEDD02378023B122BE9D8A378013B55
:103660000F2BE5D84FF0FF304FF0FF31FEF730FE63
:10367000074650B96FF06800DCE7204B1B7813F069
:10368000010FDFE7012BE5D0D2E700F10C0905219E
:10369000484607F02FFD98F801300546037023785F
:1036A00043706378013BDBB2032B8EBFFF23144AC8
:1036B000D35C8370A378C370E17839B1484607F0D2
:1036C00019FD6168E2780AF089F9E1782971002230
:1036D000394642F25100FEF77FFE0028AAD1D6E813
:1036E000EF3F43F40033C6E8E23F002AA2D0F6E7FA
:1036F0006FF085009EE700BF00000020B32500208A
:103700007DEC00002DE9F74F1746D2F810A00278A3
:103710000646042A0D4601F1FF3325D0052A78D04C
:10372000022A4DD1032B4BD9002200230820FEF79B
:10373000E3FB0446002843D00422D6F8013000F110
:103740000C0840460DEB0201019307F0D9FCBDF8CF
:103750000630053D9D424BD1404607F019FD85429C
:1037600046D82A46711D49E0012B29D943783E2BC2
:103770002CD1C378022B26D00D2B27D10379012B16
:1037800024D1B0F805B0CBF3001BB6F80130033DEF
:10379000B5EB132FADF8043012D1BBF1000F18D0E8
:1037A0004FF000084FF0000942464B4659469DF83D
:1037B0000400FEF7B9FB044670B9BBF1000FF3D06B
:1037C00003B0BDE8F08F4FF0010BDEE74FF0000BC8
:1037D000DBE74FF4A028E5E700F10C08022201A97D
:1037E000404607F08DFC404607F0D2FC854203D9E5
:1037F0002046FEF713FAE3E72A46F11C404607F09D
:103800007FFC21463846DAF8003003B0BDE8F04FBF
:103810001847032BD4D9002200232020FEF76CFB8D
:10382000DFF83890044698B10422D6F8013000F150
:103830000C0840460DEB0201019307F061FC0023E8
:10384000C9F80030BDF80630053DC3F30D0381E72C
:10385000D9F800300133C9F80030B1E73413002043
:10386000102208B5034B0120C3F84024FEF7F2FAFA
:10387000002008BD00300050084B70B5C31A0D463B
:1038800007499B10044659434022064807F0E3FFCE
:103890002B4601462046BDE8704018474C130020D7
:1038A000B76DDBB648DC0000402373B50B4C0093CA
:1038B000041B0B460D460A49A41061430646094AFB
:1038C000094807F0F4FF011E05DA30462B4602B026
:1038D000BDE87040184702B070BD00BF4C13002017
:1038E000B76DDBB619B9000048DC00002DE9F047E0
:1038F0000022012107460520FDF7ECFD124800F0EB
:10390000C5FF0446D0B900F0F5FF25464FF01C0A6C
:103910004FF00C08DFF834903E6949460AFB056019
:1039200007F026F8031E0CDB012308FB05661D4487
:10393000042DB367F0D12046BDE8F0876FF0040492
:10394000F9E71C46F7E700BF853A0000F0E1000008
:103950007FB500220123CDE9022304ABCDE9043376
:10396000094A6B46CDF800D0CDF804D007F0CDFF62
:10397000002805DB4FF480420023684602F02EFA4F
:1039800007B05DF804FB00BF43B9000010B5EFF3CA
:103990001184202383F31288BFF36F8F074A1368C3
:1039A00023F00201DB07116002D4012008F043FA82
:1039B00084F31188BFF36F8F10BD00BFEC1300209C
:1039C0000C22104B014602FB0033002030B4D3E937
:1039D0001C521867EFF31180202484F31288BFF380
:1039E0006F8F9C6F04F0C00444F002049C6780F366
:1039F0001188BFF36F8F1DB12B4630BC02481847AA
:103A000030BC70474C13002048DC000010B4EFF3CA
:103A10001182202383F31288BFF36F8F1748016848
:103A200041F002040460C80707D482F31188BFF391
:103A30006F8F012010BC08F0EFB94FF05021D1F882
:103A40000C04D1F80C14C907EFD5EFF3118083F300
:103A50001288BFF36F8F0A498B6F03F0C00343F0E6
:103A600002038B6780F31188BFF36F8F82F3118895
:103A7000BFF36F8F002010BCFFF7A2BFEC13002034
:103A80004C130020092813D8DFE800F005101212AB
:103A9000121212120E0C074B986F10F0070007D18C
:103AA000FFF78EBF0220FBE70320F9E70120F7E7CD
:103AB000704700BF4C1300202DE9F041012207465A
:103AC0003649D1E8EF3FC1E8E02F0028F9D133B9FA
:103AD000334934484B60CB608A6006F05CFF7B1E44
:103AE000012B2BD8012F07D14FF05023D3F81C34D2
:103AF00003F00303022B21D009F038FD0546F8B985
:103B0000294B1B78E3B14FF0502302220646C3F83D
:103B100008234FF05024DFF89480D4F81824D4F808
:103B20001834D20315D503F00303022B01D0012F63
:103B30000FD16DB386F31188BFF36F8FBDE8F081AD
:103B4000EFF31186202383F31288BFF36F8F0125D3
:103B5000DFE7C5B1304607F04DFAD4F81835DBB2CF
:103B6000012BDAD1D4F80421002AD6D00022C4F8DF
:103B70000421D4F804210222C4F818252022C8F810
:103B80008021A360C9E70021212009F08BFDE4E733
:103B90004FF050230222C3F80423CFE7481300203C
:103BA0003813002068130020B927002000E100E04E
:103BB00008B5074809F0B6FA38B10648FDF74CFFDA
:103BC0000448FCF7CDFB002008BD6FF01200FBE7B6
:103BD000D4DC0000D93B00000A2838B50446074D64
:103BE00004D1AB680D2128465B689847AB68034851
:103BF0005B68E1B29847204638BD00BFD4DC0000C6
:103C0000F0B544681646A068227C01F01F0587B015
:103C100045EA421500286CD0B6F5001F04D12946AC
:103C200008F040FC002055E06268607CB6F5800F2B
:103C300050624FF0000001AA0190506037D1B3F1FB
:103C4000007F14BF052304238DF804300023CDE941
:103C500004230393E3680DF1030723FA01F111F044
:103C6000010139D1B6F1A07F36D105F01F036A09F1
:103C700003F1800326D0012A3ED1214A52F8233095
:103C8000DB0729D43A462946A06808F09EFB163087
:103C90001AD002972946A06803AA08F062FA002801
:103CA00018DB01222946A06808F0AAFBBAE7B3F1A5
:103CB000C06F05D0B3F1007F14BF01230223C3E717
:103CC0000323C1E70F4AD9E73946A06801F038F865
:103CD0000028DEDA07B0F0BD3A462946A06808F0B1
:103CE00074FB0028D6D19DF80310A06801F01EF8DF
:103CF000D0E76FF08500EDE751F82330FFDE00BF1D
:103D000000288450002584504209034670B502D033
:103D1000012A17D070BD0D4E326951680029F9D0C3
:103D2000012503F01F030C689D400029F2D08A682A
:103D30002A4002D030464B6898472CB12368214670
:103D40001C46F2E7024EE7E72346F8E780DC000076
:103D500064DC000038B54568A86890B108F048FBFD
:103D6000014670B9A86800F0AFFF044658B9024692
:103D70000649A86808F026FB224605210D20FDF71C
:103D8000A9FB002038BD6FF00400FBE7093D0000EF
:103D90002DE9F04340F206364768D00648BF4FF0A1
:103DA000030C3B7C02EA060658BFC2F3401C87B0F6
:103DB00001F01F05B6F5837F144645EA43158DF8DB
:103DC00003C044D00DD8062E16D005D8A6B1022EB9
:103DD0003FD06FF0150037E0B6F5807FF9D10126AE
:103DE0000AE040F20222964235D0B6F5407F34D048
:103DF000B6F5007FEDD102260123220303FA01F17B
:103E00002DD57B689960B86880BB05F01F036D09EC
:103E10002AD0012D73D13C4A02EB830284F4803313
:103E2000D2F80012C3F30043C4F3404444EA43040D
:103E300021F4706144EA8C0421F00F0144EA062366
:103E40000B43C2F80032002007B0BDE8F08307261C
:103E5000D2E70426D0E70526CEE70326CCE76303A6
:103E600044BF7B68D960CEE7284AD5E729460DF1E3
:103E7000020208F0AAFA14F4403F80460CD1294609
:103E8000B86808F0BBFAB8F1000FDCD19DF8021059
:103E9000B86800F04BFFD6E74FF0000901ABCDE961
:103EA0000199CDE90439CDF80C902946B86803AAE8
:103EB00008F057F94845C6DB14F4003314D09DF8D8
:103EC000033084F48034C4F300448DF80E308DF850
:103ED0000C608DF80D404B462946B86803AA08F0DF
:103EE000F8F90028CFDAAEE7CDE904330DF103038A
:103EF00003932946B86803AA08F033F9F1E7803341
:103F000050F82330FFDE00BF002884500025845085
:103F100010B504460269A2B0C2F88000164900201C
:103F200001F004F8002201212A20FDF7D3FA8422AF
:103F3000002101A8646809F078FD0023012001AA8E
:103F400061680432D940C90744BF00FA03F142F85E
:103F5000041C2168D940C90748BF00FA03F103F1E6
:103F6000010348BFD163102BEAD101A800F0F2FF92
:103F7000002022B010BD00BF55BA0000036803F056
:103F80001F025B09026004D0012B034818BF002008
:103F900070470248704700BF0028845000258450B5
:103FA0002DE9F04F1546824640F2FF19DFF8B0B117
:103FB00085B000EB8108D04503D1002005B0BDE8F5
:103FC000F08FDAF80030C3F3C3210829C3F30804E3
:103FD00000F2C080634A4C45515C4FEA136311D034
:103FE000222B1DD94E2B40F0B880C5F81445012670
:103FF00003A80394FFF7C2FF039B06FA03F3836051
:10400000374654E0222B09D94E2B40F0A6804FF0C2
:10401000FF33C5F814350AF1040ACCE74FF0FF343A
:10402000222B00F29A80DFE803F012171E362127B8
:1040300036989898983963989898989898989898F6
:104040006B76797C9898987F86898C8F9200C5F8DA
:104050000C45631CCBD1DEE7C5F81445631CDAD0F0
:104060000026002723E0C5F80845F2E7601CC5F8E4
:104070000845D0D0002604E0621CC5F80C45CAD023
:104080000126012703A80394FFF778FF039B07FA93
:1040900003F3C3600BE0C5F81045DFE7C5F808453A
:1040A0000029DBD1671CB6D0002606213746DAF896
:1040B0000030039403F40040002803A81CBF01262D
:1040C00000270193FFF75AFF039C019B00EB84003C
:1040D000D0F80042C3F3412C0B0243EA8C033B436C
:1040E00004EA0B04234343EA4603C0F8003292E794
:1040F000C5F80C450029D5D0661C8CD000267FE77A
:10410000C5F86045601CDAF8003084D0C3F3004382
:10411000002BB5D06BE7C5F86445F3E7C5F86845F3
:10412000F0E7C5F86C45EDE7C5F82445621C3FF49F
:1041300072AF012695E7C5F828458AE7C5F83045EE
:10414000F4E7C5F83445F1E7C5F83845EEE7C5F8BA
:104150003C457EE76FF0150030E76FF085002DE7F6
:10416000F0F0FCFFE5EC00002DE9F04104460D46BF
:10417000476809F0FBF988B14FF02008EFF311868A
:10418000314688F31288BFF36F8F606807F002FD35
:1041900050BB86F31188BFF36F8FEFE71F4B1B787F
:1041A000002BE9D04FF020086426606807F0F2FC8D
:1041B00070B9012007F0DCFD013EF6D1002121207D
:1041C00009F070FAF0E786F31188BFF36F8FF5E717
:1041D000EFF31186314688F31288BFF36F8F606862
:1041E00007F0D8FC0028EED0FB6900201D70636842
:1041F000FA691B68C3F844250122C3F84825C3F8AF
:104200002001D3F82041C3F85801D3F858019A602F
:1042100081F31188BFF36F8FBDE8F081B9270020CB
:104220000123834070B5DC430B4AD2E8EF1F01EA5B
:104230000405C2E8E65F002EF7D14FF480328240D9
:104240000648C0F80823BFF35F8FBFF36F8F0B42A0
:1042500014BF0120002070BDA014002000500150A8
:1042600070B40E4922F07F46D1E90034D01AC31849
:1042700044F10004C1E90034A6F50013B3F5400F82
:1042800009D2074B1B681A0A1B069C19054B42F101
:104290000005C3E9004570BC02F0CABC480A002012
:1042A000A4140020500A0020D9B101230D4A8340F4
:1042B000D2E8EFCF4CEA030CC2E8E1CF0029F7D1F6
:1042C0004FF48033084A8340C2F80433074BD3E8E5
:1042D000AF3FC340DB0742BF4FF40012044BC3F8AB
:1042E00000217047A0140020005001509C140020B1
:1042F00000E100E00D4B1868010A0006BFF35F8F74
:104300000B4BD3F80435181841F10001B3F5801FA9
:104310000AD2084BD3E90023904271EB030303D286
:1043200010F1807041F10001704700BFA41400201B
:1043300000500150500A00202DE9F04F85B016467C
:104340001F4604469DF840A0FFF76AFF0190FFF763
:10435000D1FFB04271EB070352D23B4B301A67EBEF
:104360000101984271F100014DD2384B03EB041367
:10437000D3E902239F4208BF964258D04FF48038B9
:10438000334908FA04F8204626F07F4BC1F84883E9
:1043900007F0BCFC4FF00309584604F15005AD008E
:1043A000ADB205F1502504F5A87305F580350293EB
:1043B000029A20F07F4341F82230C1F84483D1F8BB
:1043C0000435244AC01A033820F07F4090422ED989
:1043D000286868B1D1F80435A3EB0B0020F07F40CA
:1043E000B0F5000F039322D9204607F08FFC039B02
:1043F000BAF1000F07D109EB030009F10109D7E772
:10440000BAF1000F09D06FF0150520460199FFF7AA
:104410004BFF284605B0BDE8F08F01230E4AA340AC
:10442000D2E8EF0F1843C2E8E10F0029F8D107499D
:104430000E982301C8500F9B01EB04120025C2E91E
:1044400002675360E1E700BF01008000380A0020E6
:1044500000500150FDFF7F009C1400207FB5002517
:104460004FF0FF304FF0FF31194C1A4B0226C4F8C1
:104470000833C4F84833184BC4F80855C3E902019F
:104480004FF480334FF40012C4F80433134B01216E
:10449000C4F804631520C3F880212A46FDF71AF8F2
:1044A0001520FCF7E7FF01230D4AA360236013608A
:1044B0000C4B0D4A009328460023CDE90155FFF728
:1044C0003BFF3046FFF7F8FA284604B070BD00BF46
:1044D0000050015003000F00380A002000E100E006
:1044E000A014002061420000FFFF7F002DE9F74388
:1044F0002E4BD3F8042390070BD5D3F8042142B1F7
:104500000022C3F804212A4AD3F804311368013386
:104510001360264AD2F80433D90326D5254BD3E8B5
:10452000EF1F21F00100C3E8E40F002CF7D1CB0707
:1045300002D4D2F84031C3B100251C4CC4F840511C
:10454000D4F84031FFF7D6FEEFF31182202383F336
:104550001288BFF36F8F184BD3E90267B042B9419D
:1045600006D282F31188BFF36F8F03B0BDE8F083EA
:104570004FF0FF38D3E900104FF0FF391D60C3E959
:1045800002894FF48033C4F84833C4F84051D4F85A
:10459000403182F31188BFF36F8F0029E5D000907E
:1045A00032463B4628468847DFE700BF00500150AF
:1045B000A41400209C140020380A002030B5431CAD
:1045C000124C85B005D08442A8BF0446012CB8BF68
:1045D0000124FFF78FFE0E4B0C4DD3E90013401A58
:1045E000B0F5000F0FD22218AA4228BF2A46002099
:1045F00052180849CDE90100009143F10003FFF78B
:104600009BFE05B030BD2A46F1E700BFFFFF7F00EB
:10461000480A00206142000008B5FFF76BFE024B1C
:104620001B68C01A08BD00BF480A00204FF4007183
:10463000014802F04BBD00BFB92500204FF47F03B5
:10464000D3F83021D3F83431072A05D1023B032BAC
:1046500002D8024AD05C70470020704700ED00008D
:1046600008B5FFF7EBFF58B1644BD3F8202A3AB9ED
:104670000D21C3F8201A0121C3F81C19C3F81C2905
:104680000022D30003F57F03D3F80013013107D0D4
:10469000D3F800130132D3F80433202A0B60F0D191
:1046A000FFF7CCFF002840F0A080FFF7C7FF40B124
:1046B000534B544AC3F830254FF050230122C3F81E
:1046C00058254FF47F03D3F83021D3F83431072A2B
:1046D00009D1023B032B06D84B4AD35C1BB1002205
:1046E0004A4BC3F84C25FFF7A9FF50B14FF05023B8
:1046F000D3F80024D10742BF0022C3F81421C3F825
:1047000018214FF47F03D3F83021D3F83431072A2E
:1047100009D14FF05023D3F80024D20744BF6FF0E3
:104720000102C3F80024FFF789FF18B16522334B5B
:10473000C3F80C274FF47F03D3F83021D3F834317A
:10474000072A16D1314BD3F82034002B11DA4FF061
:1047500050230322C3F8182501229A60D3F80421BC
:10476000002AFBD00022C3F804210122DA60C3F83A
:1047700018254FF47F03D3F83021D3F83431072ABA
:1047800023D1023B032B02D8214AD35CEBB17E221A
:104790001A4B1B49C3F80C27C3F83C297F231D4A39
:1047A000C2F818310023C1F8043EC1F8083E01F5F3
:1047B0004821C1F81031C2F82431C2F82C3102F579
:1047C000FF1202F58052C2F8A032134AD2F88C30A0
:1047D00043F44063C2F88C30104A114B1168C3F89F
:1047E0004415D269C3F84C2508BD2922034BC3F8F0
:1047F0000C270322C3F83C2757E700BF00400050B6
:10480000009003504400EFBEFCEC00000020035079
:10481000F8EC00000020005000ED00E00080FF00F8
:1048200000600050014B1860704700BFA8140020C2
:1048300010B5054B1446186807F09CFA0028A4BF71
:104840002070002010BD00BFA81400200123024AE0
:104850008340C2F80435704700700150014B0020BE
:104860001B681847AC140020014B1B68184700BF99
:10487000AC140020014B09201B681847AC14002021
:10488000014B08201B681847AC14002010B5144CCD
:10489000237913BB01232371124B0028206018BF1A
:1048A000184600F037F8D0B923680F48002B08BF2E
:1048B000184600F0B9F890B923680C48002B08BFDF
:1048C000184600F0F9F850B923680948002B08BFD2
:1048D0001846BDE8104000F063B86FF0770010BDD7
:1048E000AC1400205D4800007548000069480000D5
:1048F0008148000008B5064B1B6843B10520FCF752
:10490000DBFD20B9BDE808400520FCF7B3BD08BDBC
:10491000AC140020074B0246187938B91A600122FE
:104920001A714FF05023C3F8142570476FF07700C9
:10493000704700BFB41400204FF050230022C3F88A
:104940000021D3F80021012208491A60096811B139
:10495000C3F804237047D3F80021002AFBD00022BB
:10496000C3F80021D3F80031704700BFB414002011
:104970004FF05023D3F80423D2070DD5D3F80021EC
:1049800052B10022C3F80021D3F800210122C3F85C
:104990000823024B1B681847704700BFB41400205F
:1049A000054B0246187918B91A6001221A7170472E
:1049B0006FF07700704700BFBC1400204FF0502309
:1049C0000022C3F82021D3F8202101229A61094A4C
:1049D000126822B14FF48072C3F804237047D3F8F1
:1049E0002021002AFBD00022C3F82021D3F8203157
:1049F000704700BFBC1400204FF05023D3F80423AD
:104A0000D2050ED5D3F820215AB10022C3F82021B7
:104A1000D3F820214FF48072C3F80823014B1B68A0
:104A200018477047BC140020074B0246187938B964
:104A30001A6001221A714FF05023C3F88025704785
:104A40006FF07700704700BFC41400204FF0502370
:104A50000022C3F82421D3F8242101221A62094A32
:104A6000126822B14FF40072C3F804237047D3F8E0
:104A70002421002AFBD00022C3F82421D3F82431BA
:104A8000704700BFC41400204FF05023D3F8042314
:104A900092050ED5D3F824215AB10022C3F824215F
:104AA000D3F824214FF40072C3F80823014B1B688C
:104AB00018477047C4140020074B0246187938B9CC
:104AC0001A6001221A714FF05023C3F8182570475D
:104AD0006FF07700704700BFCC1400204FF05023D8
:104AE00010B5D3F818141E4C11F4803FD3F81824D5
:104AF0001AD002F00302022A04D0012A01D007F0E2
:104B00000AFA01224FF05023C3F818250022C3F8F7
:104B10000421D3F8042101229A6022688AB9D3F8CB
:104B20000421002AFBD014E0D3F81424D207E8D5DE
:104B3000D3F81C2402F00302013A012ADFD82268CC
:104B40001AB10222C3F8042310BDD3F80421002AAD
:104B5000FBD00022C3F80421D3F80431F4E700BFEE
:104B6000CC140020F8B54FF0502301250026D3F8CF
:104B70000443184F04F0820404B9F8BDB4FA84F079
:104B8000C0F11F00830003F580739BB203F1502333
:104B9000196805FA00F224EA02040029ECD01E602C
:104BA0001B684FF050230128C3F808230ED1D3F817
:104BB0001824D3F8182402F00302012A06D1022196
:104BC000C3F81815C3F804139A60D5E73B68C0B260
:104BD0009847D1E7CC140020036803F01F025B095B
:104BE000026004D0012B034818BF00207047024820
:104BF000704700BF0028845000258450034A4309B1
:104C0000D35C00F01F001844C0B2704704ED0000F0
:104C1000034611F0010010B5CCB20BD1A207C4F3CA
:104C200040000DD5074A106A58601062003818BF5E
:104C3000012005E004490A6A1A600A62002AEDD0E0
:104C400010BD00BF0028845000258450F7B50446ED
:104C50000846FFF7D3FF06B204EB4606B38A0D46BB
:104C6000DB072BD5204607F059FA2946204607F0E6
:104C7000C5F958B1204607F0D7F90022276800B2DD
:104C800007EB8003C3F81025C3F8102529462046FA
:104C900007F0F3F9002101A8B1820195FFF79CFF0D
:104CA000019B00EB8300D0F80022064B134043F039
:104CB0000203C0F80032084603B0F0BD6FF01500E3
:104CC000FAE700BFF0F0FCFF70B590F88C400546A5
:104CD00090F88D6024BB21466022143008F0A5FEB8
:104CE0002146114B286853F836608E420ED10024BD
:104CF000C0F87C41D0F87C3140F30730FCF7BAFBB8
:104D00000123204685F88C30AB6770BDCBB29B0089
:104D100003F580727C2B04BF845083580131E4E793
:104D20006FF07700F1E700BF94E2000090F88D008B
:104D3000024B03EB800007F037B800BF6802002089
:104D400010B5064B90F88D000C4603EB800007F081
:104D500011F80028A4BF2070002010BD68020020B8
:104D60002DE9F04F814659F804BB90F88D40DBF8EF
:104D700004136B4BC9B2804653F8342058468BB0AD
:104D800041F0004107F0A3F9051E36DA0023CDE912
:104D90000833634B08A803EBC4035B68194601930F
:104DA000FFF736FF042303EBC40303935D4B0DF1C0
:104DB000200A02930023029A009312F8013B5849FB
:104DC0000292039A02EBD3028A5C03F0070322FAF1
:104DD00003F3DA0719D4009B0AF1040A9BB14FF0E0
:104DE00000410022584607F072F9019908A8FFF720
:104DF0000FFF0028DAD125F000450124002D78D1DD
:104E00000BB0BDE8F08F0123D5E7009B464A134461
:104E10000493DAF800100029DDD091FAA1F1B1FA7B
:104E200081F1049B1C7841EA44142046FFF7E6FE1A
:104E300008EB4000878AC808BB08059301231AF8CD
:104E4000002001F0070103FA01F122EA01020AF849
:104E5000002007A80794FFF7BFFE079A059B803242
:104E600050F82220C7F382065B073746C2F301429F
:104E700023D54846D6B221463A4607F0DFF807A8C0
:104E80000794FFF7A9FE079B803350F82330C3F344
:104E900001439E4207D10021204607F0A0F8314689
:104EA000204607F09CF807A80794FFF795FE01221B
:104EB000079B02FA03F30362ABE7022A0DD1032139
:104EC000204607F08CF806F00503012BEBD13A469B
:104ED0002146484607F0B2F8E5E702212046059250
:104EE00007F07DF8032EF2D0059A032ADBD1022EBB
:104EF000ECE795FAA5F3B3FA83F304FA03F225EA93
:104F0000020503F5A2725BF8222008EB4303484632
:104F1000B3F87C10C2F3014207F090F86EE700BFCF
:104F200094E2000014ED000014ED0000F8B5084D07
:104F30000F462C79164644B92A20FCF79BFA012328
:104F400020462B712F60AE60F8BD6FF07700FBE755
:104F5000D4140020002330B50D4A50F8234003F547
:104F6000A2710133102B42F82140F6D10023084AE8
:104F700000F13C0103F5B27451F8045F0133102BCA
:104F800042F82450F6D1D0F88030C2F8043330BD56
:104F900000A002500123024A8340C2F80433704744
:104FA00000A002500123024A8340C2F80833704730
:104FB00000A00250F8B5012600270B4B0B4DD3F88B
:104FC0000C4304B9F8BD94FAA4F0B0FA80F006FAE4
:104FD00000F324EA0304064B82009F502B68002B49
:104FE000EFD0A9689847ECE700A00250D414002045
:104FF00000A102502DE9F0410E4617460C4D55F820
:105000001C4FAC4203D16FF01200BDE8F081314675
:1050100054F8440CA4F14408FBF79CF830B9C7F8E5
:1050200000804046BDE8F04107F00EBB2468E8E789
:10503000E014002010B5D0E909124A60416A00F17D
:1050400024031160C0E909334368044603B198475B
:10505000054A936833B11279062A03D907202268DA
:1050600002499847002010BDE014002016ED000012
:105070002DE9F04107460D460B4E56F80C4FB44251
:1050800002D16FF001000AE0394654F8240CA4F173
:105090002408FBF75FF820B91DB1C5F80080BDE812
:1050A000F0812468EBE700BFE014002038B5044627
:1050B00000B30068F0B10378E3B10021FFF7D8FF37
:1050C000D8B104F11C03C4E907330D4B04F12402E9
:1050D000196903F10C00A16260621A610A609D689F
:1050E00035B11B79062B03D9072022680549A8474B
:1050F000002038BD6FF01500FBE76FF01000F8E7F7
:10510000E014002018ED000038B5114C0546216868
:1051100019B100200131216038BD2422204608F059
:1051200084FC2B682846A3602B79237104F10C03BF
:10513000C4E9033304F11403C4E9053304F11C0387
:10514000C4E9073300F018F80028E5D12168E0E74A
:10515000E014002038B5074D2C68013C2C6044B9A0
:1051600000F012F821462846BDE83840242208F015
:105170005CBC38BDE014002008B50248FFF796FF7C
:10518000002008BD700200200148FFF753BF00BF98
:10519000700200200EB4431E062B33B588BF0020DA
:1051A000094B05AC54F8045B53F82010074805F090
:1051B00076FB214628460194FBF7D8F802B0BDE8FB
:1051C000304003B0704700BFA4E2000033ED0000A0
:1051D0002DE9F04F87B017469B460446DDF840A006
:1051E00000284BD0056A35B12D6825B1AC4607B013
:1051F000BDE8F04F6047E36A9F4242D80026BE42B6
:1052000003D1002007B0BDE8F08F182303FB06F898
:10521000D4F83090A26909EB08052B1D0593CAB993
:10522000686969680368B5F80CC0C91AAB680CF105
:10523000030E5D1E05EB0C155B4205EB4E051D4094
:1052400005EBCC0385680633A94228BF4FF0FF3138
:1052500007F0C7F959F8083020460293236AB1B223
:105260009B6A01935AF8263000935BF82620059B31
:1052700007F02FFA0028C5D10136C0E76FF01500FE
:10528000C0E70148BEE700BF40F4FFFF10B5044689
:1052900090B1028D43899A4209D0084A936833B18C
:1052A0001279032A03D94268054904209847204609
:1052B000BDE8104008F03DBB10BD00BFE014002069
:1052C000CEED000030B544898C4212D9436A013CCE
:1052D0005D882C4003EBC40359609A60BFF35B8F79
:1052E000426A538801335380438D01334385002044
:1052F00030BD0148FCE700BF41F4FFFF70B4039EDE
:10530000144660B1006A50B14BB1013407D0002E91
:1053100005DBD0F8844014B1A44670BC6047014856
:1053200070BC70472DF8FFFF70B4039E144660B147
:10533000006A50B14BB1013407D0002E05DBD0F824
:10534000944014B1A44670BC6047014870BC7047DB
:105350002DF8FFFF2DE9FF47DDF834800E4691461A
:105360009A460546002876D0002974D0B8F1000F7F
:1053700071D001F16407384607F016FBBAF1FF3F20
:1053800049D1346E06F1500204F18000844204F0E9
:105390001F0C07D2C4F3411152F8211021FA0CF16D
:1053A000C90736D4012104F07F04600952F8203087
:1053B00004F5806A01FA0CF104F201440B4304F095
:1053C0007F0442F8203034666B6C4A4603930E9B90
:1053D0002946CDE901830C9B30460093534607F0E4
:1053E00092FB384600F0C0FC2C7874B196F8A440CB
:1053F0005CB1AB6A013330D10021284607F013FBC2
:10540000044610B1284607F0E4FA204604B0BDE88F
:10541000F0870134BAE7BAF5806FD5D3AAF5806377
:105420007F2B06F150010FD8580951F8204003F0A6
:105430001F0324FA03F2D2070BD4012202FA03F36A
:10544000234341F82030BFE7054C384600F08CFC80
:10545000DBE7044CF9E7024CD7E70024D5E700BFAF
:105460002DF8FFFF29F8FFFF08B583681A0C0AD151
:10547000094A93682BB11279022A02D903200749FD
:105480009847002008BDA3F5803383601B0C0CBF38
:1054900001200020F6E700BFE0140020F0ED00003E
:1054A00038B50446E0B100F16405284607F07CFBFE
:1054B000D4F8B4309B6953B9D4F8A840103C002C00
:1054C00000DC084C284607F06DFB204638BD012B58
:1054D000F7D1D4F8BC0007F04FFAA0F11004EEE7C2
:1054E000014CF2E72EF8FFFF2DF8FFFF38B5044618
:1054F000E0B100F16405284607F056FBD4F8B4305B
:105500009B6953B9D4F8AC40103C002C00DC084C2B
:10551000284607F047FB204638BD012BF7D1D4F8C9
:10552000B80007F029FAA0F11004EEE7014CF2E709
:105530002EF8FFFF2DF8FFFF2DE9F04385B00F4651
:10554000904603A90D9A0546994607F0EEFC0446DD
:10555000E0B10C9E039BD5F8C0009E42A8BF1E463A
:105560000168D0F808C0611A33464A46614528BF31
:105570004FF0FF3106F0FBFF2346424639462846EE
:10558000009607F072FC05B0BDE8F0830048FAE72A
:105590002EF8FFFF2DE9F0478AB00D46DDE912979E
:1055A00016469846044620B9954E30460AB0BDE8E6
:1055B000F0870029F8D0002BF6D00021A822C0F8EF
:1055C000D01008F032FA012204F16400114607F00D
:1055D00008FF8C4BC4F8B450E667AC62C4F8843062
:1055E000894BC4F88830894BC4F88C30884BC4F898
:1055F0009030884BC4F89430874BC4F89830874B70
:10560000C4F89C30864BC4F8A030AB693BB9002F7E
:10561000CAD097E8070004F1A80383E80700AB6944
:10562000012B04D02B6A03BB6FF00506BDE7D4F84D
:10563000B400002800F0E080036A002BF4D09B68DF
:10564000002BF1D0984742060CD50021D4F8B400C5
:1056500007F098FA06460028A7D10021212008F07B
:1056600021F8E4E74307F8D5DCE71B69002BDBD022
:1056700028469847AB69012B04BF0023286100F03E
:10568000010008BF6B6184F8A400AB69DBB93B7A09
:10569000002B00F0838009F10C03C4F8C430B9F189
:1056A000000F81D0D9F80820002A00F0A3809B6861
:1056B000002B00F09F805B4B04935B4B05935B4B8F
:1056C00006935B4B0793AB69012B07D1564B0493B1
:1056D000544B0593564B0693544B0793002104F10A
:1056E000C803C4E9323306ABC4F8C0800222009379
:1056F0002846019104ABFFF76BFD064600287FF4B6
:1057000054AFAB693BB92B6B1B68C4F8B8302B6B3B
:105710009B69C4F8BC30AB69012B07D12B6B9B692B
:10572000C4F8B8302B6B1B68C4F8BC30D4F8BC008C
:1057300007F0BDF82B6B1B68C3F82C802B6B9B69A3
:10574000C3F82C80D5F818A0BAF1000F07D1D4F80F
:10575000AC300993D4F8B8305B89534520D894F81D
:10576000A430C4E9004463B100230293314B2046C6
:1057700001933523304A0394009304F1080107F0A4
:10578000C2F9AB69002B7FF410AF0421284607F063
:10579000F9F9074600283FF408AF26E04B467CE7BE
:1057A0004846D4F8AC1007F0B1FB0746E0B1D8F892
:1057B00000100890411AD8F808000022814228BF42
:1057C0004FF0FF31D4F8AC30404606F00AFF0097A6
:1057D00001230022D4F8B80008A906F0A7FF074665
:1057E00018B90AF1010AB5E7144F284607F0C3F9C2
:1057F0003E46DAE6114ED8E66FF01506D5E600BF54
:105800002DF8FFFF39550000FDCB00006BCD0000E7
:105810002BCF00006BCE0000B5CB0000ED54000094
:10582000A154000011EE000017EE00009FCD000013
:10583000A3CB000021CC00001DEE00002EF8FFFFDE
:10584000F0B505460E46174687B0074A03AC07CAAF
:1058500084E807000C9A3146009228463A460194A3
:10586000FFF798FE07B0F0BD38E0000038B5EFF361
:105870001185202383F31288BFF36F8F064B9C683A
:1058800007F063FC85F31188BFF36F8F2046BDE8F6
:105890003840FBF793BD00BF0415002038B50A4B14
:1058A00053F82040013053F82050A54200D838BDAD
:1058B000606830B1037EDB0701D407F01BFC0834BD
:1058C000F3E723689847FAE7C4E20000012270B5C5
:1058D0002A4B032086B01A70FFF7E0FFFCF71AFA94
:1058E00008F02EF80420FFF7D9FF254C254D264659
:1058F000AE4204F1300410D300F08EFE204C224E54
:10590000AC4226D300F09CFEFAF746FC1F4A137BFC
:1059100023F00103137306B070BD54F80C3C0593DB
:1059200054F8103C049354F8143C039354F8183C76
:10593000029354F81C3C019354F8203C009354E922
:105940000A2354E90C0100F03FFC54F8303C5E653A
:10595000CDE7D4E90A23B3F1FF3F08BFB2F1FF3F1F
:1059600005D052EA0301206803D100F025FF30344E
:10597000C6E73146183001F0CBF8F8E7B927002028
:105980006CDF00006CDF000067D60000100B002009
:10599000B82370B5144E86B003FB0066134B01228A
:1059A00005930F23CDE903320023CDE901331423FE
:1059B0004FF4A0720E4D0F4903FB0055044602FB45
:1059C00000110D4B3046009500F0FEFB737B2C74EC
:1059D00023F004037373094B013403EBC423EE601B
:1059E0006B6006B070BD00BF580A002020EE0000BA
:1059F00004150020203B002059D200002033002055
:105A0000BFB50020FFF74AFF294B03F5006282F380
:105A1000088883F30A880024E023264D264F85F862
:105A20002230EC772C766C76AC7685F820406B6A69
:105A300043F4E0236B6285F82340FBF739FCFBF766
:105A4000BFFD4FF0FF33AB62EB62FBF745FFFBF7A7
:105A5000DBFD1A4800F04AFCFCF73EF90120FFF795
:105A60001DFF0220164DFFF719FF00F01DFE154B1C
:105A700015495D61154B4FF40062059301232846DB
:105A8000CDE90343CDE901443B46009400F09CFB83
:105A900006466A7B284622F004026A7307F0A6FDD8
:105AA0002046FFF775FF3A4631462846FBF766FD6C
:105AB0002033002000ED00E0CD580000C80B00208E
:105AC000100B002004150020603C002025EE000093
:105AD00038B5064C064DAC4201D3002038BD2046F7
:105AE000D4E9011207F034FB1434F4E73803002042
:105AF0004C030020002038B5054C064DAC4200D3C5
:105B000038BD204607F048FB0028F9DB1C34F5E7D8
:105B1000380300203803002073B50C46EFF31181E1
:105B2000202585F31288BFF36F8FC5685DB12560AE
:105B30002B68C360836901338361002081F311887E
:105B4000BFF36F8F11E052EA030603D16FF00B0031
:105B50002560F3E7CDE900230246083000F0A2FCFF
:105B600018B9034B9B681B69236002B070BD00BF6E
:105B7000041500202DE9F341044617461E46EFF3B5
:105B80001188202383F31288BFF36F8FC368334AD1
:105B90007BB180689168884219D057EA060318D112
:105BA00088F31188BFF36F8F6FF00F0002B0BDE86C
:105BB000F081916891F90E100133E36093682161DF
:105BC000A36088F31188BFF36F8F0020EEE721698F
:105BD000F2E791F90E1090F90E306FF07E029942C3
:105BE000A8BF19469142B8BF11468B422DDD07F080
:105BF0003EFB054622464146CDE90076184800F0B6
:105C000051FC0028E1D0EFF31186202383F31288A2
:105C1000BFF36F8FA068D0B1236821699C420AD07E
:105C20004BB193F90E309942A8BF19466FF07E032D
:105C30009942B8BF194607F01AFB40B131460848EF
:105C400000F0C4FC6FF00A00B0E70025D2E7002D99
:105C5000F4D186F31188BFF36F8FF3E704150020AA
:105C6000BA270020F8B583680546002B40D0234AA8
:105C7000926893423FD1C368012B03D9013BC360B3
:105C80000020F8BDEFF31187202383F31288BFF3C0
:105C90006F8F0169806807F0EAFA2C68A54207D186
:105CA0000023C5E9023387F31188BFF36F8FE7E75D
:105CB000002CF5D0D4E90032002613605A60637BD3
:105CC000C4E9006623F002036373A66004F11800C0
:105CD00007F043FDAC6094F90E3020462B61C4F808
:105CE000B06007F083FC3946054800F06FFCC7E759
:105CF0006FF01500C5E74FF0FF30C2E70415002034
:105D0000BA27002037B51146EFF31185202282F320
:105D10001288BFF36F8F04689CB12368426823F038
:105D200003039442036008BF43600121204607F04B
:105D30002BFB044685F31188BFF36F8F204603B019
:105D400030BD51EA0302F5D000F10802CDE900139D
:105D50001046294600F0A6FB0028EFD1014B9B68B6
:105D60001C69EBE70415002070B5EFF311862023C2
:105D700083F31288BFF36F8F0468A0421BD0D4B1A5
:105D8000D4E90032002513605A60637BC4E90055F2
:105D900023F002036373A56004F1180007F0DDFC33
:105DA0002046C4F8B05007F021FC3146BDE87040F1
:105DB000094800F00BBCD0E902329A4218BF013307
:105DC00002218360103007F07DFD0028EDD186F3BD
:105DD0001188BFF36F8F70BDBA27002013B5EFF3A2
:105DE0001181202484F31288BFF36F8F846844B13B
:105DF000013C846081F31188BFF36F8F002002B0F3
:105E000010BD52EA030406D181F31188BFF36F8FEE
:105E10006FF00F00F3E7CDE900230246014800F0E0
:105E200041FBECE7BA2700202DE9FF41044620277B
:105E30004E4EEFF3118887F31288BFF36F8FD4F8BB
:105E4000BC50F5B9022104F1D40007F0DAFA0028B9
:105E500068D004F1CC0500220121284607F043FC5C
:105E60000028F8D100234FF0FF3202934FF0FF33A8
:105E70004146CDE900233E4804F1C40200F068FD2C
:105E8000D7E7D4F8C0202B689542C4F8BC3008BFCF
:105E9000C4F8C030D4F8D43043F00203C4F8D4308E
:105EA000EB6823F0040343F00103EB606B6888F3B5
:105EB0001188BFF36F8F28469847EFF3118887F357
:105EC0001288BFF36F8FEB68D80623F0010236D437
:105ED000EA60EB689A0716D5306823F00203EB609E
:105EE00088B10021036870B14268954235D10368DA
:105EF00069BB72683360824200D17360002340F84E
:105F0000083BFFF731FFD4F8D43023F00203C4F884
:105F1000D43088F31188BFF36F8FDB0589D400F08C
:105F2000CBFB86E7D4F8D430D9069BD5C4F8D4008F
:105F300088F31188BFF36F8F04B0BDE8F08123F0C0
:105F40001103EB6005F11000FFF70EFFC1E70B60D6
:105F50007368834208BF7160D0E723B11A680146B5
:105F600018461346BFE71A46F9E700BF2815002078
:105F7000BA270020F8B5C36804469A070F46C3F352
:105F800040062ED45B071CD40B680BB983680B60EA
:105F9000E368DD0742BFA36802263B603D6858BF47
:105FA0000126002D3CD0204B9A68D5F8B8309A4293
:105FB0000AD0D5F8D430D807C3F3800214D46FF0D8
:105FC000120600233B6025E007F0D0FAD5F8D43064
:105FD0000028F0D1D907C3F3C002F0D552B15B0756
:105FE00008D46FF00F06ECE7002AFAD1C3F3C00320
:105FF000002BF6D100232360D5F8C03063B9C5E982
:106000002F44284607F018FAE36843F00403E360DE
:106010003B68A3603046F8BD1C60C5F8C040F0E79F
:106020006FF01506CDE700BF04150020F8B5C36872
:10603000064603F00503002B0C4614BF012700277A
:106040001CD085680122002104F1100007F0C9F975
:106050002046134907F02AFAE36843F01003E3608F
:10606000F3685B0712D5336823606BB9D5F8C0308D
:1060700033B9C5E92F44284607F0DEF93846F8BDA4
:106080001C60C5F8C040F6E73460F4E7D5F8BC30D2
:106090002360D5F8C030C5F8BC40002BEBD1F0E749
:1060A00019D400000146014807F01CBAA00C0020DA
:1060B000F0B50446002089B0C4E92F000E9D04F11C
:1060C000C400C4E9310004F1CC00C4E9330055B385
:1060D0002879002840F2011008BF0120C4F8D4003C
:1060E00000204FF0FF364FF0FF37CDE90330CDE908
:1060F0000100CDE9066720460C4B009400F0CAF879
:1061000055B1296811B1204600F04EF86B791BB1EA
:10611000237B43F001032373204600F04DFBC4F8BA
:10612000B84009B0F0BD0120D8E700BF295E0000EB
:1061300030B50A46044685B0EFF31185202383F37A
:106140001288BFF36F8FD0F8D43013F0060F1DD133
:10615000B1B143F00C03C4F8D430204607F06CF919
:1061600000234FF0FF3202934FF0FF332946CDE971
:1061700000230C4804F1CC0200F0EAFB05B030BD6E
:10618000D0F8BC0048B143F00403E4E743F0040155
:10619000C0F8D410002AE0D0DBE785F31188BFF304
:1061A0006F8FEBE7BA27002010B5044608B9054BFE
:1061B0009C681F2204F1780007F061FC002084F83D
:1061C000970010BD041500202DE9F04F984685B0CA
:1061D00000F15803C0E91633129B00250373042312
:1061E000D61D26F007064373119B01EB060A0F46E6
:1061F000C0E90655514685608373C5730446DDF8D2
:1062000038B0DDF84C90FAF745FE109B073020F0CF
:106210000700C4E92676C4F8A00002930F9BAAEBFE
:106220000006CDE900B33246434639462046FBF727
:1062300089F90F9BC4E9198BE366109B6565236799
:10624000EFF31183202282F31288BFF36F8F104F78
:106250003A6A3C62626783F31188BFF36F8FB9F1CA
:10626000000F11D01F22494604F1780007F007FC07
:1062700084F89750BB680BB1D3F8A4303046C4F80B
:10628000A43005B0BDE8F08F84F87890F2E700BF45
:1062900004150020F0B5002587B00595109DDDE9B7
:1062A000127604950F9D044603950E9D02950D9D53
:1062B00001950C9D0095FFF787FFB6F1FF3F08BFE2
:1062C000B7F1FF3F05D056EA070305D1204600F09D
:1062D00073FA204607B0F0BD3A46334604F1180081
:1062E000014900F015FCF4E767D6000040F2011305
:1062F0008381002310B50446C0E9263300F05CFD1D
:10630000014B9C6010BD00BF041500206FF00A0116
:10631000094A9368C3F8B0100849C3F8AC004B6849
:1063200043F080534B60002383F31188BFF36F8FDA
:106330009368D3F8B00070470415002000ED00E02A
:1063400070B590F90D20437B002A36DBD90634D195
:106350001B4C63F07F032246437352F8183FE169F8
:10636000934207D1C0E900210860E06111E0994241
:10637000F8D01B68002BF5D090F90E5093F90E6001
:10638000B542F4D0AE42F2DD5968C0E90031086090
:106390005860A569954200D005B9E568A3685A7BA5
:1063A000D20604D1DA897F2A01D9AA6932B1AB4277
:1063B00002D0284600F00EFB656170BD6361FCE70A
:1063C0000415002038B590F90D200146002A437BC2
:1063D00004DA03F07F03437307F0CEF80D4D2A462D
:1063E00052F8184FAB68944200D004B9EC688B4265
:1063F00007D05A7BD20604D1DA897F2A01D9A26953
:106400002AB1A34202D0204600F0E4FA23466B6191
:1064100038BD00BF04150020B3F1FF3F08BFB2F143
:10642000FF3F03D00249183000F072BB704700BF35
:1064300067D6000038B5194CA168E0690B68814245
:1064400014BF1A46002249680B605960A368E169CD
:106450002AB9134AC3E900210B60E3610CE093F908
:106460000E0092F90E50A84214D0854212DD5168F8
:10647000C3E900210B605360A569094B9D4200D020
:1064800005B9E568A3689D4202D0284600F0A2FA4B
:10649000656138BD9142DCD01268D9E7041500204F
:1064A0001C150020F8B5DDE906670D4B0C46986811
:1064B00011460C4A1060EFF31182202282F31288F9
:1064C000BFF36F8F9D68284607F068F8284632466C
:1064D0003B46FFF7A1FF2046BDE8F840FFF716BF97
:1064E0000415002030150020F8B50446EFF311879D
:1064F000202383F31288BFF36F8F437B49B203F0ED
:106500001F02002A0CBF0126002639D103F07F03A9
:106510002D4D437307F030F82A46437B817363F0B7
:106520007F03437352F8183F934227D1E869C4E9C7
:1065300000200460EC610FE09842F8D01B68002B4B
:10654000F5D093F90EC06145F6D08C45F4DD59685D
:10655000C4E900310C605C60AC69944200D004B9BD
:10656000EC68AB689C4202D0204600F033FA6C61C4
:1065700087F31188BFF36F8F3046F8BDE869DEE717
:106580009B071ED5856806F0F7FF81732B689D4237
:1065900009D16B68C4E900531C606C60E8E76A6865
:1065A0009342F6D01B68002BF3D093F90E20914252
:1065B000F5D08A42F3DD5A68C4E9003214605C60A9
:1065C000D6E78173D4E700BF0415002049B9EFF383
:1065D000058030B9054B5A699B689A4201D0FFF794
:1065E00095BE81F31188BFF36F8F704704150020AB
:1065F000034648B9EFF3058232B9064A51699268F9
:10660000914201D0FFF782BE83F31188BFF36F8FF1
:10661000704700BF04150020EFF31181202383F39E
:106620001288BFF36F8F054B9A68D37B013BD373FE
:1066300081F31188BFF36F8F704700BF04150020EE
:1066400070B5EFF31186202383F31288BFF36F8FA9
:10665000144DAB68DA7B0132DA732A4652F8184FD0
:10666000944200D004B9EC685A7BD20604D1DA898E
:106670007F2A01D9A2692AB1A34202D0204600F0A4
:10668000A9F923466B6186F31188BFF36F8FEFF38F
:106690001180202383F31288BFF36F8FBDE8704011
:1066A000FFF7A6BF04150020024B03F11802C3E94F
:1066B000062270470415002070B5EFF311862023E1
:1066C00083F31288BFF36F8F1B4CA168E0690B68DE
:1066D000814214BF1A46002249680B605960A368C2
:1066E000E1692AB9154AC3E900210B60E3610CE0B6
:1066F00093F90E0092F90E50A84218D0854216DD8B
:106700005168C3E900210B605360A5690B4B9D42A2
:1067100000D005B9E568A3689D4202D0284600F084
:1067200059F965613046BDE87040FFF7EFBD8A4218
:10673000D8D01268D5E700BF041500201C15002032
:10674000F8B550EA010306460C4603D1FFF7B4FF43
:106750000020F8BDEFF31187202383F31288BFF3E5
:106760006F8F124D124BA8681860FFF72BFEA868B8
:10677000234632460F49183000F0CAF9AA68044689
:10678000537B384643F004035373FFF7BFFDAB68F8
:10679000D3E90A23B3F1004F08BF002AD8D107F08C
:1067A00004F8201A20EAE070D3E700BF04150020A7
:1067B0003015002067D6000038B50446EFF3118588
:1067C000202383F31288BFF36F8F437B5B070FD5C2
:1067D000183006F0C2FF637B204623F00403637386
:1067E000FFF7AEFD2946BDE838400448FFF7EEBE8E
:1067F00085F31188BFF36F8F38BD00BFBA27002023
:10680000014B9868704700BF041500202DE9F8433C
:106810000446077BEFF31185202383F31288BFF32F
:106820006F8F437B190705D585F31188BFF36F8FF1
:10683000BDE8F883D90943F0080260D14273A36828
:1068400013B1204606F0A0FE04F1180006F085FF03
:10685000A66D04F15808B04511D04FF0000976B18B
:10686000304606F091FE06F1180006F076FF30463D
:10687000C6F8B090FFF764FDA66DB045EFD1DFF824
:10688000C480D8F808309C4241D1EFF30589B9F1B2
:10689000000918BF4FF00109D8F818602A4A96423B
:1068A00000D00EB9D8F80C60B34202D0304600F0E8
:1068B00091F82046C8F8146004F079FB204600F0F7
:1068C000DBF8B9F1000F02D02048FFF70FFDD8F830
:1068D00008309C4231D1EFF3058373BB227BD20792
:1068E00018D42846FFF712FDFB07A1D5002383F338
:1068F0001188BFF36F8F0423184602DF98E703F077
:106900007F0343F00803437306F036FE97E74FF02A
:106910000009C1E785F31188BFF36F8F83F31188F6
:10692000BFF36F8F0423184602DFEFF3118020239B
:1069300083F31288BFF36F8FD4E785F31188BFF319
:106940006F8FD1E7041500201C150020C80B002014
:10695000D3B5DDE90667089CCDE90067FFF7A2FD26
:106960001CB1034B9B681B69236002B0D0BD00BF04
:1069700004150020427B034612F01F0210D10A4981
:1069800088420DD00949086868B1D9897F2909D89A
:1069900093F90E20064B1B689A42B8BF002070473F
:1069A0000020704710467047580A00209C020020C3
:1069B000341500200122044BC01A044BC010584368
:1069C000034B1A54704700BF800C0020ABAAAAAA40
:1069D000BA27002070B50D4B0D4D1E7CFFF7CAFF86
:1069E00006EB460305EBC3050446284606F0B5FE54
:1069F0000022084B9A553CB1621E2846BDE8704003
:106A00000549D31700F084B870BD00BF04150020FD
:106A1000800C0020BA270020B569000038B5EFF3DC
:106A20001185202383F31288BFF36F8F0F4B104A19
:106A30009C681068A04206D1FFF7CCFF85F311884F
:106A4000BFF36F8F38BD00211B7C1160094AD35CF6
:106A5000002BF3D02046FFF78DFF0028EED0637B9C
:106A6000DB0601D1FFF7E6FC2046E5E70415002030
:106A700030150020BA270020EFF31181202383F383
:106A80001288BFF36F8F0A4A136A834207D15B6F84
:106A9000136281F31188BFF36F8F70471346002B89
:106AA000F7D05A6F8242F9D1426F5A67F1E700BFBF
:106AB00004150020024B1868984208BF0020704758
:106AC000A0020020034B1B680BB9FDF7A5BD0020F9
:106AD000704700BF3815002030B570B10B4B5B68B4
:106AE00098420AD0036843B1D3E90421D0E90445B0
:106AF000121941EB0501C3E90421D0E9003213600A
:106B00005A600023C0E9003330BD00BFA00200205E
:106B1000B3F1FF3F08BFB2F1FF3F2DE9F84F044644
:106B2000994615461F467AD08160EFF311882023DD
:106B300083F31288BFF36F8FB9F1000FDFF8E4A081
:106B400020DBFFF7BFFFDAE90027013549F1000933
:106B50002D1849EBE07306464FF00109C4E90453D0
:106B6000AD1843EB0707FFF7A5FF0346DFF8B8E0D2
:106B7000DEF804A0EBB9C4E900EACAF80040CEF898
:106B8000044028E06FF00103DAE900125B1A4FF0CD
:106B9000FF3161EB02025B1B62EB0902012B72F118
:106BA0000001BCBF012300224FF00009C0E90432FC
:106BB000D9E7D3E9041CD4E904208A4270EB0C0B1A
:106BC00024DA891A5A686CEB0000C3E90410C4E99E
:106BD000003214605C60FFF76DFF84420ED1134BEE
:106BE0001B685BB9B9F1000F02D1FFF76BFF0646D6
:106BF000304606F09BFD0021FDF7E0FC88F311888C
:106C0000BFF36F8F28463946BDE8F88F521A60EB04
:106C10000C009A45C4E90420ADD01B68AAE7002502
:106C20002F46EFE7980C0020A00200203815002026
:106C30002DE9F047EFF31185202383F31288BFF38A
:106C40006F8FDFF8A0900026C9F800000027FFF73B
:106C500031FFDFF89480D9F80030D8E900ECD9177B
:106C600050B1D0E90442A34271EB020A1BDAE41AE4
:106C700062EB0102C0E90442002413EB0E034CEB6B
:106C800001012046C8E90031C9F8004006F04EFD78
:106C90002146FDF793FC85F31188BFF36F8FBDE8A4
:106CA000F047FFF7BBBE14EB0E024CEBE473C0E9F8
:106CB0000467C8E90023FFF70FFF85F31188BFF3CE
:106CC0006F8F83689847EFF31185202383F3128831
:106CD000BFF36F8FD9F800301B1BC9F80030FFF7E6
:106CE000E9FEB8E738150020980C002010B5EFF346
:106CF0001184202383F31288BFF36F8FFFF7E2FE26
:106D00000346054AD2E90001181841EBE37184F308
:106D10001188BFF36F8F10BD980C002038B5034663
:106D2000EFF31185202282F31288BFF36F8FC160C9
:106D3000012181600068834206D185F31188BFF389
:106D40006F8F0024204638BDD0E9003213605A60AE
:106D50000023C0E9003306F072FD294604460248CC
:106D6000FFF734FCEEE700BFBB2700202DE9F04120
:106D700005460E46174606F0F9FB30B9074B9B68EF
:106D8000D3F8A44014B9BDE8F081054C3B46324627
:106D900029462046BDE8F04106F0B3BD04150020A9
:106DA0003803002002460021014B024806F0A9BD2D
:106DB000E5A7000038030020014BC0F8A43070475D
:106DC000380300200146024A0020FFF7CFBF00BF72
:106DD000E5A7000007B5074B4FF480620093064912
:106DE0004FF0FF330548FFF763F9002003B05DF86B
:106DF00004FB00BFDCE2000060540020A00C002077
:106E000001680E4A0346914215D1C169A2F11022D0
:106E1000A2F1EF1291420ED18268012A0BD8C2680A
:106E200012B101698A4206D0586928B19B691B1AC0
:106E30005842584170470120704700BF55AA00FFD3
:106E400070B50D4B9E68A6B13046FFF7D9FF0446DA
:106E500078B9F3686BB935690DB9204670BD28461D
:106E6000FFF7CEFF28B9EB68B34202D12E462D6959
:106E7000F2E70124F1E700BF3C1500202DE9F041C5
:106E8000444B454C05461B6820468846984718B138
:106E900000242046BDE8F081A4F1140754F8144CF6
:106EA000FB68DCB1BC68CCB1002D66D0B8F1000F36
:106EB00065D008FB05F6B6FBF5F5A84561D1311D97
:106EC0005FD8B20711D026F0030204321C4603E05B
:106ED0006168914257D2A469002CF9D12F4B2E48FA
:106EE0001B6898470028D4D0D2E73246EEE7891ACB
:106EF000232904F120051CD80123A360D4E905232C
:106F0000AAB19361A3690BB162695A610023C4E914
:106F100005333B69DB0703D5FFF792FF002835D126
:106F20003246002128462C4606F07FFDD6E7FB605E
:106F3000E8E702F1200C04EB0C032039C3E901104F
:106F4000DC6021691648196144F80C00A0F110209A
:106F5000A0F1EF10D86101B1CB6061695961A069FE
:106F6000986141B18B61996901B14B610121236144
:106F7000C4E90121CAE7FB60F5E72C46AEE74446C9
:106F8000ACE70446AAE7A0680028B0D0012002F0D0
:106F900079FF00BFB802002050150020B402002085
:106FA00055AA00FF70B5464B464C05461B68204667
:106FB0009847002840F08280002D43D054F8143CBC
:106FC000A4F11406002B3DD0B268002A3AD09D42AD
:106FD00003D3726813449D4202D3012002F052FF92
:106FE000A5F120042046FFF70BFF0028F5D155F846
:106FF000183C012BF1D155F8143C45F8180C3BB363
:107000009A682ABB55F81C2C02F120015A680A44E0
:107010005A6055E905321A6155F8145C2B6903B1C1
:10702000DD6020220021204606F0FFFC286910B117
:107030008368002B2ED033699B0703D5FFF700FF31
:107040000028CAD1BDE870401F4B1E481B68184776
:1070500055F8100C00282AD0836843BB4268636847
:1070600013442033636003692361D4E905239AB98B
:10707000CBB9436963618269A261B3B19C61A369C1
:1070800003B15C61236903B1DC602022002106F0BA
:10709000CCFCD0E72C46E1E79361A369002BE8D054
:1070A00062695A61E5E7F360F7E7F460E7E7F368E0
:1070B00045F8083C03B15C61F460BCE770BD00BFFB
:1070C000B802002050150020B402002038B50C464C
:1070D0001C2200210546154806F0A7FC144B154854
:1070E0001B6898471449154800F032F8232C1CD926
:1070F00015F003031FBF043CE418C3F10403ED18AB
:1071000022460021284606F090FC084B0C49C3E9B2
:107110000054203C9D606C609A6811609A68A1F1EF
:107120001021A1F1EF11D161DA6038BD3C150020CA
:10713000BC02002050150020A56F00007D6E0000ED
:1071400055AA00FF014B1B68184700BFA80200208A
:10715000024B1860024B002019607047AC020020FF
:10716000A802002010B50A46044619B1024B0021BE
:107170001B68984710BD00BFB0020020F8B50D4E47
:107180000D4C0E4D33680E48984767782B680C48B5
:10719000984733680B489847022F08D12478E31F9B
:1071A0005C425C412B68074898472046F8BD0024A4
:1071B000F8E700BFB802002058150020B4020020F4
:1071C000280100203001002038B504460D46FFF7A5
:1071D000D5FF30B12A462146BDE83840024806F0C6
:1071E000EABB6FF0880038BD5C15002070B51D4EFD
:1071F0001D4C33681D4898472378590744BF23F036
:107200000403237023789A0705D500F0C1F823788A
:1072100023F002032370164D14482B6898473368F7
:1072200014489847637813B1134806F0D5FB002340
:10723000042111486370FFF795FF2B680D489847AC
:1072400033680A4898472378DB0705D506F0B0FB7A
:10725000237823F0010323702B680448BDE87040B5
:10726000184700BFB8020020581500203001002048
:10727000B4020020280100205C1500202DE9F04117
:10728000FFF77CFF18B100242046BDE8F081364F9F
:1072900036483B689847044620B16FF08F04FFF7EB
:1072A000A5FFF1E7324D2B78D80706D406F07EFB18
:1072B00004462B7843F001032B702E4E2B48336885
:1072C000984710B1002CE8D0E9E7002CE7D13B68E3
:1072D0002648984704460028DFD12B78990706D422
:1072E00000F04EF804462B7843F002032B7033680D
:1072F0001E4898470028E5D1002CD0D13B681B4898
:1073000098470028C9D13368184895F800809847F5
:107310000028C2D13B681848984704460028BCD1D1
:107320006B7843B918F0010F05D0144806F041FB03
:10733000022304466B7033680F4898470028C1D178
:10734000002CACD13B68094898470028A5D12B7880
:1073500006485A075CBF43F004032B703368984714
:10736000002890D099E700BFB8020020300100202B
:1073700058150020B4020020280100205C150020D0
:107380000122024B002083F8802570476015002001
:107390002DE9F0410A4C002526464FF0010803274D
:1073A0002046C4F820802777013506F0E2FA202D28
:1073B00004F12C04F4D1002386F88035BDE8F08177
:1073C00060150020014B1B68184700BFDC0200203D
:1073D000014B9B68184700BFDC020020014BDB68B3
:1073E000184700BFDC02002010B50C4C236813B115
:1073F0000B4B1B682BB900F05FFE30B90122084B24
:107400001A6001232360002010BD0138072801D92C
:10741000044810BD044B53F8200010BDE81A0020AA
:10742000E41A0020FE8FFFFFE8E20000BFF34F8F59
:107430000549064BCA6802F4E0621343CB60BFF310
:107440004F8F00BFFDE700BF00ED00E00400FA052C
:1074500030B44FF0FE3200250B4B0C4C0C49496800
:10746000C3F80024C3F80424C3F80824C3F80C2488
:10747000C3F81024C3F81424C3F81824C3F81C2438
:10748000C4F8005530BC0847005084500040845078
:10749000C0020020024BD0E90012C3E9001270477D
:1074A000C0020020144B2DE9F043002814BF04460D
:1074B0001C46124F236883B0BB4219D016460D46B6
:1074C00020464FF4E07104F1040900F0EDF804F5F2
:1074D0008E78484600F0D0FC404600F0F3FA2B4688
:1074E0004A4640460649009600F002FB08B927606C
:1074F000002003B0BDE8F083EC1A0020A5BCC95AF7
:10750000FD7E000070B50D4C1D46002814BF0646D8
:1075100026460B4B306882B098420DD106F58E702E
:10752000002633460096144600F032FB002818BFB0
:1075300034462C6002B070BD0248FBE7EC1A002014
:10754000A5BCC95AE88FFFFF10B5044650B1636867
:1075500013F0685F05D0064A934202D000236260B0
:10756000236010BD034B04485B689847EFE700BFFA
:107570002C5F5CA9C002002008E30000C8B143688A
:107580000D4A934213D013F0685F0ED0012350E8E8
:10759000002F194640E8001C9CF0000FF7D1012A8B
:1075A000F5D0BFF35F8F0020704704487047044850
:1075B00070476FF4E04070472C5F5CA9E98FFFFFD4
:1075C000EA8FFFFF034680B1426809498A420AD028
:1075D00012F0685F05D0BFF35F8F002210461A607B
:1075E000704704487047044870476FF4E0407047A4
:1075F0002C5F5CA9E98FFFFFEA8FFFFF10B50446FF
:1076000020B10023034A2360626010BD0248FFF7E7
:107610001FFFF6E73A00003A30E3000070B5194C5E
:10762000D0F804C00668C4F804C0D0F808C0C06828
:10763000C4F808C0E06026600868134B134D18605A
:107640004868D5F818215860886812F0685F98601B
:10765000C8680969D860196112D000230C4A05F581
:107660008A70C5F81431C5F8B831C5F81821C5F8C5
:10767000BC21B047236805F5DC70BDE870401847B1
:1076800070BD00BFDC020020C8020020EC1A002000
:107690002C5F5CA938B131B10022014403460130AE
:1076A00081421A70FAD1704738B131B100220144D9
:1076B0000346013088421A70FAD170472DE9F04F25
:1076C000B2F5C07FBDB000F2DA800C46DFF8B491AD
:1076D000154600214FF4D07282460DF17C084846D1
:1076E00006F0A3F9404601F047F930232146002473
:1076F00009F118062A4689F8173030466BBAA9F8FE
:107700001230A9F8104006F069F98022234672551C
:107710000DF12B0101F8013F0133202BFAD14FF479
:10772000807240460BA901F03DF98346002840F0E5
:10773000A38005F1190313AD2F4607AE0293CDF8D0
:107740000CA00196049510220021019806F06DF915
:10775000DFF834A1DDF808B005970A9B5AF8044C0D
:10776000089F099A07995AF8100C5AF80C6C5AF8A5
:10777000085C5C40019B7E40554081EA00071A4648
:1077800001214046CDE90776CDE9095401F02CF9F5
:10779000BBF1100F94BFABEB0B0BABF1100B0AF16D
:1077A000100A002847D1BBF1000FD6D1059F102247
:1077B0003846019906F012F999F803301037013371
:1077C000474589F80330BED1049D4FF480722946A5
:1077D0004046DDF80CA0019E01F0E4F8834678BB3A
:1077E00054460AF130071BAB1A460121404601F00E
:1077F000FBF8834620BB102220461BA9144406F048
:10780000EDF8A742EFD1404601F0C6F84FF4D07131
:107810001C48FFF749FF28463021FFF745FF0BA81A
:107820002021FFF741FF30461021FFF73DFF58466A
:107830003DB0BDE8F08F8346DDF80CA0019E049DAD
:10784000404601F0A9F84FF4D0710E48FFF72CFF25
:1078500028463021FFF728FF20210BA8FFF724FF3F
:1078600010213046FFF720FF30215046FFF71CFF64
:1078700058463DB0BDE8F08F13AD07AEE0E76FF0BE
:10788000370BF5E7BC1C0020CC1C00202DE9F04193
:107890008CB004460D463022002168466F4606F043
:1078A000C4F804F12006E27B0132D2B2E273002A6E
:1078B0004DD1A27B0132D2B2A273002A47D1637BA1
:1078C0000133DBB26373002B41D1237B0133DBB285
:1078D0002373002B3BD1E37A0133DBB2E372002B3D
:1078E00035D1A37A0133DBB2A372002B2FD1637A97
:1078F0000133DBB2637253BB237A0133DBB22372F1
:107900002BBBE3790133DBB2E37103BBA379013312
:10791000DBB2A371DBB963790133DBB26371B3B955
:1079200023790133DBB223718BB9E3780133DBB206
:10793000E37063B9A3780133DBB2A3703BB963781A
:107940000133DBB2637013B92378013323703B46F4
:1079500022460121304601F047F88046002841D1F7
:1079600010370CAB9F429ED1029AAB6803995340EB
:1079700002933046EE68D5F820804E400396049975
:107980002E69D5F828C04E4004966E6905990B9F64
:107990004E4005960699AE69009B4E400696EE69EC
:1079A00007994FF480724E400796089ED5F824E060
:1079B00088EA0608099E8EEA060E0A9E8CEA0601EF
:1079C000EE6A7E402F687B4000936B68019D6B40A0
:1079D0000193CDE9088ECDE90A16694600F0E2FF71
:1079E000804638B168463021FFF75EFE40460CB055
:1079F000BDE8F0811022204608A905F0EFFFF1E76D
:107A00002DE9F8431D468369B3F5C07F52D8164669
:107A1000C3F5C072AA424DD3C5F5C072D31AB342A2
:107A200048D30446DFF898904FF4C0720F4648469A
:107A3000002105F0FAFF4946D4F89430A269D4F841
:107A400098009847002838D1D4F818803DB1D4E97F
:107A500025302A4609EB0801984770BBA84407B1B6
:107A6000C6B9174942460846FFF728FE054638B111
:107A70004FF4C0711248FFF717FE2846BDE8F8839F
:107A800020460F49FFF702FF05460028F0D10123E9
:107A90002361EDE73946324609EB080005F09EFF09
:107AA0000749B04442460846FFF708FE054600284D
:107AB000DED1E5E76FF03705DFE76FF03305DCE790
:107AC0005C1E002010B5A4220021044605F0ADFF85
:107AD0004FF0FF314FF6F072044B2161E26104F187
:107AE0009C001B68BDE81040184700BFBC02002086
:107AF0002DE9F047054688B00F46164600212022A2
:107B00006846984605F091FF1F4B05F19C094846D1
:107B10001B689847044618B1204608B0BDE8F087B6
:107B200005F1200A504600F027FFAA69C5E925762D
:107B3000F2B920232E69AB61002E22DB6946504644
:107B40004FF4807200F02EFF044630B933464146B0
:107B50002846109AFFF754FF04460C4B48461B6812
:107B60009847002818BF0446204608B0BDE8F087B3
:107B70002E69002EE2DA2F2A96BF013226465608D9
:107B8000DCE71026DAE700BFB8020020B4020020CC
:107B90002DE9F04FB2F5806F91B01A9F00F2E380AB
:107BA000B7F5807F00F2DC80044615460E46302291
:107BB000002104A8984605F038FF6C4B04F19C099D
:107BC00048461B6898478346002840F09280226907
:107BD000E3699A4200F391806369002B40F08D8045
:107BE000002F40F0A980DFF888A16F46002D00F03B
:107BF00098806F4604F120080EE0102DAB4628BF98
:107C00004FF0100B304639465A4605F0E7FEB5EB0B
:107C10000B055E4400F08580E37B0133DBB2E37348
:107C2000002B4DD1A37B0133DBB2A373002B47D1D3
:107C3000637B0133DBB26373002B41D1237B0133C0
:107C4000DBB22373002B3BD1E37A0133DBB2E37267
:107C5000002B35D1A37A0133DBB2A372002B2FD1D5
:107C6000637A0133DBB2637253BB237A0133DBB235
:107C700023722BBBE3790133DBB2E37103BBA3793E
:107C80000133DBB2A371DBB963790133DBB263711A
:107C9000B3B923790133DBB223718BB9E3780133B4
:107CA000DBB2E37063B9A3780133DBB2A3703BB9F5
:107CB00063780133DBB2637013B923780133237027
:107CC0003B4622460121404600F08EFE83460028B6
:107CD00093D0DAF80030484698470346302104A88C
:107CE000002B18BF9B46FFF7DFFC10213846FFF73B
:107CF000DBFC584611B0BDE8F08F3A464146002300
:107D00002046FFF77DFEDFF868A000283FF46DAF46
:107D10004846DAF800309847834600283FF465AFBC
:107D2000E7E7204604A9FFF7B1FD83460028D0D13C
:107D3000236901332361CCE73A46414604A8FFF7A3
:107D4000BDFC834618B16F46DFF824A0C1E720468A
:107D500004A9FFF79BFD834600283FF444AFF2E7F8
:107D60006FF0370BC5E76FF0350BC2E7B8020020A4
:107D7000B40200202DE9F043202B1D46064688461C
:107D800091468BB026D8DBB202AF8DF80480B046A6
:107D900058F8041B8DF8053021B9404600F066FE06
:107DA000044640B9012302224046336001A900F095
:107DB00071FE044638B138462021FFF775FC204695
:107DC0000BB0BDE8F0832A464946404600F062FE0B
:107DD0000446F0E702AF1946104600233A4600F089
:107DE000DFFF04460028E6D12023B9461D46CCE734
:107DF0002DE9F041D0F8F830A6B0002BD8BF02AE84
:107E000031DD05460027D0F80C4102AEA4F101088F
:107E10009022D5F8FC403146D0F8000101AB019723
:107E2000B8FA88F8A0474FEA5818044620B9019BD1
:107E300053B9B8F1000F16D030469021FFF734FC4B
:107E4000204626B0BDE8F081014632462846FFF7BD
:107E500091FF58B9D5F80431019A1344C5F804319B
:107E6000B8F1000FE8D16FF03C04E5E70446204686
:107E700026B0BDE8F08100BF70B50025044614228D
:107E800004F588762946C0F8F850FC3005F0CDFDA1
:107E900008222946304605F0C8FD144B30461B68C1
:107EA0009847204640F8045B00F0C6FD104B304672
:107EB0001B689847C8B9D4F8F830AB420FDC03EB25
:107EC000830204EB82022021C2F800010120C2E9F2
:107ED000421008490133C2F8FC10C4F8F830064BD0
:107EE0003046BDE870401B68184770BDBC020020DA
:107EF000B802002075880000B40200202DE9F04788
:107F0000202A88B07AD83F4B00F5887904461B6850
:107F100048461746884698470546F8B940F2011684
:107F2000D4F8F830002B65D02046FFF761FF0546F6
:107F300038B9D4F8F830002B14DC013EF2D16FF0E0
:107F40003B056E4620213046FFF7AEFB2E4B4846E0
:107F50001B689847002818BF6FF01D05284608B019
:107F6000BDE8F087D4E94132934203D3D4F80C2121
:107F7000012A02D0013ED7D1E1E71F2BFAD96E4684
:107F800001462022304604F1040A05F04EFD314638
:107F9000504600F0A9FD05460028D3D1504600F018
:107FA0005FFD504600F048FD2946504600F05EFD5A
:107FB00005460028C6D150462022314600F06AFD11
:107FC00005460028BED1034632462021304600F047
:107FD000E7FE05460028B5D1D4F8F8303A46002B24
:107FE000C8BF002340463146C8BFC4F8043105F07D
:107FF000F5FCA7E76FF03F056E46A3E76FF03B0582
:10800000ACE700BFB8020020B4020020002130B568
:108010008DB0282202A8019105F007FD02A800F00A
:10802000E7FE044610B120460DB030BD1B4D4FF0A9
:10803000FF31286800F034F960BB194BD3F8340ED7
:1080400010F0010017D100F05BF9F8B9154A02A948
:1080500001A800F001FC0446012000F051F988B9A4
:10806000286800F025F90028DDD00F48FFF7F0F967
:1080700020460DB030BD2868052400F019F900280D
:10808000D1D0F2E70948FFF7E3F9E9E70848FFF73D
:10809000DFF9DBE70748FFF7DBF9CEE71003002045
:1080A00000608450DC1F0020ACE300008CE3000083
:1080B0006CE3000054E3000030B583B000F036F804
:1080C00078B900F055F890B9144BC3F80C0AFFF7D3
:1080D0009DFF0446F8B9124D2B6863B1204603B0EA
:1080E00030BD032400F072F8204603B030BD0424F4
:1080F000204603B030BD02460146FFF7D3F950B920
:108100006822084901ABFFF7FDF920B92046064B6C
:108110002B6003B030BD0524E0E700BF0050845061
:10812000FC210020002200205AEA5A5A0020704701
:10813000430504D54FF0FF32034BC3F80821024B2F
:10814000C3F8080A704700BF00508450014BC3F8C1
:10815000040A70470050845008B100F071B84FF421
:108160007500704708B100F04FB84FF475007047C4
:1081700010B5114800F080F800B110BD0F4800F0B4
:108180007BF80028F9D10E4C204600F075F8002845
:10819000F3D10C4B0C481C6000F06EF8014600282F
:1081A000EBD100F02DF8044608B1204610BD00F0D8
:1081B00089F82046FAE700BF200300201C030020B6
:1081C00018030020100300201403002008B50848FD
:1081D00000F05CF8074800F059F8074800F056F83E
:1081E000064800F053F8BDE8084000F00BB800BFA7
:1081F000200300201C03002018030020140300208B
:1082000000207047704700BF10B402460B4C01E0DD
:10821000134207D1D4F8003A13F48070F8D001204B
:1082200042F4807229B1054BD3F804410C60C3F8C5
:108230000841024BC3F8082A10BC70470050845014
:108240000246084901E01A4207D1D1F8003A13F476
:108250008070F8D0012042F48072024BC3F8082AE3
:10826000704700BF0050845005F0C5BB05F0DDBB72
:108270000A46002105F0D9BB08B5034B02681B680C
:1082800010689847002008BDDC02002008B5034BA9
:1082900002685B6810689847002008BDDC02002077
:1082A000024B02689B681068184700BFDC02002080
:1082B00008B5034B0268DB6810689847002008BDCA
:1082C000DC02002070B5094C094D2069AB68984765
:1082D00018B1084B08485B6898470021074AEB68CB
:1082E00011602069BDE87040184700BFC802002037
:1082F000DC020020C0020020C4E30000682200204D
:10830000F8B51A4D1A4E0446B26828699047E8B984
:10831000184F3B684CB1A3B1012B19D0013B3B6016
:108320002869F36898470020F8BD43B90121124A33
:10833000C2F800151149D1F81029002AFBD10133E8
:108340003B60F368286998470020F8BD0C48F8BDE9
:108350000A4AD2F81039002BFBD1074A6FF07E4051
:10836000C2F80035FFF7F2FE3B68D7E7C8020020ED
:10837000DC0200206822002000408450005084501D
:10838000E98FFFFF2DE9F041002873D00C4600294A
:1083900070D01D46002B6DD007461AB10122002374
:1083A0002A6003602B68002B5FD02946204600F02E
:1083B000D9FD804600285AD12146286800F0B8FD32
:1083C0008046002853D12868082867D0042867D041
:1083D000A0F10200B0FA80F040090121314EC6F848
:1083E000C411C6F84011C6F8C411636AC6F830312A
:1083F000D6F830219342F6D10023C6F82C314FF045
:10840000FF33C6F808316FF01B03C6F80031C6F819
:108410000C01D6F8040A40F48060FFF797FE0A23A7
:10842000C6F83831069B012B29D023691E4AA2FBCE
:1084300003231B09626A404602FB03F303EB430379
:10844000184ADB039B09C2F8D8310123C2F82C314A
:108450003B682A6823F07F4343EA02633B602A6853
:1084600043EA02233B60BDE8F081DFF840804046EC
:10847000BDE8F081DFF838804046BDE8F0814FF478
:108480007F03D3F80C2C013206D0D3F80C3C064AFB
:10849000A2FB03231B09CDE71623CBE703209CE7B0
:1084A00002209AE700508450ABAAAAAA310CF1002E
:1084B000350CF10058B34B1EB3F5047F27D230B50D
:1084C0004FF0000ECD00744671464B0901F01F0CB1
:1084D00050F82330BCF11F0F23FA0CF306D003F041
:1084E000010319B901211C468E46EEE79C4201F1B9
:1084F000010106D01C464FF0010EA942E5D1002033
:1085000030BD0EF1010E9645F7D1024830BD01484D
:10851000704700BF360CF100C0B32DE9F0434C1E8C
:10852000B4F5047F1DD2E3B1DAB100252E46A8468A
:108530002C46CF0003F1FF394FEA541C04F01F0E04
:1085400050F82C10BEF11F0F21FA0EFC0CD00CF0CD
:10855000010C4CB90126E04634463546ECE796421C
:1085600016D90C48BDE8F083AB420BD0C44508BF18
:108570000136A945F3D001350134BC42DCD10020DD
:10858000BDE8F0830125E0462E46F5E70148704737
:108590001D46F1E7370CF1002DE9F04F8FB0824610
:1085A000DDE919460D46002E6ED1096904911C6063
:1085B000002318990B60002A00F02881994B6A6A01
:1085C000D3F83811D3F830319A4269D10A2967D1EA
:1085D0009AF80330069304F1080305930423049AE0
:1085E0000393914B8F4CA3FB023B4FEA9B0B0BEB8E
:1085F0004B0BA2EB4B0B189B049E1E60002E00F051
:10860000E580002700F0BEFC0797BAF1000F00F0EC
:10861000D0804FF00109DDF81480002D00F0C980F2
:10862000069B002B3ED0284606A900F09BFC0028A4
:108630003AD07E4B984220D0069B082B00F0E08079
:1086400000225B000693294606AB50460092FFF7D6
:1086500099FE774B984200F0CF8070B9DAF800208D
:10866000130A03F47F03134323F07F43CAF8003057
:10867000039B013B0393BED10020039000F082FCDA
:1086800003980FB0BDE8F08F4FF47F01D1F80C0CC8
:1086900001300CBF4FF40471D1F80C1C049186E733
:1086A0006448EAE76248C4E72946069800F040FCBF
:1086B0000028BED1069B082B00F0A480042B00F0FC
:1086C000A380A3F10203B3FA83F35B09C4F8C49156
:1086D000C4F84091C4F8C4916A6AC4F83021D4F84F
:1086E00030118A42F6D10022C4F82C214FF0FF321B
:1086F000C4F808216FF01B02C4F80021C4F80C3143
:10870000D4F8040A40F48060FFF720FD0A23C4F87F
:1087100038312B69444AA2FB0313696A1B0901FB28
:1087200003F303EB4303DB039B09C4F8D831C4F81C
:108730002C910698DAF8003023F07F41030243EAD7
:1087400000630B43CAF8003007A800F0E1FB079B69
:10875000354A03F01A0303437FF46EAFA2FB0632DF
:10876000D4F81431B7EB920F0893D4F81831099369
:10877000D4F81C310A93D4F820310B93D4F8243167
:108780000C93D4F828310D9302D1BBF1000F12D114
:108790004046182208A9183EFFF766FD08F11808A0
:1087A00001379EB100F0EEFB00230793002D7FF40C
:1087B00037AF21483DE740465A4608A9A6EB0B06CD
:1087C000FFF752FDD8440137002EEBD1049F059EE0
:1087D0006A6939463046FFF76DFEAA6940B94FF421
:1087E000806339463046FFF797FE00283FF444AFD8
:1087F0000023189A13601CE72B6A002B3FF43DAF4F
:108800000E483AE7032361E702235FE70122294686
:108810005046009606ABFFF7B5FD00283FF4DBAEEF
:108820002BE700BF00508450ABAAAAAA020CF100AB
:10883000310CF100300CF100350CF100320CF1007C
:1088400010B4DDE9013401940024DDF80CC0CDE959
:1088500002C410BCFFF7A0BE30B51546012487B096
:1088600005AB00930022CDE9015404ABFFF794FE61
:1088700007B030BDF0B587B0002967D01E46002B89
:1088800064D01446002A61D0324F0D4638684FF04C
:10889000FF31FFF705FD00283DD12F4BD3F8340EF3
:1088A00010F0010015D04FF0FF354FF408712B4840
:1088B000FEF7F0FE04212A48FEF7ECFE29482821A5
:1088C000FEF7E8FE3868FFF7F3FC40BB284607B028
:1088D000F0BDFFF715FD002834D1224800F088FADA
:1088E00070B91E4A0346029205AA019204AA039097
:1088F00000921C4902461A48FFF7A2FF0346A0B1A6
:108900004FF0FF350120FFF7FBFC0028CDD01648C3
:10891000FEF79EFDC9E71548FEF79AFDBDE714482E
:10892000FEF796FD284607B0F0BD28461D46059B7C
:1089300022469C4228BF1A46049932600831FFF74C
:1089400093FCDFE70B48FEF783FDC6E74FF0FF35EA
:10895000BCE700BF10030020006084509822002074
:108960006C220020702200208CE3000054E3000001
:10897000E4E300006CE3000010B5044630B10022CF
:1089800001236265A265E365236610BD0148FEF719
:108990005FFDF4E7FCE3000018B174220021FFF74B
:1089A00065BC7047C8B1D9B108B50023C02A83633C
:1089B00080F83C300FD0B2F5807F04D0802A03D0FD
:1089C0006FF01F0008BD02230363D2081030FFF7C9
:1089D0004BFC002008BD0123F6E76FF02100704733
:1089E0006FF01F00704700BF70B5044686B0F8B145
:1089F0001046EAB1E3B101291AD8A26B16D0012AB8
:108A000016D1102500210DEB0506019602AA61631F
:108A10002946009500F0C8FA50B92B463246204648
:108A200002A900F073FD18B906B070BD002AE8D0A5
:108A30006FF02100F8E700BF10B5044628B12046CA
:108A4000BDE81040F421FFF713BC0448FEF700FD19
:108A50002046BDE81040F421FFF70ABC10E40000F6
:108A600010B1F421FEF716BE704700BF08B521B162
:108A7000012908D06FF0360008BD012100F058F838
:108A80000028F7D108BD022100F052F80028F9D0E3
:108A9000F0E700BF30B505468818B0F5801F0B46DB
:108AA0001446A1B001D8802A0CD9B3F5801F17D97C
:108AB00022461946284600F07DF8044684B920462F
:108AC00021B030BD6846FFF7CFFB224669462846F5
:108AD00000F070F8802104466846FFF7C9FBEDE717
:108AE0006FF03604EBE700BF70B5E8B10E46D9B1C0
:108AF000044600F031F80546B0B92368012B0BD0CD
:108B0000022B01D0284670BD1C22304604F108011A
:108B1000FFF7AAFB284670BD2022304604F1080169
:108B2000FFF7A2FB284670BD6FF03605EAE700BFED
:108B300078B138B50D46F0210446FFF799FB402384
:108B400020462560E36500F061FA003818BF012077
:108B500038BD0120704700BFF0B5056EA5B00446D2
:108B600004AEE5B90023012701933046676029462A
:108B700002AA009300F018FA10B1012025B0F0BD50
:108B80002A46204602A900F069FA0028F5D12046BD
:108B900000F06CFB0028F0D1206625B0F0BD802DE0
:108BA0002A46304628BF802204F16401FFF75CFBAF
:108BB000256ED7E7002800F0AE802DE9F04F14466F
:108BC000A5B0002A3DD00F46002949D0B2F5803F1C
:108BD0000546006E20D34FF6FF7805F1640AEB6D71
:108BE0001A1AB2FBF3F103FB1122002A65D183426A
:108BF000B9464FF6FF7672D0B6FBF3FB03FB0BFBD7
:108C0000BBF1000F30D1002E45D1A4F57F44FF3CCD
:108C1000B4F5803F4744E2D2EA6D161AB6FBF2F390
:108C200002FB1366A64228BF2646002E75D182425B
:108C300000F08D80B4FBF2F602FB06F62EB9002C94
:108C400079D1002025B0BDE8F08F002331463846A9
:108C5000CDE9003302AA00F0A7F9002800F09580C2
:108C6000012025B0BDE8F08F002359464846CDE9E4
:108C7000003302AA00F098F90028F1D15A4628469C
:108C800002A900F0EBF90028EAD1A6EB0B06286E4A
:108C9000D944002EB9D019304946324605EB800040
:108CA000FFF7E2FAA4F57F44286EFF3C3044B4F5A8
:108CB000803F4744286692D2AEE7424528BF4246ED
:108CC000164639465044FFF7CFFA286EEB6D304414
:108CD000834207EB06092866A8EB06068CD1802B99
:108CE00028BF802351461A4604A8FFF7BDFA002387
:108CF000E96D02AACDE9003304A800F055F9002877
:108D0000AED12846EA6D02A900F0A8F90028A7D143
:108D1000EB6D286670E70120704705F16403394662
:108D200032461844FFF7A0FA286EEA6D3044A41BBF
:108D3000374428667BE72B6E2246193305EB830008
:108D40003946FFF791FA2B6E23442B6679E7802A88
:108D500028BF802205F1640104A8FFF785FA0023EB
:108D6000E96D04A8CDE9003302AA00F01DF900283E
:108D70007FF476AF2846EA6D02A900F06FF900286B
:108D80007FF46EAFEA6D286654E73246284602A9A2
:108D900000F064F900287FF463AF3744A41B4EE76A
:108DA000F8B51C460546114816460F46FFF744FE27
:108DB00021460E48FFF75AFE044620B10B48FFF744
:108DC0004FFE2046F8BD3A4629460848FFF762FEA6
:108DD00004460028F2D131460448FFF785FE0446D8
:108DE0000248FFF73DFE2046F8BD00BFB824002032
:108DF0001C2370B582B001A90546019300F032F83A
:108E0000044638B9019B1C2B07D0144C1C21284662
:108E1000FFF72EFA204602B070BDD5E90112131EED
:108E200018BF0123003918BF0121012628689B00C3
:108E3000EA6843EA4103002818BF43F00103EE61EA
:108E40002AB9C5E90834002BE4D1054CDEE72046F9
:108E500043F00803C5E9083402B070BD370CF000D8
:108E60000E0CF000034618B111B10A681C2A01D09B
:108E7000012070474FF47F02D2F8101C01310CBF63
:108E800040F2DC51D2F8101C4FF47F020160D2F89E
:108E9000141C01310CBF40F2DC51D2F8141C4FF409
:108EA0007F024160D2F8181C01310CBF40F634013A
:108EB000D2F8181C4FF47F028160D2F81C1C0131DB
:108EC0000CBF40F63401D2F81C1C4FF47F02C16085
:108ED000D2F8001C01310CBF9021D2F8001C4FF4D5
:108EE0007F020161D2F8041C01310CBF5121D2F87C
:108EF000041C4FF47F024161D2F8081C00200131AC
:108F00000CBF40F23732D2F8082C9A61704700BF8C
:108F1000014608B54FF48060FFF724F90022034BA7
:108F2000C3F8C821C3F82C2108BD00BF00508450ED
:108F30000138072805D8DFE800F0100E040A040401
:108F4000040607487047CB6800204B6270478B6867
:108F500000204B6270474B68F6E70B68F4E700BFF0
:108F6000310CF1000B6802E0082B0B6006D8026A96
:108F700013424FEA4303F7D0002070470048704780
:108F8000310CF100002310B5064C4FF48060C4F89A
:108F90002C31C4F8C431FFF7CBF84FF0FF33C4F8DD
:108FA000083110BD005084502DE9F041002482B0FA
:108FB00015461E4601220DF107030746DDF8248001
:108FC0008DF8074000F05AFFD0B99DF807300446ED
:108FD0002F602B71B8F1000F0ED04EB102460899E8
:108FE00030460DF1070300F049FF48B99DF80730FE
:108FF000C8F8006088F80430204602B0BDE8F0816F
:109000004FF47504204602B0BDE8F081D8B108B530
:109010000368012B04D0022B0FD043B10B4808BDCD
:1090200020220B490830FFF71FF9002008BD142249
:1090300008490830FFF718F9F7E7202206490830F9
:10904000FFF712F9F1E74FF4730070470100F300E6
:1090500020E4000060E4000040E400002DE9F04757
:10906000002900F0EB800446002800F0EB80036844
:1090700088469146002B00F0B580013B012B00F2A1
:10908000C9804FF0FF3171484FF0020AFFF708F92D
:10909000002840F0B1800020FFF732F90746002891
:1090A00040F0B4806A4DD5F81069002EFBD14FF026
:1090B000FF30FFF73DF8D5F8040A20F40060FFF711
:1090C00045F801230722C5F81838C5F82038C5F837
:1090D0000029C5F8C437C5F8A466A36CC5F8CC3719
:1090E000E36CC5F8D037C5F8C0A723685BB1013B76
:1090F000012B18D8636AC5F85C36236AC5F8583660
:10910000E369C5F85436A269514BC3F85026626929
:10911000C3F84C262269C3F84826E268C3F84426FF
:10912000A268C3F84026B9F1000F56D063684FF427
:109130000060012B04BF464AC2F8843698F8043018
:10914000D8F80010424A5B0003F00203C2F80C3B5F
:10915000C2F8281CC2F82C9CFEF7FEFF07462368C5
:1091600063B1013B012B19D8394BD3F85C266262FD
:10917000D3F858262262D3F85436E361344BD3F83F
:109180005026A261D3F84C266261D3F848262261AA
:10919000D3F84426E260D3F84036A36000220121D0
:1091A0002B4BD3F8CC07A064D3F8D007E064C3F806
:1091B000C417C3F88426C3F8C827C3F81828C3F80F
:1091C0002028AFBB0120FFF79BF868BB1F48FFF7C3
:1091D0006FF818BB3846BDE8F08704221C4BC3F873
:1091E000C827BCE74FF0FF3118484FF0010AFFF7DE
:1091F00057F800283FF44FAF1648FEF729F9002032
:10920000FFF77EF8074600283FF44CAF1248FEF700
:109210001FF947E7114F3846BDE8F0871048FEF7C1
:1092200017F93846BDE8F0870E48FEF711F9CDE78B
:10923000102104F10800FFF71BF8C3E70A4F384676
:10924000BDE8F0874FF47307C4E700BF2003002098
:109250000050845054E300006CE300000100F30070
:10926000ACE300008CE300000300F300A0B303466E
:1092700070B4D0E90240D3E9041226BA05BA0CBA98
:1092800010BAC3E90440D3E90612986A09BAC3E9DF
:10929000026512BA996100BAD3E9084125BA0CBA3D
:1092A000C3E90725D3E90B12C3E9094009BAD86B12
:1092B00012BAD962D3E90D4125BAC3E90C250CBA1B
:1092C00000BAD3E9101209BA12BAC3E90E40196400
:1092D00000205A6470BC70474FF47300704700BFA1
:1092E00070B500284DD0436B0446032B3CDD063B94
:1092F000012B3BD8A36B012B3BD8E36D012B3DD851
:10930000236E012B41D8224ED6F81059002DFBD1E7
:109310004FF0FF30FEF70CFFD6F8040A20F400608F
:10932000FEF714FF0123C6F80039C6F8BC54636B7E
:1093300023F00402032A18BFA16B226B0CBF29463D
:1093400001F00101022A17D89B0003F01C0343EA35
:1093500002330F4A0B43C2F8C034636B072B06D1AC
:109360000123C2F87C3402E0002BC3DA094D284601
:1093700070BD094D284670BD084DF8E7084D2846D8
:1093800070BD4FF47105284670BD064DEFE700BF74
:10939000005084500100F1000200F1000600F100CD
:1093A0000300F1000400F10000287DD038B590F8EA
:1093B0003C300446002B55D0022B23D03C483D4D79
:1093C0002A683D4B1268C3F800242A685268C3F823
:1093D00004242A689268C3F808242A68D268C3F86B
:1093E0000C242A681269C3F810242A685269C3F849
:1093F00014242A689269C3F818242A68D269C3F829
:109400001C2438BD016B006C00F032FB294D002894
:10941000D6D12A68284B1268C3F800242A685268FB
:10942000C3F804242A689268C3F808242A68D2681A
:10943000C3F80C242A681269C3F810242A685269F8
:10944000C3F814242A689269C3F818242A68D269D8
:10945000C3F81C24216B206C00F020FB0028AFD146
:10946000002038BD0269144BC3F800244269C3F8D8
:1094700004248269C3F80824C269C3F80C24026B6F
:10948000013A012AECD8026AC3F81024426AC3F8F0
:109490001424026B022AE3D1826AC3F81824C26A38
:1094A0000020C3F81C24DCE74FF47100704700BFB4
:1094B0000900F1000C03002000508450114A124BA7
:1094C00011680968C3F8001411684968C3F80414E6
:1094D00011688968C3F808141168C968C3F80C14C6
:1094E00011680969C3F8101411684969C3F81414A4
:1094F00011688969C3F818141268D269C3F81C246A
:10950000704700BF0C030020005084502DE9F04F3D
:1095100085B0002958D01746002A55D004460028A7
:1095200000F0DC809846C36D0E46002B42D1B8F5A2
:10953000805F44D294F83C30042B00F0C7804FF099
:10954000000A4FF0FF31B548FEF7AAFE002840F0B0
:10955000B9800020FEF7D4FE002840F0AF804FF025
:109560000109DFF8BCB22046CBF81098CBF8209860
:10957000FFF7B6FE054620B92046FFF715FF054662
:1095800038B3BAF1000F40F085800022A44B0120CF
:10959000C3F81028C3F82028FEF7B2FE002840F0D8
:1095A00089809E48FEF784FE00287CD1284605B0BD
:1095B000BDE8F08F012BBDD1B8F5803FBAD3994DEE
:1095C000284605B0BDE8F08F974D284605B0BDE8A8
:1095D000F08F636B072B00F2CA8009FA03F919F0C8
:1095E0008A0F40F0D38019F0440F40F0C28019F088
:1095F000010F00F0BC8033793A795B0002F0010280
:1096000003F002031343864A31683868C2F80C3B02
:10961000636B23F00403032B0AD0236E012B0BBFD3
:10962000C2F8280DC2F8300DC2F82C8DC2F8348D66
:10963000E36D4FF40060012B794B0BBFC3F8281C7E
:10964000C3F8301CC3F82C8CC3F8348CFEF784FDAF
:109650000546002895D1626B072A15D8012393404F
:1096600013F08A0F40F09F8013F0440F0CD06C4B26
:10967000D3F860242260D3F864246260D3F86824AD
:10968000A260D3F86C34E3600123A365BAF1000F44
:109690003FF47BAF0423202104F1100084F83C3018
:1096A000FEF7E6FD71E76148FDF7D2FE284605B0FA
:1096B000BDE8F08F5E48FDF7CBFE72E75D48FDF731
:1096C000C7FE4CE75C48FDF7C3FE42E7216B206C08
:1096D00000F0B8F928B14FF0010A32E74FF47105F4
:1096E00064E7DFF858914E4DD9F800301B68C5F893
:1096F0000034D9F800305B68C5F80434D9F800307C
:109700009B68C5F80834D9F80030DB68C5F80C341C
:10971000D9F800301B69C5F81034D9F800305B69FE
:10972000C5F81434D9F800309B69C5F81834D9F855
:109730000030DB69C5F81C34216B0229CBD8236DBE
:109740004FEAC10A0193E36C0AF1100A04F1100B0D
:109750000093CDF80CA0CDF808B0206CD4E911230B
:1097600000F09CFA68BB002384F83C30B3E7344D2A
:1097700007E72368CBF860346368CBF86434A368E8
:10978000CBF86834E368CBF86C3434E72368CBF863
:1097900040346368CBF84434A368CBF84834E368BA
:1097A000CBF84C3427E71E4BD3F840242260D3F883
:1097B00044246260D3F84824A260D3F84C34E360B8
:1097C00062E7D9F8003051461B685846C5F80034A6
:1097D000D9F800305B68C5F80434D9F800309B68CC
:1097E000C5F80834D9F80030DB68C5F80C34D9F86E
:1097F00000301B69C5F81034D9F800305B69C5F832
:109800001434D9F800309B69C5F81834D9F8003001
:10981000DB69C5F81C34FEF72BFDA4E7200300200C
:10982000005084500500F1000B00F100ACE3000093
:109830008CE300006CE3000054E300000C03002004
:109840000100F1002DE9F04701B3FAB10446002808
:1098500054D01D46436B0E46072B1BD05DB9032B1E
:1098600010D1836D73B945668566C5660567102599
:1098700000F164030B602B4631462046BDE8F047FB
:10988000FFF744BE2F463846BDE8F087644F3846A0
:10989000BDE8F087C36DA3BBB5F5805F36D20DB9C7
:1098A000A36D9BBB4FF0FF315E48FEF7F9FC00282B
:1098B0004CD10020FEF724FD002843D14FF00108D1
:1098C000DFF864912046C9F81088C9F82088FFF7AE
:1098D00007FD0746E0B10022534B0120C3F81028D2
:1098E000C3F82028FEF70CFD40BB4E48FEF7E0FC15
:1098F0000028C8D04D48FDF7ABFDC4E74FF4710711
:10990000C1E7012BCBD1B5F5803FC8D3484FBAE7AB
:109910002046FFF749FD07460028DCD1636B072B83
:109920000AD808FA03F818F08A0F13D118F0440F78
:109930005AD118F0010F19D13E4FCCE73E48FDF740
:1099400087FDD2E73D48FDF783FDB7E73C48FDF7CB
:109950007FFDAEE72368C9F840346368C9F8443432
:10996000A368C9F84834E368C9F84C3401212E4A89
:10997000C2F87C14C2F8BC54337930688B4003F0D1
:109980000203C2F80C3BE5B9A36D0BB9C2F824156C
:10999000626B072A9FD80123934013F08A0F30D1BE
:1099A00013F0440F97D0204BD3F860242260D3F8F3
:1099B00064246260D3F86824A260D3F86C34E36056
:1099C00089E7E36D012B0BBFC2F8280CC2F8300CFD
:1099D000C2F82C5CC2F8345C4FF40060FEF7BCFBAC
:1099E0000028D5D0074676E72368C9F86034636855
:1099F000C9F86434A368C9F86834E368C9F86C34FA
:109A0000B4E7094BD3F840242260D3F844246260C1
:109A1000D3F84824A260D3F84C34E3605BE700BF7E
:109A20000B00F1002003002000508450ACE3000044
:109A30000500F1000100F1008CE300006CE3000080
:109A400054E300007F2809D851B10139022909D80F
:109A500005497F280CBF0846002070470248704720
:109A600008467047014870470100F7000300F700FF
:109A70007F2809D851B10139022909D805497F2821
:109A80000CBF0846002070470248704708467047E0
:109A9000014870470100F7000300F7000129F0B406
:109AA00007D0022900F0898000295AD07248F0BC02
:109AB00070470022714C724B4FEAC00CC4F800157D
:109AC000451C0CF57F04C3F8082104F50444C3F8D1
:109AD0000021C3F80421C3F800556A4E2468B4423B
:109AE00040F0B380196002E0002940F0B580D3F85F
:109AF0000021D3F80841D3F804112243F4D0002CFC
:109B000040F0B180002940F0A78001245B4AC3F8EF
:109B100000150230C2F800455B4AC3F80811C3F8CB
:109B20000011C3F80411C3F8000552F80C00574A9D
:109B3000904240F08E80524A1C6002E0002840F0C3
:109B40008B80D2F80031D2F80811D2F804010B430F
:109B5000F4D0002940F08C8000287DD1C2F80005A7
:109B600028E00124464BC200444E204402F57F0207
:109B7000C6F8004502F50442C3F80811C3F8001105
:109B8000C3F80411C3F800053E4D1268AA4260D123
:109B90001C6001E000285FD1D3F80021D3F8081140
:109BA000D3F804010A43F5D000295CD1002853D131
:109BB000C3F800050020F0BC704701250022304B9F
:109BC0002E4F4FEAC00C44190CF57F01C7F8005521
:109BD00001F50441C3F80821C3F80021C3F80421AA
:109BE000C3F80045274E0968B1422ED11D6000E040
:109BF00091BBD3F80021D3F80841D3F804112243D4
:109C0000F6D084BB41BB01241C4AC3F800150230C6
:109C1000C2F800451C4AC3F80811C3F80011C3F884
:109C20000411C3F8000552F80C00184A904210D1F4
:109C3000134A1C6000E078B9D2F80031D2F808115C
:109C4000D2F804010B43F6D083E7C3F8002510488F
:109C50002DE7C3F80015FAE70022094B0D48C3F8B9
:109C60000025F0BC70470022C3F800250A481EE713
:109C70000023C2F80035F9E70C00F10000408450E1
:109C800000900350005484500884FF001054845006
:109C90000600F7000200F7000100F7002DE9F04789
:109CA0000024CCB0824689461646214674220EA86E
:109CB0001F46579DDDF8588103F0B7FE80222146EC
:109CC0002CA82B9403F0B1FE8423B5F57F6FCDE96A
:109CD0000A440D940C94059364D8FFF7EFFB05AB91
:109CE00030462BAE01933946DDE9542302950096A8
:109CF00000F064F8002850D1022307228DF81330B9
:109D00009DF813301B928DF874300022012301243A
:109D100010211C900EA8CDE92423CDF86890CDF831
:109D200078A02694FEF7A4FA10220DF120090092E3
:109D3000304605990AABCDF8049006AAFFF734F92E
:109D4000074688B11EE0102D2E4628BF10260EA90A
:109D50003246FEF789FA10210EA8FEF789FA01347F
:109D6000AD1B3744E4B222D0059B4A4606A90EA893
:109D70008DF8AC40FFF766FD034608EB0700002BAB
:109D8000E1D01F460EA874220021FEF76FFAFFF7FC
:109D900095FB38464CB0BDE8F087064F38464CB0CE
:109DA000BDE8F087044F38464CB0BDE8F0872F4639
:109DB000E8E700BF0E00F1000F00F1002DE9F041CF
:109DC000002482B00A9D0194B5F57F6F40D8ED0064
:109DD000B5F5807F1E4634BF0323042301F1FF3C09
:109DE000BCF13F0F0C46009332D888B3174666BBD0
:109DF000089A6AB3099A116851B3A2191344994297
:109E000026D3089B01462246581CFEF72DFA089BD4
:109E100004F102081C440023637026BB089BFF2D3D
:109E2000009503EB080017D92B029BB243EA1523D8
:109E3000022201A90193FEF717FA08F1020300209C
:109E4000099A136002B0BDE8F0810AB1402ECFD963
:109E5000094802B0BDE8F08101226946FEF704FA24
:109E600008F10103EBE7089B324603EB0800394693
:109E7000FEF7FAF9B044D1E7060000800020187020
:109E8000704700BF08B5054B044613B10021AFF37E
:109E9000008000F0ABFA2046F7F7CEFD000000008E
:109EA000F8B50E4B06461D68AB789B0712D56F6858
:109EB00016F8014B29462CB90A20B847002805DBC3
:109EC000204609E02046B8470028F1DAAB7843F095
:109ED0000403AB704FF0FF30F8BD00BF44E1000059
:109EE0000CB430B589B005460C461C22002101A8EF
:109EF00003F09BFD022305958DF806300D4B029370
:109F000023462CB1B4F1004F28BF4FF00043013B72
:109F10001D440DAA0C9901A80695009200F00CF8BA
:109F200014B1059B00221A7009B0BDE8304002B0A0
:109F3000704700BF63DB00002DE9F04F43688DB030
:109F400015468046029383789A0740F10D810024DC
:109F50000E78002E00F00A81252E0BD04B1C0393A7
:109F6000013441463046029B98470028C0F2F680F3
:109F70000399EDE74E788B1C252E0393F0D0002734
:109F8000B946BB46BBF11F0F38D8A6F12003102BF2
:109F90000AD8DFE803F02A0909300909092109096B
:109FA0000928092D09091F00A6F13003092B33D90F
:109FB0002A2E37D11BF0400F55F8043B40F0828029
:109FC000002BA7BF4BF0200B9946C3F100094BF0C3
:109FD000280B01E04BF0010B039B13F8016B03937B
:109FE000002ECFD130E04BF0020B4BF0040BF3E727
:109FF0004BF0080BF0E74BF0100BEDE7BBF17F0FD8
:10A0000019D8A6F13003092BD2D81BF0400F03D08A
:10A010000A2101FB0737DFE70A214BF0200B01FB88
:10A020000939D9E72E2E06D11BF0400F40F09E8053
:10A030004BF0400BD0E76C2E31D02BD8682E36D0A9
:10A040006A2E3CD04C2E3AD0002F46F02003B8BFE9
:10A050002BF04002A3F16501BCBF00271FFA82FB71
:10A06000022901D9612B2FD107350727DFF8ACA2D0
:10A0700025F0070508351BF0080F66D00AEB070B23
:10A0800056465E4563D1A4EB0A0AA9EB070906EB25
:10A090000A026FE1742E9FD07A2E9DD0D4E71BF078
:10A0A000800F18BF4BF4007B4BF0800B94E71BF440
:10A0B000807F18BF4BF4007B4BF4807B8CE74BF424
:10A0C000207B89E71F4687E7A6F16301122900F28A
:10A0D000F080DFE811F013004F00EE00EE00EE001C
:10A0E000EE004F00EE00EE00EE00EE00EE00FE008F
:10A0F000E900EE00EE001B00EE00AF0055F8043B57
:10A1000001270DF1180A8DF81830B4E755F804ABA3
:10A11000834BBAF1000F08BF9A461BF0400F504620
:10A1200014BF39464FF0FF3103F0B9FC0746A2E7F0
:10A1300041462020029B984700280FDB013EB74292
:10A14000F6D34C44B146A41B98E74E46F7E7414688
:10A1500016F8010B029B9847002892DA98F8023013
:10A1600043F0040388F802304FF0FF3420460DB06E
:10A17000BDE8F08F1BF0800F34D01BF4007F2CD093
:10A18000073525F00705AA4669685AF8080B2BF031
:10A1900010050029ADB237DA404245F4806561EB25
:10A1A00041010DF1180B0A235A4603F084FCA0EB81
:10A1B0000B0301936B0662D5019B25F001019F42C1
:10A1C00089B240F3A180002E00F0998015F01002B2
:10A1D00040F09C80BB460D4623E0AA465AF8040B8B
:10A1E000C117D4E7AA461BF4807F5AF8041B01D19B
:10A1F0000846F5E71BF4007F19BF48B241F3C011D0
:10A2000008B241F3C031C2E750EA0103C9D11BF0E3
:10A21000400FC6D0002FC4D12BF01102BB460197CE
:10A2200095B240F2064115EA01021CBF0BF1010B89
:10A2300000222CE02BF010020A231FFA82FB1BF0F5
:10A24000800C49D01BF4007115BF0735AA4625F0D4
:10A2500007055AF8040B1EBFAA4669685AF8080B8E
:10A2600050EA010545D12BF016051BF0400FADB2A9
:10A2700042D0002F40D12BF01702019795B215F074
:10A28000100248D0019B002E42D103F1010B290797
:10A290005AD4EB0706D5D9456FDDA9EB0B0301991D
:10A2A000CB465F185B4649E04BF0100B1023782635
:10A2B000C5E7782B04D1C6F1780343F01003BEE75D
:10A2C00041462520029B98470028FFF647AF0234FD
:10A2D00047E608230026B2E7AA461BF480715AF825
:10A2E000040BBDD01BF400711ABFC0B2614680B22E
:10A2F000B6E72BF0060295B20DF1180B54E725F0E6
:10A300001105BB46ADB28CE70D46B8E73B460D469E
:10A3100003F1020BBBE7DDF804B082E73AEE000080
:10A3200033EE0000CDE9043241462020029B9847DD
:10A330000028FFF613AF049B059A01339945F1DC21
:10A34000A4EB0B019B46CC180AB341463020029B7C
:10A3500098470028FFF602AF8EB901342744391B15
:10A36000019B994224DC1D4655BB019AA9EB0B09C0
:10A37000554622441446914433E0019F92E702344B
:10A3800041463046029B98470028E7DAE6E640F26D
:10A3900006410D42E2D015F0020F04F101044146DE
:10A3A00014BF2B20202015F4806F18BF2D20E9E763
:10A3B00041463020029B013498470028CFDACDE691
:10A3C00006AB013D4146585D029B98470028CBDA19
:10A3D000C4E641462020029B013498470028FFF63E
:10A3E000BDAEA9EB0403002BF3DCC1E538B5074D86
:10A3F000074C641BA41024B9064B0BB1AFF30080CB
:10A4000038BD013C55F824309847F4E700000000BF
:10A4100000000000000000007047836800EBC101ED
:10A42000B3F5004F2CBF51F8220031F812007047ED
:10A4300000EBC1018068B0F5004F2CBF41F822301D
:10A4400021F812307047012208B5FFF7E6FFD0402F
:10A4500008BD836800EBC101B3F5004F08D34B681A
:10A460001AB143F001034B60704723F00103FAE790
:10A470004B881AB143F001034B80704723F001036E
:10A48000FAE753000122FFF7D3BF8368B3F5004F0B
:10A4900034BF04230823C91A081AC0087047836808
:10A4A000481CB3F5004F34BF042308230833A0EB46
:10A4B000D300B0FA80F0C0F11F0070472DE9F041E1
:10A4C000174603220E460446FFF7A7FF86420546BD
:10A4D00007F104080AD10122E368BA4023EA020323
:10A4E000E360002344F82830BDE8F08131460222C1
:10A4F0002046FFF792FF06462B46014603222046E0
:10A5000044F82850FFF794FF334629462046BDE81B
:10A51000F0410222FFF78CBF70B50D4686680446F5
:10A52000FFF791FFB6F5004F014601D3012809D08E
:10A530002046FFF7B4FF294602462046BDE870409A
:10A54000FFF7BCBF70BD2DE9F0470546FFF7A7FF39
:10A5500005EB800ADAF8109088460646B9F1000F3C
:10A560001BD00327DAF8104028462146FFF76BFF7F
:10A57000404507D3324621462846FFF79FFF204635
:10A58000BDE8F087032221462846FFF746FF013F3A
:10A59000CAF8100001D08145E4D14FF0FF34EB68D8
:10A5A0000136B4401C40EAD094FAA4F2B2FA82F226
:10A5B000131D55F82340DEE72DE9F04114460E4601
:10A5C0000546FFF740FFA4EB0608371B0744424649
:10A5D00031462846FFF755FF3A4621462846FFF701
:10A5E00050FF4346002221462846FFF721FF21461F
:10A5F0002846FFF728FF3B46211800222846BDE8E1
:10A60000F041FFF715BF2DE9F041164604460F460D
:10A61000FFF719FF314605462046FFF714FF0544B2
:10A620002A4639462046FFF72CFF31462046FFF7E1
:10A630000AFF2B46311800222046BDE8F041FFF703
:10A64000F7BE2DE9F0410D4686680446FFF7FBFE94
:10A65000B6F5004F014601D3012832D02046FFF75E
:10A660001EFF04EB80010E6996B90122E368824067
:10A670001343E36002220D612B4629462046FFF773
:10A68000D7FE032229462046BDE8F041FFF7D0BEA1
:10A69000022231462046FFF7C0FE07460346294600
:10A6A0002046FFF7C5FE0322334629462046FFF722
:10A6B000BFFE39462B462046FFF7BAFE022231463E
:10A6C000E1E7BDE8F081F8B50C460546FFF7BBFEB3
:10A6D0002618012231462846FFF79FFEC3070CD4F7
:10A6E00031462846FFF718FF21462846FFF7ABFE04
:10A6F000214622182846FFF786FF002221462846D9
:10A70000FFF78BFE271A012239462846FFF785FE00
:10A7100010EA020613D139462846FFF7FDFE21460E
:10A7200032462846FFF779FE2246211A2846FFF7CF
:10A730006AFF214632462846FFF76FFE241A21465B
:10A740002846BDE8F840FFF77CBF38B571B1056811
:10A7500000222846FFF799FE044601462846FFF7E7
:10A7600078FE2146BDE83840FFF7ADBF38BD70B573
:10A77000056809B9002070BDAB6801F00704B3F5A6
:10A78000004F2CBF0822042207341444E40804EBD1
:10A79000D1049C4228BF1C4628462146FFF7D3FE21
:10A7A00006460028E6D001462846FFF74CFEA042A8
:10A7B00009D93444314628462246FFF7FDFE21469A
:10A7C0002846FFF73EFF284601223146FFF741FEAB
:10A7D000AB68B3F5004F34BF0423082303EBC60373
:10A7E0001844C8E71146FFF7C2BFB2F5802F2CBF4F
:10A7F000082304232DE9F0410026D21A8C18CD1D20
:10A8000025F0070524F00704641BE40805602146D1
:10A810002846AC60EE60FFF742FE421D9200013018
:10A8200002F107074FEAD7073146A2F1100205F1FE
:10A830001000B8BF324603F0F8F83A4631462846D1
:10A84000FFF71FFE3346324631462846FFF7F0FD3C
:10A85000A4EB0708284631460122FFF7FAFD4246DD
:10A860003946FFF70EFE3B46324639462846FFF78B
:10A87000DFFD21462846FFF704FE434632462146C7
:10A880002846FFF7D5FD214628460122FFF7E1FDC6
:10A890003946BDE8F041FFF7D4BE002070470FB441
:10A8A00007B504A951F8040B0191F5F75FFD03B05A
:10A8B0005DF804EB04B070470FB407B504A951F874
:10A8C000040B0191F5F752FD03B05DF804EB04B001
:10A8D0007047038B13F0070305D10368002B0CBFEF
:10A8E000002003207047022B05D1408BB0FA80F086
:10A8F000400980007047012B05D10368002B0CBF75
:10A900000020052070470020704710B50C4600B1AC
:10A9100011B96FF0150010BD081D00F0B7F8002840
:10A92000F9D1A368032BF6D9F3E72DE9F0410D46E1
:10A9300007461946281D90461E4600F0BBF80446FF
:10A9400038B13346424629463846A446BDE8F04170
:10A950006047BDE8F08110B4EFF31182202484F346
:10A960001288BFF36F8F416110BC0121F5F730BD34
:10A9700038B50C46054658B151B10B6843B14B6828
:10A9800033B11C22002103F050F800202C6138BDA7
:10A990006FF01500FBE770B505460E46FFF7B5FFF3
:10A9A000041E14DBEFF31182202383F31288BFF31C
:10A9B0006F8F4FF6FF716B8B2C8B8B4204F007046B
:10A9C00007D182F31188BFF36F8F6FF00A0420461E
:10A9D00070BD022C0CD101336B8382F31188BFF35D
:10A9E0006F8F0023224631462846FFF79EFFEEE791
:10A9F000062C14D8DFE804F004131313041A04001F
:10AA0000002333606B683BB9C5E90066ACB902212D
:10AA10002846F5F7DDFCDAE71E606E60F6E782F3A4
:10AA20001188BFF36F8F6FF00404D0E782F31188B1
:10AA3000BFF36F8F6FF08504C9E782F31188BFF30E
:10AA40006F8FC4E710B5EFF31182202383F31288D0
:10AA5000BFF36F8F048B04F00704022C0AD0012C83
:10AA60000CBF6FF004006FF0850082F31188BFF314
:10AA70006F8F08E0438B013B9BB2438323B9214690
:10AA8000F5F7A6FC204610BD2046EEE7034640B190
:10AA9000426802F00302022A06D0032A04D0012AE7
:10AAA00005D06FF0150070471A68002AF9D0002011
:10AAB0009860704710B54268034602F00302022A0C
:10AAC0004FF00004816007D0032A02D05C600020B0
:10AAD00001E018685C6010BD18685C600028F6D062
:10AAE000FCF71CF9F3E7704720B183682BB11B68B2
:10AAF00033B118476FF0150070476FF004007047CE
:10AB00001846704720B183682BB15B6833B1184792
:10AB10006FF0150070476FF00400704718467047DB
:10AB200030B450B149B142B1846854B1256945B1DE
:10AB300041F8040B236930BC18476FF0150030BC96
:10AB400070476FF00400FAE710B5044650B1006892
:10AB500058B1836863B15B6953B16168984700B9C4
:10AB6000206010BD6FF01500FBE76FF00100F8E703
:10AB70006FF00400F5E730B41346044650B10068A6
:10AB800060B182686AB195685DB10A46AC46616899
:10AB900030BC60476FF0150030BC70476FF00100AB
:10ABA000FAE76FF00400F7E70369D3F8B0037047E2
:10ABB0006FF085007047084608B5114618B101F0DE
:10ABC00055FF002008BD6FF00100FBE7084608B5FF
:10ABD000114618B101F041FF002008BD6FF00100DF
:10ABE000FBE713B504460846216901F56B71D1E80E
:10ABF000AF1F022909D15BB168B100931346D0E9B8
:10AC00000912FAF791FB02B010BD6FF00F00FAE7DE
:10AC10006FF04C00F7E76FF00100F4E72DE9F8431F
:10AC20001C46DDE90853164698460F46006939B3BD
:10AC30004AB344B36A1C43F10003022A73F10003D0
:10AC400024D2226842B1D0F8B0339A4204D96FF0CE
:10AC50000B002360BDE8F88305EA080909F1010348
:10AC60005A425A412146384601F009FF88B9B8F1E5
:10AC7000FF3F08BFB5F1FF3FF0D06FF06800E9E794
:10AC80006FF00100E6E76FF01500E3E76FF0850075
:10AC9000E0E730600020DDE701F056BF38B50D4633
:10ACA000044600F148012846F5F754FA30B1284629
:10ACB00004F1C001F5F74EFA20B90120782303FB17
:10ACC000004038BD0020FCE702F5307102F5347019
:10ACD00002F008BCD0F8E830A0F53070003B18BF97
:10ACE000012300EB8300D0F8AC0201F057BEC86826
:10ACF00028B1096983681B680BB1002218477047A7
:10AD0000FAF7B0BFD0E8EF3FC0E8E21F002AF9D160
:10AD1000704710B5436804691B68C4F8A83304F58C
:10AD2000EC7002F0ACFA002104F56B70FFF7EAFF5B
:10AD3000084610BD2DE9F74317460D4691B30B7831
:10AD400083B3D0F8C440A4F5E27914344FF0FF3255
:10AD50004FF0FF332046FAF70DFF2A46484601A977
:10AD6000F5F770FC019E80462EB9204603B0BDE881
:10AD7000F043FFF7C5BF58B12046FFF7C1FF3B4680
:10AD80002A463146484603B0BDE8F043F5F738BCE3
:10AD90001F22294606F1480002F071FE86F86780FE
:10ADA000B766E2E703B0BDE8F083030103EB4003BD
:10ADB000093323F0030303EBC00348430330083394
:10ADC00020F003001844400070472DE9F843064680
:10ADD0004FF001080569D0F8049005F56B77D7E8C6
:10ADE000EF3F022B03D1C7E8E28F002AF7D141D110
:10ADF00095F86C30002B40D195F8E430002B3CD115
:10AE00002846D5F8A81300F054F8044680BB7368B0
:10AE10003669D3E9050183681B693BB3224698472D
:10AE2000044628BB414606F53470FBF781F9D6F895
:10AE3000880305F5F876F6F7C1FA3046D9F8001020
:10AE400000F072F8044698B90146D022304602F06C
:10AE5000ECFD21464FF4F672284602F0E6FD21464D
:10AE60003846FFF74FFF2046BDE8F8836FF05704E0
:10AE70000221F5E76FF07704F5E76FF00F04F2E7D2
:10AE800010B50846029B114652B993F86C202AB9B6
:10AE90000122184683F86C20F5F7CEFC002010BD87
:10AEA0001A6F9468002CF9D05A6FA047F6E701F0AA
:10AEB0004BBE38B50D46044660B1F03002F0E3F801
:10AEC0000DB1002038BDC4F8C451C4F8C851C4F84D
:10AED000CC51F6E76FF01500F4E70268D2F8C830FD
:10AEE00013B1D2F8C41018477047704783690BB983
:10AEF000C36B19707047012070478369012B03D120
:10AF0000C36B1878C0B270470420704738B5C41DB1
:10AF1000E4002046FBF746FF054618B12246002113
:10AF200002F083FD284638BD38B50446382200219A
:10AF300002F07BFD1822002104F1A40002F075FD4F
:10AF40001822002104F18C0002F06FFDD4F8C0003B
:10AF5000FAF79CF9D4F8BC00FAF798F9D4F88030E5
:10AF600004F154050BB128469847382200212846A1
:10AF700002F05BFDFAF7EEF8002038BDFEE702F0C4
:10AF800054BD02F02BBD01460068F5F74FBF08B570
:10AF9000F5F77CFFBDE80840F5F79CBF00210120D4
:10AFA000F5F744BFD0F8983083F30B8870476FF003
:10AFB0008500704761B662B680F31188BFF36F8F6A
:10AFC000704708B572B6002383F31188BFF36F8F03
:10AFD000F6F750FE50B1BFF34F8F30BF00BF00BF38
:10AFE00000BF00BF00BF00BF00BF00BF62B6BFF31D
:10AFF0006F8F08BD10B5044672B6002383F3118825
:10B00000BFF36F8FF6F736FE50B1BFF34F8F20BFFF
:10B0100000BF00BF00BF00BF00BF00BF00BF00BF38
:10B0200084F31188BFF36F8F62B610BD40E800F360
:10B0300013F4803FD8B208BF6FF01500704730B5E9
:10B040000C684B6885B00A894D890094013B24F057
:10B050001F04234402F01F0242EA451223F01F039B
:10B0600069468DF808200393F6F704FB05B030BD60
:10B0700008B5F6F7E9FC002008BD704700230382FD
:10B080004369C3607047416A8968F6F749BDEFF3C9
:10B090001182202383F31288BFF36F8F00230B608C
:10B0A000436833B9C0E9001182F31188BFF36F8F91
:10B0B000704719604160F7E7034610B5EFF311815F
:10B0C000202282F31288BFF36F8F006828B15C687A
:10B0D0000268A0421A6008BF5A6081F31188BFF36A
:10B0E0006F8F10BD027A01320272704783680B4481
:10B0F000036070478388026819448180D0187047C4
:10B1000030B484880568A3188380281930BC02F005
:10B1100065BC10B5838802685C1C8480D154D0184B
:10B1200010BD838830B502689D1C8580D418D15429
:10B13000090A617030BD034600689A88401A1144BC
:10B140001860998070470268531E0360838801333A
:10B15000838002F8011C704703468288521A82805D
:10B160000068084418607047034600689A88521ABD
:10B1700001449A801960704710B5036801211C785A
:10B18000FFF7EAFF204610BD02688068101A70477A
:10B190008388C2888168D21A03685B1AD01A704704
:10B1A0004FF05023012270B50C460546C3F8142613
:10B1B0000020F6F7E5FD28462346BDE87040002153
:10B1C0001847012310B50621044600F8013B00F0A2
:10B1D00095FA18B9A37963F03F03A37110BD0B680A
:10B1E00003608B8883808B798371037823F002035B
:10B1F000037070470078C0F34000704738B50446CC
:10B20000807AF6F763FC6169054649B1637ADB072A
:10B2100004D4436A20461B689B68984700236361F7
:10B2200021462846BDE8384002F0D1B8034610B5A3
:10B23000D3E8EF0F40EA0102C3E8E42F002CF7D176
:10B2400010BD01210C30FFF78FBF30B40446084613
:10B2500002EBC3039A4201D130BC7047114611F88A
:10B26000085BA54206D1018A53789942F4D330BCD9
:10B27000536818470A46EDE7D0E8EF3F0B40C0E8B7
:10B28000E23F002AF8D17047072208B502F0D5FB4B
:10B29000B0FA80F0400908BD00280CBF0846002025
:10B2A000704770B50D460446002845D0002943D0AC
:10B2B00000F11803D3E8AF2F920711D40A68C0F841
:10B2C00009208A88A0F80D2001220272D3E8EF1F1E
:10B2D00041F01001C3E8E21F002AF7D1002070BD41
:10B2E0004FF0FF304FF0FF31F6F7F2FF064630B374
:10B2F00007210C30FFF7FEFE03466278314603F863
:10B30000012B2A68C0F80120AA8842F235009A80F1
:10B310000022F7F761F80028E1D104F109039D420A
:10B320004FF001031EBF2A68C4F80920AA882372BF
:10B3300018BFA4F80D20D1E76FF01500CFE76FF02C
:10B340006800CCE713B5044680B10621684600F0DA
:10B35000D5F948B99DF80530694603F03F0320460A
:10B360008DF80530FFF79DFF02B010BD6FF015009E
:10B37000FAE71830D0E8EF3F23F02003C0E8E23FBF
:10B38000002AF7D17047D0E8AF0F084100F0010064
:10B390007047034610B5D3E8EF0F00EA0102C3E897
:10B3A000E42F002CF7D110BD2DE9F8430025044609
:10B3B0000F461646A8462068A268E36850F8321087
:10B3C000B4F810E001EBC301497800EBC20C023184
:10B3D0008E450BD1A4F81080DCF8041001338B42A9
:10B3E00003BF0132C4F80C80A260E360D4E90123FA
:10B3F000934214D0D4F80CC050F8332012EBCC0395
:10B400000DD0218A781981B95B7801337B55238A65
:10B41000013501339BB2EDB2B5422382CBD36369D0
:10B4200028465B1B6361BDE8F883012903D112F84C
:10B430003C300370EBE793F80190721BA9EB010914
:10B4400009F10209914528BF91465B6802394A46D5
:10B45000194402F0C3FA238A4B44A9449BB25FFA11
:10B4600089F5D9E738B5102204460D460830002189
:10B4700002F0DBFA012340F2726063600023256072
:10B480006A68934201D3002038BD2A68616902EBE3
:10B49000C302527802310A448242626101D8013308
:10B4A000EEE76FF01500EFE7012310B403FA01F1A6
:10B4B000044642B1D4E8EF3F0B43C4E8E23F002A20
:10B4C000F8D110BC7047C94310BCFFF762BF01231D
:10B4D0008B40D0E8EF2F1A43C0E8E12F0029F8D1C4
:10B4E000704773B51D469DF81C3004469DF82060DA
:10B4F00063B15EB1069B6A4642F238012046009570
:10B500000193F7F7EDFC68B102B070BDCDE9001210
:10B5100020466A4642F23701F7F7E2FC0028F3D1F1
:10B52000002EE7D104F118000221FFF7D0FF002020
:10B53000EAE72DE9F04180460F464FF0FF304FF02B
:10B54000FF3186B01446F6F7C3FE064688B300F115
:10B550000C0537B301212846FFF7DBFD0121284602
:10B56000FFF7D7FD284698F80110FFF7D2FDD4B1B8
:10B5700021882846FFF7D5FDA1782846FFF7C9FDA9
:10B58000304608F1180203A908230097F6F78EFE4B
:10B590000022314642F23900F6F71EFF06B0BDE840
:10B5A000F0813946D7E721462846FFF7BAFD214604
:10B5B000E3E76FF06800F1E7203001F0C4BF70B539
:10B5C0000C460546B8B300F1180608213046FFF7CF
:10B5D000DAFE98BB24B3238823BBA278003A18BFB5
:10B5E000012207213046FFF75FFF09213046FFF7B0
:10B5F000CAFE70B90C213046FFF7C5FE48B96FF09E
:10B6000008013046FFF7C5FE03070DD42846FFF7B3
:10B6100099FE22462846BDE870400121FFF789BF08
:10B620002246DEE70122DCE70E213046FFF7ABFEC3
:10B630000028EBD1EDE76FF0150070BD6FF07700DB
:10B64000FBE72DE9FF41DDF828800F460446F8B1FD
:10B6500000F118060B213046FFF795FE05460A213A
:10B660003046FFF790FE45B128B9B8F1000F04D07D
:10B670006FF0850009E0002AFAD1CDE90150394682
:10B680002046CDF80080FFF72CFF04B0BDE8F08124
:10B690006FF01500F9E70121F7F7D0BB7FB5C5685A
:10B6A0002878F7F79FFE044698B143688BB19B68F2
:10B6B0007BB101352846FFF79DFD02AE294650B10A
:10B6C0003046FFF78CFD636820469B68019601A910
:10B6D000984704B070BD2078FFF7DEFD0346006890
:10B6E00002909A889B79B280B371ECE708B5FBF7BA
:10B6F000C5FD002818BF6FF0040008BD08B5FBF7B2
:10B7000063FD002818BF6FF0040008BD2DE9F0416B
:10B7100007460D4686B000F11806D6E8AF3F1A047A
:10B7200004D46FF0150006B0BDE8F081D6E8AF3F55
:10B730009B03F6D5D6E8AF3FC3F38043994223D0AD
:10B740004FF0FF304FF0FF31F6F7C2FD0446C0B1B5
:10B7500002210C30FFF7CEFC4FF00008A0F800806B
:10B760007B7832460370457003A92046122300956A
:10B77000F6F79CFD4246214642F25200F6F72CFEB7
:10B78000D1E76FF06800CEE76FF07700CBE70121DB
:10B79000FFF7BCBF00692830FAF7E6BAF8B504260F
:10B7A0000D460769374438462A8AE968FFF7E3F906
:10B7B00010F10C0F044606D14B2001F097FC013E1E
:10B7C000F1D12046F8BD0028FBDB2846F6F726FA23
:10B7D0000024F6E738B5046900200D46F8F740F874
:10B7E000B0B9206CFFF780F910B110F1780F0FD1CC
:10B7F000206C04F10C02211DFFF792F940B94FF4BF
:10B800008032002304F12800FAF7E8FA00B9256035
:10B8100038BD10B50469201DFFF796F9034648B9F5
:10B82000206CFFF76FF9034620B900F005F80346D6
:10B8300000B92060184610BD08B50020F6F70AFBD5
:10B84000002008BD0C220369C9B201FB0233986FC6
:10B8500000F00700704770B5C9B20369EFF31185B6
:10B86000202484F31288BFF36F8F0C2606FB01346B
:10B87000A46F14F0C00408D0A24206D085F311884A
:10B88000BFF36F8F4FF0FF3070BD012206FB013315
:10B890009A6785F31188BFF36F8F436803EBC10389
:10B8A0005B6898470020EFE78022FFF7D4BFF8B528
:10B8B000069F0469C9B2EFF31186202585F312882B
:10B8C000BFF36F8F0C2505FB0144A56F05F0070C36
:10B8D000BCF1010F0CD1A76786F31188BFF36F8FFE
:10B8E000C4E91C23436853F8313098470020F8BD61
:10B8F00005F0C005AF4286F31188BFF36F8F0CBF10
:10B900006FF077004FF0FF30F1E713B5802400941B
:10B91000FFF7CDFF02B010BD10B41C240069CBB2FC
:10B9200003FB0400002110BC1047032000F074BA90
:10B93000022000F071BA032000F07DBA022000F06E
:10B940007ABA1046FAF710BA00F0FEBAF9F7C6B89C
:10B950000020704708461146F6F7C4BD002208B51E
:10B9600011461046FBF79EFD002818BF6FF015002A
:10B9700008BDF7B50F4616464FF480650024A64271
:10B9800003D816D0162003B0F0BD331BB3F5806F7B
:10B9900038BF1D4600202A4601AB3919FBF7B2FD1E
:10B9A00020B9019BAB4201D12C44E8E76FF01500B0
:10B9B000E9E70020E7E7436800205B681B690B604C
:10B9C0007047436802EA01005B6821EA020198605F
:10B9D0000020D9607047436800205B689960704719
:10B9E000436800205B68D960704743685A685368B1
:10B9F00021EA03000B4090600020D360704710B52F
:10BA000003695868F8B1884219D19C680868A14256
:10BA1000586000D19860002008602AB15A680A6016
:10BA20009A68596002B99960002010E0814206D1FD
:10BA30000868206098688142EDD19C60EBE704467D
:10BA400000680028F2D1002AE8D16FF0150010BD7F
:10BA5000F9F786B930B451F820500C4601EB80025A
:10BA60003DB10146AC46D4F88000002330BC126CD6
:10BA7000604730BC704710B500690F299FBF00EBCD
:10BA8000810440F821202364002088BF6FF0150056
:10BA900010BD00207047102070470F290ED8436852
:10BAA0005B68CB40DB0709D501228B00DBB203F1D9
:10BAB000A04303F5283300201A6070476FF015008B
:10BAC000704738B50F290C46056933D843681B68A1
:10BAD000CB40DB072ED5D5F8841021FA04F303F010
:10BAE00001031AB99BB96FF0770022E0002BFAD15D
:10BAF00011B92A20F5F7BEFC0122D5F88430A24006
:10BB00001343C5F88430E0B2F9F744FA0AE0E0B232
:10BB1000F9F748FA0122D5F88430A24023EA02035B
:10BB2000C5F88430D5F8843013B92A20F5F7B0FC75
:10BB3000002038BD6FF01500FBE730B54368136097
:10BB4000057A446804EBC504A34202D36FF00100F8
:10BB500030BD5C798C4201D00833F0E70020F7E774
:10BB600043681B68D3F88004C3F8800470474268B8
:10BB70001368D3F8100150B10020126A12780A70CD
:10BB8000C3F81001D3F8102101221A6070474FF05A
:10BB9000FF30704702680346D2F8580140B95B682D
:10BBA000DB0706D4D2F82001003818BF0120704707
:10BBB0000120704743681B68D3F80423D20517D5CA
:10BBC000D3F82021A2B1EFF31182202181F3128852
:10BBD000BFF36F8FD3F8201131B10021C3F82011CA
:10BBE000D3F820110121D96082F31188BFF36F8F40
:10BBF000D3F85831704713B501AA0446FFF79DFFEB
:10BC0000002805DB019B226819791868F8F7C8F944
:10BC100002B010BD2DE9F0410546002201210820A7
:10BC2000F5F758FC0820F5F725FC6C680121E06861
:10BC3000FFF7E1FF6B6819682369C1F82435A27D1D
:10BC4000637D207D1343228B02431343C1F86C357F
:10BC50006E68D6E9004313F001033DD00027D5F804
:10BC6000108004F10C01C4F8A07108F10802C4F8B6
:10BC70008C7004F5907000F0B0F800282ADB98F87A
:10BC80000800F8F7E3FD0823C4F80035F369C4F8A9
:10BC900044350123C4F84875A360D4F85831002B0B
:10BCA000FBD00021C4F800156D68E8682C68FFF728
:10BCB000A2FF0823C4F800352A7A52B92B6AC4F8C7
:10BCC00034350123C4F83835C4F81021D4F81021D4
:10BCD00023600020BDE8F0810822C4F80025F26945
:10BCE000C4F84425C4F848350123A360D4F82031B2
:10BCF000002BFBD00023C4F82031D4F820310123DD
:10BD0000E3604FF48073C4F80433C6E7002200F107
:10BD100050039B009BB203F1502303F580331A605C
:10BD20001B68704708B5F8F7E5FA08BD08B5F8F7DD
:10BD30007DFC002008BD08B5FBF7A0FA48B1002340
:10BD400083F31188BFF36F8F0423184602DF6FF06F
:10BD5000040008BDFBF748BB08B5F4F741FFF5F751
:10BD600027F8BDE80840FBF73FBB03460020184713
:10BD700001F0BCB9024610B5116891B1B1FA81F376
:10BD8000C3F11F000123834021EA0303D2E8EF4FF0
:10BD90008C4204D1C2E8EC3FBCF1000FF6D1EBD1EC
:10BDA00010BD6FF00B00FBE710B50368CB40DB075D
:10BDB00010D401238B40026843EA0201D0E8EF4F20
:10BDC000944204D1C0E8EC1FBCF1000FF6D1F2D1CF
:10BDD000002010BD6FF01500FBE770B5D0F8803083
:10BDE0000646002B0C46154613DBD1F88030002B9D
:10BDF0000FDB00210846F8F71BFD48B92B7843F00C
:10BE00000043C6F880302B7843F00043C4F88030FC
:10BE100070BD6FF01500FBE703280BD8DFE800F0DA
:10BE200002040608F8F75ABEF8F786BDF8F70EBE0A
:10BE3000F8F7C4BD704703280BD8DFE800F0040210
:10BE4000060800F02EB800F07FB800F062B800F0ED
:10BE500044B8704708B5F8F78BFDF8F783FEF8F79C
:10BE600013FEBDE80840F8F7C7BD38B54FF05024C1
:10BE70000123C4F808336360002342F21075C4F84C
:10BE80000031D4F80031D4F80C24D4F80C34D203A7
:10BE900006D5DB0704D50120FFF76AFF013DF2D18B
:10BEA00038BDFFF7E2BF38B54FF050244FF4807330
:10BEB000C4F808330123E361002342F21075C4F88B
:10BEC0002031D4F82031D4F85434DB0304D50120D8
:10BED000FFF74EFF013DF6D138BDFFF7E4BF38B59F
:10BEE0004FF050244FF40073C4F808330123636209
:10BEF000002342F21075C4F82431D4F82431D4F868
:10BF00005C34DB0304D50120FFF732FF013DF6D19D
:10BF100038BDFFF7E4BF38B54FF050240223C4F812
:10BF200008330123E360002342F21075C4F80431A2
:10BF3000D4F80431D4F81834DB0304D50120FFF71A
:10BF400017FF013DF6D138BDFFF7E5BFF7B516463F
:10BF5000DDE90847019001A81D46F8F73DFE019B69
:10BF6000B6F1000C18BF4FF0010C00EB83000B1E64
:10BF700018BF0123002D43EA4C0314BF4FF00C0CF3
:10BF80004FF0000C002C43EA0C0314BF4FF4706C0C
:10BF90004FF0000C002F43EA0C0314BF4FF4403C59
:10BFA0004FF0000CD0F8002243EA0C0322EA03030E
:10BFB00001B109780EB13678760019430DB12D78AC
:10BFC000AD0031430CB12478240229430FB13F78EE
:10BFD0003F040C433C43C0F8004203B0F0BD1FB522
:10BFE0000DF10F03019300238DF80F101A46194627
:10BFF0000093FFF7ABFF05B05DF804FB10B50446F6
:10C000000846F8F7FBFD04EB4004A08AC0F340109B
:10C0100010BD10B504460846F8F7F0FD04EB4004E7
:10C02000A08AC0F3400010BD10B504460846F8F7DA
:10C03000E5FD04EB4004A08A400B10BD70B504463A
:10C0400008461646F8F7DAFD083034F810300D4689
:10C05000DA0509D5C3F3432304EBC302314628466E
:10C0600054F8333052689847A3682BB131462846BC
:10C07000E268BDE87040184770BD10B50446084638
:10C08000F8F7BCFD00B204EB4000838ADA051DD549
:10C09000C3F3432123F4F853838204F1120204F121
:10C0A000720032F8023F13F4807F03D0C3F34323BE
:10C0B00099420BD08242F4D1002204EBC1035A60B2
:10C0C00004F17800BDE81040FFF76EBE10BDF0B57A
:10C0D0000446002001270546844695420AD1D4F83B
:10C0E0007C3133B10023C4F87C31D4F87C3140F08A
:10C0F0000040F0BDEBB29B0003F580769B0807FA89
:10C1000003F3194208D054F806E0BEF1000F03D043
:10C1100044F806C0A65918430135DEE738B5044691
:10C120000D46FFF76BFFB0B12046FFF772FF90B9E5
:10C130002046FFF779FF012322688340C2F80833C5
:10C14000236800B203EB8003D3F8102522F003022A
:10C15000C3F8102538BD2846BDE838400021FFF758
:10C160003EBF2DE9F0431746044685B00846F8F770
:10C1700045FDD7F800800E460546B8F1000F1FD0E8
:10C180002046FFF746FF18B12046FFF737FF30BBC8
:10C1900000230DF10F02CDE900338DF80E308DF83C
:10C1A0000F30304643460DF10E01FFF7CFFE2AB2A5
:10C1B00004EB4202938A23F0020343F001039382CB
:10C1C0007B68002B34D03146204693F80080D3F8AA
:10C1D0000490FFF71EFF28B1B9F1000F1FD06FF0D8
:10C1E000150028E028B204EB4000838A23F4604362
:10C1F00023F020038382B9F1000F10D0B8F1030FB0
:10C20000EDD87B6821685B6893F800C001EB8C0176
:10C21000B8F1000F12D1C1F81085C1F810852AB20B
:10C2200004EB4202938A23F01C0343EA88039382BF
:10C23000BB684BBB002005B0BDE8F083D1F81025EA
:10C2400022F00302C1F81025226802EB8C03D3F818
:10C25000102522F44F3222F44072C3F81025320226
:10C26000D3F8101502F47C5242EA08420A43C3F89C
:10C27000102504EB4C03A3F87C60838A43EA4C331B
:10C2800043F020038382CAE73146D3E90078204691
:10C29000FFF7F3FE002FCDD063689F4206D004F174
:10C2A0007800FFF767FD002804DAC4E7A368984523
:10C2B000F5D1002004EBC003C3E901782DB204EBF3
:10C2C0004505AB8AC0B243EA402343F48073AB8296
:10C2D000B0E72DE9F043054685B0084617461E46EF
:10C2E000F8F78CFC0C46804637B32846FFF791FEE2
:10C2F00018B92846FFF782FE28BB0FFA88F905EB2C
:10C300004909B9F8143013F01C0F02D07B78012BC7
:10C3100019D001238DF80F3000232046CDE900739A
:10C320007A1CBB1C0DF10F01FFF710FEB9F8143099
:10C3300043F00303A9F81430002E41D021462846CB
:10C34000FFF767FE20B96FF0150005B0BDE8F08378
:10C35000002237782B684FEA870C03EB8703C3F87A
:10C360001025C3F810250FFA88F205EB4202938AD4
:10C3700023F4604323F020039382707800B329688C
:10C38000B6786144D1F81035000423F4991323F4EE
:10C39000F853C1F81035230200F4403003F47C5305
:10C3A00003433005D1F8105500F4801003432B43AC
:10C3B000C1F81035938A43EA473343F02003938250
:10C3C0000020C2E7C0E90312704770B50446154665
:10C3D000FFF714FE48B10846F8F710FC04EB4004E0
:10C3E0000020A38A5B0B2B7070BD6FF01500FBE77C
:10C3F00090F88C00003818BF01207047F8F726BC71
:10C400002DE9F34104461746FFF7F8FD0D4626686F
:10C4100000B32046FFF7FDFD8046D8B92046FFF760
:10C4200003FE05B2AD0005F5807246F80280216872
:10C43000B2582944D1F8102542F00102C1F8102564
:10C440002FB10122216802FA00F3C1F8043302B0CF
:10C45000BDE8F081D6F804332846002BA4BF4FF086
:10C460000043C6F80433F8F7C9FB04EB4004A38A81
:10C47000C3F38203042B11D0052B11D001A8019521
:10C48000F8F7AAFB019B0169D94001F001010231D3
:10C49000284602B0BDE8F041FFF7A1BD0321F7E750
:10C4A0000221F5E7FFF73ABE2DE9F04389B0109E6F
:10C4B0000446894690460021202268461F46129D68
:10C4C00001F0B3FA1F2E97BF01234FF0FF33B340A3
:10C4D00003F1FF332361119BC4E90098C4E902769C
:10C4E0006361183445B10FCD0FC495E80F0084E89F
:10C4F0000F0009B0BDE8F0836D46F4E773B504683A
:10C50000661C31D08568A9422ED264182CD05E18E2
:10C51000AE4288BF6B1A056A35B100930523A84760
:10C520000346184602B070BDBFF35B8F1946A41ACC
:10C53000101919B140EA0205AD070AD103290DDC33
:10C54000013811448A42ECD010F8014F02F8014B37
:10C55000F8E70078013902F8010BE9E750F8044BDD
:10C56000043942F8044BE9E76FF02103D9E773B5CA
:10C570000468651C32D08568A9422FD264182DD07A
:10C580005E18AE4288BF6B1A456ACDB10093052391
:10C59000A84702B070BD12F8015B0139057015465D
:10C5A000A01819B140EA0206B607F4D103290ADC43
:10C5B000013D014488420CD1BFF35B8F1846E8E788
:10C5C0001946A41AEBE755F8042B043940F8042B5C
:10C5D000ECE715F8012F00F8012BEBE76FF02100D5
:10C5E000D7E773B51C46036815465A1C29D08268E4
:10C5F000914226D25B1824D066189642866A88BF7C
:10C60000541A36B105232A460094B047204602B09A
:10C6100070BD184622464AB9294601F006FABFF312
:10C620005B8FF3E700F8015B013AF4E78307F9D188
:10C630004FF001336B43032AEEDD40F8043B043A2C
:10C64000F9E76FF02100E2E70020704710B4046BB7
:10C6500002460B4684B9C1681F2998BF23FA01F42A
:10C66000416861B18068834209D21069184051F86D
:10C670002430184410BC7047234610BC18474FF0B4
:10C68000FF30F7E770B5436B05460E46E3B9046922
:10C69000621C09BF43680C401C680C1B21462846DD
:10C6A000FFF7D4FF864207D02B6901331C44AB68E7
:10C6B0009C42F3D34FF0FF342868431C07D0AB688B
:10C6C000A34204D9204470BD98470446F4E70020F3
:10C6D000F9E730B5059CC4E90002039A2181198964
:10C6E000E260049A618121856261D3E9002502EB51
:10C6F0000113C4E906128A1C236203EB42036A1C7D
:10C7000013446D422B406362836953B90139E26976
:10C710008B4202EB031206DB002393736FF07F035F
:10C72000D373002030BD0133D381F0E72DE9F04F02
:10C73000B0F830A004465546002685B002EB030849
:10C7400091460E9A00EBCA031FFA88FB9A63A3F87E
:10C750003CB008F1FF32C3690F1D0192B0451ADCED
:10C76000238D2586A3EB0B032385236A61895A88D1
:10C7700001390A4003EB4203A3F804A0BFF35B8F27
:10C780000020226A538801335380638D013363850F
:10C7900005B0BDE8F08FE06A2A0157F8041C03EBEE
:10C7A0000515029303680392C91A836808379942F2
:10C7B00028BF4FF0FF31FFF749FFDDE90232985003
:10C7C00000226A6057F8082CAA60019A9642ACBF12
:10C7D00000220122B145D8BF42F00202AA810136EF
:10C7E000ED89BBE7F0B550B3456A448E6B88A34230
:10C7F00030D0631C43864389BFF35B8F013B1C40F1
:10C8000005EBC4056B689EB209B1AD680D60D0F848
:10C810001CC09BB20CEB031100EBC3039D8F078D73
:10C820002F44013D07859D878D896F070ED5058EA5
:10C83000CD8100210686986B996302B11480F0BD0A
:10C840009D8FC989013D0CEB01119D878D89ED07F5
:10C85000F6D4ECE70020F2E7C36903EB0113986814
:10C860007047C36909015958C06AFFF70BBF70B51B
:10C87000BFF35B8F0D46016A1646838E4A880446D5
:10C880009A4212D05A1C82864289013A134001EB27
:10C8900043018988298089B2FFF7E3FF2A88E36989
:10C8A00003EB02139B68336070BD0020FCE710B5FA
:10C8B000026893691269920017D543B9438E026AE0
:10C8C00081694489013B1B1B02EB41029380036891
:10C8D0009B69012B08D1838E426A81694089013BA3
:10C8E0001B1A02EBC102938010BD23B9026A1388A0
:10C8F00043F00103138003689B69012B01BF426A67
:10C90000138843F001031380EEE710B5BFF35B8F8C
:10C91000036804461A699B6912F0005F1AD07BB95C
:10C92000036A426A5B888169013B02EBC10292881B
:10C930009B1A628D9BB29A4214D80023638510BD66
:10C94000012BFAD1436A026A5B888169013B02EBE1
:10C950004102ECE763B9436A1B88DB4303F0010340
:10C96000002BEAD06369002BE7D020469847E4E724
:10C97000012BE2D1036AEFE7036A828E5988914264
:10C980000AD0418901390A4003EB42039A88C369FE
:10C9900003EB02139868704700207047BFF35B8F6A
:10C9A000C36803B1184770474FF0FF324FF0FF33B1
:10C9B000F9F714BA10B1C36A0133C362704738B1D2
:10C9C000C26A013AC2621AB9026B02B1104702622E
:10C9D000704770B50446056A05F164063046FFF7F6
:10C9E000E3FF636AA3F580637F2B0BD8012259090B
:10C9F000503503F01F039A4055F8213023EA020313
:10CA000045F82130D4E90F124A60E16B04F13C0390
:10CA100011602046C4E90F33FFF7D1FF3046BDE86F
:10CA20007040F9F7A1B910B5436A8CB00A9320237E
:10CA3000044602460B9102A8194600F038FB282351
:10CA40000122CDE9003220463522616A02ABF8F7B7
:10CA500055FC00EAE0700CB010BD30B1006A20B1A6
:10CA600019B1D0F8883003B11847704730B1006A67
:10CA700020B119B1D0F88C3003B11847704730B1EC
:10CA8000006A20B119B1D0F8903003B118470020E6
:10CA900070472DE9F84306468846174699460468CC
:10CAA000A64201D1002520E07A1CA4F13C0502D069
:10CAB0006B6ABB4219D0B8F1000F22D02022414648
:10CAC000284600F0CAFFE0B9B9F1FF3F02D0AB6AD7
:10CAD0004B450AD07B1C0BD02468B442E2D054F8FA
:10CAE000183CA4F13C059F42E8D12846BDE8F883F4
:10CAF000AB6A0133F9D02468B442D3D0A4F13C0529
:10CB0000D9E72468CCE770B505460C461E46CAB185
:10CB100020232046194600F0CAFA0123E362049B51
:10CB20006662A362059B25626363069BA363079B02
:10CB300063646A6804F13C03C4E90F526B60226CC1
:10CB4000136070BD0A70E8E710B5044690B1036A3F
:10CB500083B102784AB193F8A43033B1436AB3F594
:10CB6000806F02D30121FFF75EFF2046BDE8104031
:10CB7000FFF72FBF10BD20B1036A13B15B6803B18B
:10CB80001847704708B530B1036A3BB1DB682BB179
:10CB90009847002008BD6FF01500FBE76FF0050017
:10CBA000F8E77047F9F7E0B84FF0FF324FF0FF3386
:10CBB000F9F714B9F8B50C4600F164070546A4F17D
:10CBC00010063846FFF7F0FF3046F8F74DFC80B10D
:10CBD00054F8083C24F8083CD5F8CC3044F80C3C18
:10CBE00005F1C80344F8103CC5F8CC6054F80C3C7F
:10CBF0001E603846FFF7D6FF0020F8BD38B50D4659
:10CC000000F164042046FFF7CFFF55F8083C2046AA
:10CC100003F5803345F8083CBDE83840FFF7C2BF54
:10CC20002DE9F04188B00E9C282A8846D4F8C0002F
:10CC30006ED101688568A8EB0101A94228BF4FF0B9
:10CC4000FF3120236A46FFF759FC04F16406D8F847
:10CC500020703046FFF7A8FF3B464FF0FF32694691
:10CC60002046FFF716FFD8F824300546E0B1D0F88B
:10CC7000308003F00103B8F1000F02D0DBB9AF62DE
:10CC800030E0002BFBD04FF0FF3383623046FFF7DC
:10CC900089FFAB6B83BBD4F88030002B38D03A4689
:10CCA00069462046984733E0DB071FD43046FFF73C
:10CCB00079FFE36FF1E74FF0FF338362FFF77AFE0E
:10CCC0003046FFF76FFFAB6BA3B9D4F880301BB1D0
:10CCD0003A466946204698473046FFF765FF2846A2
:10CCE000FFF76DFE3046FFF75DFF11E03046FFF7BE
:10CCF00059FFD0E74FF0010828469847D4F8803014
:10CD00001BB13A46694620469847B8F1000FE3D177
:10CD1000002008B0BDE8F081F0B504468E680D46ED
:10CD2000B6B23146D0F8B80085B0FFF795FDD4F81B
:10CD3000B43007469A6942B90095CDE90250012303
:10CD4000D4F8B80002A9FFF7F1FCD4F8B4309B691D
:10CD5000012B08D13A463146D4F8B80005B0BDE8F9
:10CD6000F040F8F7AFBA05B0F0BD70B500F1640659
:10CD7000A1F1100504463046FFF716FF2846F8F7E4
:10CD800073FB38B120462946FFF7C6FFD4F8B80038
:10CD9000FFF7BBFD3046BDE87040FFF703BF2DE94C
:10CDA000FF4103689E6A06F164084046FFF7FCFEF7
:10CDB000D6F8B4309B693BB1012B12D04046FFF747
:10CDC000F1FE04B0BDE8F081D6F8B8000DF10A021A
:10CDD00003A9FFF707FDD6F8B43004469B69012B81
:10CDE00007D1D6F8B80003AA0DF10A01FFF73FFDFD
:10CDF0000446002CE2D0BDF80A3000216268A3602E
:10CE000030464FF0FF33FFF744FE0546FFF7D2FDF3
:10CE1000A368404603F58033A360FFF7C3FE75B1F6
:10CE2000AB6A696C013308BF2368284608BFAB6250
:10CE30002368A28900916F6B04F11001B847404646
:10CE4000FFF7B2FE2846FFF7BAFD2046F8F70CFBC5
:10CE500038B130462146FFF75FFFD6F8B800FFF73C
:10CE600054FD4046FFF79EFE9FE72DE9F041A3F1F8
:10CE7000100653F8085C002388B00693ADF81E3006
:10CE800004461023CDE904120E9FD0F8C000ADF87F
:10CE90001C700168D0F808C0711A0DEB03026145DF
:10CEA00028BF4FF0FF3104F16408FFF760FB4046F4
:10CEB000FFF77AFED4F8B430ADB29B69CBB9D4F8A1
:10CEC000A820D4F8B430D4F8BC009B69C3B9CDE92C
:10CED00002620096012202A9FFF728FCD4F8BC00E8
:10CEE000FFF713FD4046FFF75DFE384608B0BDE88A
:10CEF000F0812946D4F8BC00FFF7AEFC0246E0E71B
:10CF0000012BEBD12946F8F7DDF9E7E710B548B179
:10CF100049B143688B4206D382680468D21A5B1A0F
:10CF20004360A01810BD0020FCE72DE9F34705463B
:10CF3000D0F8B4000E46904618B9002002B0BDE803
:10CF4000F087036A002BF8D09B68002BF5D0984738
:10CF50004307F2D543F69823B8F1000F18BF98465F
:10CF600005F1640705F1C8093846FFF71DFED5F83D
:10CF7000C8404C452BD054B3D4E9002353602268F9
:10CF80001A60C4E90044D5F8B43021899B69ADF832
:10CF900006107BB1012B14D03846FFF703FEBDF815
:10CFA000063004F1100003F58033A3603368103BB2
:10CFB0003360C3E7D5F8A8303360D5F8B4309B6947
:10CFC000E8E7D5F8BC00FFF747FC3060E4E7D5F8A8
:10CFD000B430D3F818A0BAF1000F36D13146D5F8E5
:10CFE000BC000DF10602FFF7FDFB04460028D3D17B
:10CFF000D5F8BC301B8DB3B93846FFF7D3FDB8F177
:10D00000000F9AD0D5E92D32182112891B6B01FB34
:10D010000233D5F8D02022BB2120002100F042FBB2
:10D0200008F1FF38A0E7D5F8A810D5F8C400FFF73D
:10D030006DFF0446D5F8A830ADF806A03360384639
:10D04000FFF7B0FD002CDAD0A9E7BAF1010FD3D178
:10D050003246D5F8BC000DF10601FFF708FC044686
:10D06000EDE71969284690476FF4FB639842D3D0E7
:10D0700000283FF479AF60E720B119B112B1C0E9DF
:10D0800001220160704738B5044618B938BD3C38F4
:10D09000FFF75AFD20688442F9D10025D4F8B40086
:10D0A000C4E92E55FFF767FDC4F8B450EEE770B53C
:10D0B00005461C4699B18B4228BF0C46661C013EB2
:10D0C00005D012F8013B00F8013B002BF7D1A1423B
:10D0D00007D9091B8A19002100F0A7FCA11B0846EB
:10D0E00070BD00230D4405F8013CF7E708B1F4F7E3
:10D0F00035BE704710B5436904463BB90020E2686D
:10D100004042537843F00103537010BD9847002804
:10D11000F4D00028B8BF4042FF28A8BFFF20E36832
:10D120001870ECE740B1C368587810F001001EBFDA
:10D130001878B0FA80F040097047EFF3118320238C
:10D1400083F31288BFF36F8FFEE708B5FFF7F5FF93
:10D1500010B400F10C04C0E9034410BCFDF745BB5A
:10D1600038B50446EFF31185202383F31288BFF30B
:10D170006F8FFDF7EAFA04F10C0000F080FA30B18D
:10D18000294604F11400BDE83840F9F71FBA85F3C9
:10D190001188BFF36F8F38BD4169826842EA01038D
:10D1A00013F003030FD1C3600369013B03FB0122AA
:10D1B000002B01DA00207047C168013B1160416912
:10D1C000C260521AF4E76FF01500704710B5C0E95D
:10D1D00004320023816083610446FFF7DDFF0028ED
:10D1E000A8BFC4E9004410BD2DE9F04105460F4633
:10D1F000EFF31188202383F31288BFF36F8FC66883
:10D20000FEB90468A0421CD0DCB1D4E9003213603E
:10D210005A60637BC4E9006623F002036373A6606F
:10D2200004F1180000F099FA2046C4F8B0602761B4
:10D2300000F0DCF9414605F10800BDE8F041F9F7DE
:10D24000C5B93E60AB69EF60013BAB6188F3118803
:10D25000BFF36F8FBDE8F081202408B5EFF3118391
:10D2600084F31288BFF36F8FFDF7ABFEF6E790F9FA
:10D270000E308B4201D0F9F737B9002070470346D2
:10D280000020C3E90033C3E902007047D0E900324F
:10D2900013605A600023427BC0E9003322F002028F
:10D2A0004273836070472DE9F843914604460D466A
:10D2B0009DF8202000F10807EFF31186202181F36B
:10D2C0001288BFF36F8F02B14568D4F808804745D4
:10D2D00018D0B8F1000F15D04046FFF7D7FF08F17E
:10D2E000180000F03AFA00234046C8F8B030C8F8F9
:10D2F000109000F07BF938463146F9F767F90020C5
:10D30000BDE8F883A3B10820F9F75CFD002838D008
:10D310000122C0F804900260016801F003015DB9C8
:10D3200022680A430260626820606AB960600BE0AC
:10D330004846C9F80030EFE72A68032A16D801608A
:10D34000616869B9C4E90000042104F1100000F02B
:10D35000B9FA0028CFD186F31188BFF36F8FCFE7DA
:10D360000A6802F0030202430A60DFE722F00302C8
:10D370000A4302602A6802F0030240EA02032B60BB
:10D38000E2E76FF00B00E6E710B5044630B1026843
:10D39000930703D0446809B100F0CBFA204610BDD2
:10D3A0000023C0E9003300F10803C0E9023300F1B3
:10D3B0001003C0E904337047012307B5009300232D
:10D3C0000A461946FFF76FFF03B05DF804FB002320
:10D3D00007B50A4600931946FFF765FF03B05DF8ED
:10D3E00004FB5AB18A4209D300F11003C0E90212CA
:10D3F000C0E90000C0E90433002070476FF0150059
:10D400007047012302688B4022EA0303036022FA7B
:10D4100001F000F001007047704710B50321044689
:10D420000C30FFF7EEFF30B104F1100000F095F979
:10D43000B0FA80F0400910BD20B10022C43011467E
:10D4400000F051B9704770B5C3680446C3F3400695
:10D450009B0716D4856802210C30FFF7D2FF80B1FC
:10D46000D5F8BC206AB194421DD122689EB9D5F886
:10D47000C030C5F8BC209C4201D1C5F8C0200023B3
:10D480002360E36813F01F001EBF43F00203E36054
:10D4900040F0020070BD3260D5F8C020944208BF51
:10D4A000C5F8C060EBE716461268DBE738B50446FE
:10D4B0000D461022002100F0B8FA656038BD13B5A2
:10D4C00001900846EFF31184202383F31288BFF301
:10D4D0006F8F01A9F8F74EFD84F31188BFF36F8FAA
:10D4E00002B010BD10B5FFF7EAFF041E08DDEFF330
:10D4F0001180202383F31288BFF36F8FF9F778F838
:10D50000204610BD70B50D46EFF31186202383F33E
:10D510001288BFF36F8FF8F789FD044686F31188F0
:10D52000BFF36F8F38B14FF0FF324FF0FF3305F18B
:10D530001000F8F753FC204670BD08B5D822002132
:10D5400000F073FA08BD38B50446EFF311852023C7
:10D5500083F31288BFF36F8FFFF75FFF2046FFF75B
:10D5600072FF85F31188BFF36F8F38BDEFF305802D
:10D57000003818BF01207047D0E9003213605A60AC
:10D580000023C0E90033704708B5FFF7F5FF437B80
:10D5900023F0020343730023836008BD38B50446BB
:10D5A0000D46F8F70FFF637B43F002036373E5B1A9
:10D5B000A5602B689D4209D16B68C4E900531C60CB
:10D5C0006C6012E06A689A42F6D01B68002BF3D0B8
:10D5D00094F90E2093F90E108A42F3D09142F1DDB6
:10D5E0005A68C4E9003214605C6038BD10B5EFF3CE
:10D5F0001184202383F31288BFF36F8FF8F7A0FE06
:10D6000084F31188BFF36F8F10BD08B5EFF311815C
:10D61000202282F31288BFF36F8F83680BB1FFF76C
:10D62000B3FF81F31188BFF36F8F08BD014610B5BA
:10D63000EFF31184202383F31288BFF36F8F437BB2
:10D6400013F0280F0AD183680BB1FFF79DFF4B7BC6
:10D65000084623F004034B73F8F772FE84F3118835
:10D66000BFF36F8F10BD01211838FFF7DFBF10B572
:10D67000FFF7CBFFBDE81040183000F06EB838B5AA
:10D68000054604680020AC4200D138BD002CFCD017
:10D690002046FFF7ECFF2046FFF7A8FF2C6801208B
:10D6A000A542F1E770B505460E46F9F749F8B6F11F
:10D6B000FF3F08BFB5F1FF3F0446284612D04FF4A4
:10D6C0007A7147F6FF730022C4FB0132D80B40EA9F
:10D6D0004240B0F1004F4FEAD23272F1000228BF4F
:10D6E0006FF0004070BD38B5EFF31185202383F350
:10D6F0001288BFF36F8F0468A04213D0A4B1C4F89E
:10D70000B01022612046FFF73FFF04F1180000F03F
:10D7100024F82046F8F714FE012085F31188BFF3A2
:10D720006F8F38BD0020F8E72046F6E708B50246BF
:10D73000F9F7C0F970B1D0E904319B1A61EBE272DC
:10D74000B3F1004F72F1000104DA002AACBF1846B1
:10D75000002008BD6FF00040FBE7024638B5EFF34C
:10D760001185202383F31288BFF36F8F0368CBB139
:10D77000F9F7A0F904461046F9F7AEF900224FF088
:10D7800000438442C0E9042306D1F9F79BF9FFF76F
:10D79000CDFF0021F6F712FF002085F31188BFF3BB
:10D7A0006F8F38BD6FF01500F7E708B5F9F79EFAEF
:10D7B00008BDB3F1FF3F08BFB2F1FF3F70B50646A9
:10D7C0001D46144614D01A4316D0002B08DBF9F777
:10D7D0008DFA041941EB0501C6E90041304670BDE0
:10D7E0006FF001031C1B4FF0FF3363EB0501F3E700
:10D7F0004FF0FF342146EFE70024FBE7B3F1FF3F92
:10D8000008BFB2F1FF3FF8B5074616461C4610D0D8
:10D8100054EA020311D0F9F769FAB0420A46A1416D
:10D8200003460AD2F31A64EB0204C7E9003438460F
:10D83000F8BD4FF0FF331C46F7E70023FBE72DE967
:10D84000F041846805460E46D4B16378012B22D19D
:10D8500014F8533C9A0711D5A4F160073846FFF736
:10D8600006FF082E0CBF6FF003030023236514F896
:10D87000533CDB0602D13846FFF7B8FE0023237085
:10D880000020EB68A860C3F38632164366F3943336
:10D89000EB60BDE8F081022BF0D12378002BEDD0B6
:10D8A00054F8048CB8F1000FE8D004F11400FFF72D
:10D8B00054FF0023A4F1140739464046E362FFF702
:10D8C000FEFDDBE738B5EFF31185202383F31288E3
:10D8D000BFF36F8F0468A04211D0D4E90032136007
:10D8E0005A6000232046C4E90033FFF7A8FF85F300
:10D8F0001188BFF36F8F201E18BF012038BD002490
:10D90000F5E7043270B504460ED2EFF311852026F8
:10D9100086F31288BFF36F8F41F00401984785F3B7
:10D920001188BFF36F8F08B9002070BD40F8044B19
:10D93000FBE720B1011F50F8040CFFF711BC704742
:10D94000704700207047704710B5044608B1F9F7DA
:10D9500009FC2046BDE81040F9F7F4BB10B50446B9
:10D96000406A10B1A16AFFF7EFFF0020C4E9090087
:10D9700010BD38B50546FFF7F1FF2B7F0446012B9C
:10D980000ED0023B012B0ED82B6A012B18BF6FF073
:10D9900096042C220021284600F047F8204638BD86
:10D9A0002B6A002BF2E76FF09604F2E70020704735
:10D9B00070470020704713B5002001AB1446F9F7FB
:10D9C000A1FD30B9019BA34218BF6FF0930002B0D4
:10D9D00010BD6FF09200FAE7002070470A44431E22
:10D9E000914200D1704710B511F8014B914203F8F4
:10D9F000014FF9D110BD884210B501EB020402D9E4
:10DA00008442234607D8431EA14208D011F8012BB7
:10DA100003F8012FF8E7024401468A4200D110BD05
:10DA200013F8014D02F8014DF7E702440346934213
:10DA300000D1704703F8011BF9E70139024410B522
:10DA4000904201D1002005E0037811F8014FA34274
:10DA500001D0181B10BD0130F2E710B56AB10139D1
:10DA6000841810F8012B11F8013F9A4203D1A0420B
:10DA700001D0002AF5D1D01A10BD1046FCE710B530
:10DA80000139044632B111F8013F013A00F8013B77
:10DA9000002BF7D10021FFF7C8FF204610BD02463A
:10DAA000014410B58A42134603D01C780132002C81
:10DAB000F8D1181A10BDF0B5C3F13707044603F0CA
:10DAC0001F031046FFB2082BE6B232D0102B3DD018
:10DAD0006508A40845EAC17544EA81748A082D19CD
:10DAE00042EB5102290941EA02716D1842EB121210
:10DAF000290A41EA02616D1842EB1222290C41EA1F
:10DB000002416D1842EB1242AD1842F10002EC08DE
:10DB100044EA4274D10804EB8402A6EB4205EDB25C
:10DB2000092D0CD90134A5F10A0541F10001EDB22E
:10DB300012E0E40806F0070544EA4174C9083035EC
:10DB400054EA010200F8015BBDD1F0BD240906F0E2
:10DB50000F0544EA01740909092D84BFED19EDB2DE
:10DB6000EDE7D1E9043293421EBF5A1C0A611870D6
:10DB7000704700000148006870470000C012002094
:10DB8000D425FF7F01000000891E00000000000076
:10DB9000ED050000000000000000000048DC00006F
:10DBA000D15A000000000000F55A000000000000FB
:10DBB0000000000080DC00000000000064DC0000C9
:10DBC00055BD000000000000000000009CDC0000CB
:10DBD00000000000B8DC000000000000D4DC000001
:10DBE000B13B0000000000005D44000000000000A8
:10DBF000A51E000000000000711A000000000000D7
:10DC000000000000F0DC000059BD00000000000032
:10DC1000D56D000000000000000000000CDD0000D9
:10DC20000000000028DD00002DBD00000000000005
:10DC300037BD000000000000611F00000000000070
:10DC4000C50B00000000000098EC0000FCE10000A3
:10DC5000B8DF0000280300204C130020ED3800003E
:10DC600000000000C2EC000024E2000074DF0000AD
:10DC70002E030020F0130020553D0000000000009E
:10DC8000CEEC000038E2000074DF0000300300201A
:10DC9000FC130020553D000000000000A3EC000034
:10DCA000000000006CDF00002A03002000000000DC
:10DCB00051B9000000000000B2EC000000000000BC
:10DCC0001CE200002C030020000000005DB90000F1
:10DCD00000000000EEEC00004CE20000D4DF000089
:10DCE000340300209014002015BC00000000000048
:10DCF000DAEC00005C02002098DF00003203002014
:10DD000008140020113F00000000000088EC000013
:10DD1000FC00002088E0000024030020780400209C
:10DD200013AD00000000000081EC000000000000C6
:10DD3000ACDF0000260300201802002000000000D5
:10DD400000000000000000009DAF00000000000087
:10DD50009DAF0000000000009DAF0000000000002B
:10DD60009DAF0000000000009DAF000055BE000008
:10DD70006BBD0000000000009DAF0000000000002F
:10DD80009DAF0000D4DC0000B5BB00000000000027
:10DD90009DAF0000000000009DAF000000000000EB
:10DDA0009DAF0000000000009DAF00006801002052
:10DDB00051BA0000000000009DAF0000000000000C
:10DDC0009DAF0000000000009DAF000000000000BB
:10DDD0009DAF0000000000009DAF000000000000AB
:10DDE0009DAF0000000000009DAF0000000000009B
:10DDF000ED440000000000009DAF000000000000A6
:10DE00009DAF0000000000009DAF0000000000007A
:10DE10009DAF0000000000009DAF0000000000006A
:10DE20009DAF0000000000009DAF0000000000005A
:10DE30009DAF0000000000009DAF0000000000004A
:10DE40009DAF0000000000009DAF0000000000003A
:10DE50009DAF0000000000009DAF0000000000002A
:10DE60009DAF0000000000009DAF0000000000001A
:10DE70009DAF0000000000009DAF0000000000000A
:10DE80009DAF0000000000009DAF000000000000FA
:10DE90009DAF0000B54F00006BBD0000000000000A
:10DEA0009DAF0000000000009DAF000000000000DA
:10DEB0009DAF0000000000009DAF000000000000CA
:10DEC0009DAF0000000000009DAF000000000000BA
:10DED0009DAF0000000000009DAF000000000000AA
:10DEE0009DAF0000000000009DAF0000000000009A
:10DEF0009DAF0000000000009DAF0000000000008A
:10DF00009DAF0000000000009DAF00000000000079
:10DF10009DAF0000000000009DAF00000000000069
:10DF20009DAF0000000000009DAF00000000000059
:10DF30009DAF0000000000009DAF00000000000049
:10DF40009DAF0000000000009DAF00000000000039
:10DF50009DAF0000000000009DAF00000000000029
:10DF60009DAF0000000000009DAF000055B900000B
:10DF700000000000913D0000B7B90000C3B90000E7
:10DF8000D7B90000E1B90000EBB90000013C000086
:10DF9000FFB90000000000009BBA000077BA000043
:10DFA00093BA000097BA0000C3BA0000D5B70000CA
:10DFB00013B800009DB7000051390000A9B8000057
:10DFC0000BB900000000000045B800000000000090
:10DFD000000000006FBB00006941000061BB000051
:10DFE000040000000F000000010000000800000015
:10DFF0002000000064000000740000000D0000001C
:10E000000C0000000E00000050000000780000002E
:10E01000AC000000FFFFFFFFFFFFFFFFFFFFFFFF60
:04E02000FFFFFFFF00
:10E0300095510000060000000002000000020000F0
:10E0400000000000000000000000000000000000D0
:10E050000338FDD8704700004006800700400000EC
:10E060000000000000040000A0000000F00000001C
:10E070000000000079010000000000000000000026
:10E08000091C000010E600006D060000CBAD00008A
:10E090006908000000000000B5080000A1090000A8
:10E0A000A9AB00001DAC0000B1AB0000E3AB000069
:10E0B000CDAB0000B7AB0000000000000000000086
:10E0C000FBAE0000EDAE0000F7AE0000EBAE0000CE
:10E0D0000000000000000000000000000000000040
:10E0E000DBAE0000000000007DAF0000500100200A
:10E0F00048010020400100200000000038010020FD
:10E100001D0D0000ED0B0000410C0000B50C0000DF
:10E1100000000020000000000600010002000000D6
:10E1200024E100000000000027EB000006000000D2
:10E13000E0FF0F00000000202FEB00002100000096
:10E14000E0FF062058010020FD1A0000000000003A
:10E150007BB00000D51D0000A1B100000000000050
:10E1600048E1000070E100004700000000000000EE
:10E170006058002048E1000084E100003D000000FC
:10E1800000000000405C002048E1000098E1000031
:10E190000201000000000000405D00200E030000AE
:10E1A000092900000F040000012A00003E010000C0
:10E1B000F11F0000FF010000B11F00003E01000040
:10E1C000D11F00001001000043B200001205000042
:10E1D00059350000130800009DB6000048E100001A
:10E1E000ECE1000003010000000000005C5E002084
:10E1F000A938000079380000000000000D3A000046
:10E200008D3900004DB9000049B9000031B9000056
:10E210003DB900002BB9000037B9000073B9000008
:10E2200000000000FFFF000000288450680100206B
:10E230000000000001000000FFFFFFFF00258450E8
:10E240006801002000000000000000000080005075
:10E25000010000000000000070E200000000D60194
:10E260000000000000000000B8250020B7250020B5
:10E27000008000507CE200000100000084E2000009
:10E280000400000014000000130000021606000144
:10E29000150600030800000003000000080000004D
:10E2A0000300000036ED000049ED00005CED0000C9
:10E2B0006FED000082ED000095ED0000A8ED00007C
:10E2C000BBED000088DB000090DB0000E8DB000015
:10E2D000F8DB000040DC000048DC00002AEE000013
:10E2E0000001000000000000FF8FFFFFFF8FFFFF15
:10E2F000FE8FFFFFFE8FFFFFFD8FFFFFFC8FFFFFF5
:10E30000FC8FFFFFFB8FFFFF6D757465785F667292
:10E3100065652063616C6C65642077697468204E64
:10E32000554C4C20706172616D657465720000001F
:10E3300043616E277420696E697469616C697A65DE
:10E34000206D757465782C20776173204E554C4C88
:10E350000D0A00004661696C20746F20616371755D
:10E36000697265206D757465780A00004661696C94
:10E3700020746F20696E63726561736520504D2053
:10E38000636F756E7465720A000000004661696C07
:10E3900020746F20646563726561736520504D2041
:10E3A000636F756E7465720A000000004661696CE7
:10E3B00020746F2072656C65617365206D7574657E
:10E3C000780A0000436F756C64206E6F74206C6F68
:10E3D000636B20706F7765722073617665206D7551
:10E3E000746578004661696C20746F20756E6C6F7F
:10E3F000636B206D757465780A0000006374782083
:10E4000063616E6E6F74206265204E554C4C000047
:10E410000A637478206973204E554C4C0A00000042
:10E4200067E6096A85AE67BB72F36E3C3AF54FA5A5
:10E430007F520E518C68059BABD9831F19CDE05BD1
:10E44000D89E05C107D57C3617DD703039590EF7D7
:10E45000310BC0FF11155868A78FF964A44FFABE9D
:10E460000123456789ABCDEFFEDCBA9876543210B4
:10E47000F0E1D2C3416476657274697365725B259D
:10E48000645D2025702073656E742025640A005336
:10E4900074617274696E6720436F6E6E6563746930
:10E4A0006F6E6C65737320426561636F6E204465A7
:10E4B0006D6F0A00426C7565746F6F746820696EC9
:10E4C000697469616C697A6174696F6E2E2E2E00B1
:10E4D0006661696C65642028657272202564290A6A
:10E4E00000737563636573730A00416476657274C3
:10E4F0006973696E67207365742063726561746502
:10E500002E2E2E00536574206164766572746973D3
:10E51000696E6720646174612E2E2E0055706461EF
:10E5200074652043544520706172616D732E2E2EE8
:10E5300000506572696F6469632061647665727406
:10E540006973696E6720706172616D7320736574A1
:10E550002E2E2E00456E61626C65204354452E2E92
:10E560002E00506572696F6469632061647665721C
:10E57000746973696E6720656E61626C652E2E2EFC
:10E5800000457874656E64656420616476657274B4
:10E590006973696E6720656E61626C652E2E2E0050
:10E5A0007075626C69630072616E646F6D00707586
:10E5B000626C69632D69640072616E646F6D2D69B0
:10E5C000640030782530327800253032583A2530D2
:10E5D00032583A253032583A253032583A253032BE
:10E5E000583A253032582028257329005374617217
:10E5F00074656420657874656E6465642061647612
:10E600006572746973696E672061732025730A00EF
:10E61000444620436F6E6E656374696F6E6C6573FC
:10E620007320426561636F6E20417070006D626F90
:10E63000785F777120232564002A2A2A20426F6F91
:10E6400074696E67206E524620436F6E6E65637408
:10E650002053444B2076332E332E302D62613136D9
:10E660003764396633646234202A2A2A0A002A2A47
:10E670002A205573696E67205A6570687972204F39
:10E68000532076342E332E39392D666439323034A6
:10E69000613032643532202A2A2A0A006D75746589
:10E6A000785F696E69742063616C6C65642077695A
:10E6B0007468204E554C4C20706172616D657465B4
:10E6C0007200436F756C64206E6F7420616C6C6FA8
:10E6D00063617465206D75746578206265666F721C
:10E6E0006520696E697469616C697A696E67007228
:10E6F000302F61313A202030782530387820207250
:10E70000312F61323A20203078253038782020723D
:10E71000322F61333A20203078253038780A007261
:10E72000332F61343A202030782530387820723108
:10E73000322F69703A2020307825303878207231B5
:10E74000342F6C723A20203078253038780A002037
:10E75000787073723A20203078253038780A004675
:10E7600061756C74696E6720696E73747275637419
:10E77000696F6E206164647265737320287231352D
:10E780002F7063293A203078253038780A00556E8A
:10E7900068616E646C6564204952516E3A2025644C
:10E7A0000A002A2A2A2A2A20555341474520464151
:10E7B000554C54202A2A2A2A2A0A00202044697605
:10E7C0006973696F6E206279207A65726F0A002022
:10E7D00020556E616C69676E6564206D656D6F7242
:10E7E00079206163636573730A0020205374616349
:10E7F0006B206F766572666C6F772028636F6E741E
:10E800006578742061726561206E6F742076616C2A
:10E810006964290A0020204E6F20636F70726F6355
:10E820006573736F7220696E737472756374696F48
:10E830006E730A002020496C6C6567616C206C6FF8
:10E840006164206F66204558435F52455455524ECF
:10E8500020696E746F2050430A002020496C6C655B
:10E8600067616C20757365206F662074686520454C
:10E870005053520A002020417474656D70742074E6
:10E880006F206578656375746520756E646566696B
:10E890006E656420696E737472756374696F6E0A55
:10E8A000002A2A2A2A2A20425553204641554C54F0
:10E8B000202A2A2A2A2A0A002020537461636B69BD
:10E8C0006E67206572726F720A002020556E737435
:10E8D00061636B696E67206572726F720A00202037
:10E8E0005072656369736520646174612062757339
:10E8F000206572726F720A00202042464152204108
:10E900006464726573733A20307825780A00202099
:10E91000496D70726563697365206461746120621A
:10E920007573206572726F720A002020496E7374CD
:10E9300072756374696F6E20627573206572726F91
:10E94000720A002020466C6F6174696E672D706FCB
:10E95000696E74206C617A792073746174652070BB
:10E960007265736572766174696F6E206572726F1D
:10E97000720A002A2A2A2A2A204D5055204641553B
:10E980004C54202A2A2A2A2A0A0020205374616320
:10E990006B696E67206572726F722028636F6E7488
:10E9A0006578742061726561206D696768742062A2
:10E9B00065206E6F742076616C6964290A002020DE
:10E9C00044617461204163636573732056696F6CA1
:10E9D0006174696F6E0A0020204D4D4641522041FE
:10E9E0006464726573733A20307825780A002020B9
:10E9F000496E737472756374696F6E2041636365E9
:10EA000073732056696F6C6174696F6E0A0052658A
:10EA100073657276656420457863657074696F6E9E
:10EA200020280053707572696F757320696E746564
:10EA3000727275707420284952512000535053450A
:10EA40004C20696E20746872656164206D6F646526
:10EA500020646F6573206E6F7420696E64696361F2
:10EA60007465205053500A002A2A2A2A2A20484135
:10EA70005244204641554C54202A2A2A2A2A0A0068
:10EA80002020427573206661756C74206F6E20764D
:10EA90006563746F72207461626C65207265616475
:10EAA0000A0020204465627567206576656E740AE9
:10EAB0000020204661756C7420657363616C61741D
:10EAC000696F6E20287365652062656C6F77290A0F
:10EAD00000415243485F455843455054207769747C
:10EAE0006820726561736F6E2025780A0A002A2AF1
:10EAF0002A2A2A204465627567206D6F6E69746FDB
:10EB00007220657863657074696F6E202A2A2A2ADC
:10EB10002A0A002A2A2A2A2A202573202564292045
:10EB20002A2A2A2A2A0A00464C4153485F300053B9
:10EB300052414D5F3000657869740000000001218A
:10EB4000200B0A0405060700000000000000FFFF7C
:10EB5000FFFFFFFF000000000000010400020000B2
:10EB6000000200000000000000050000000000009E
:10EB70000000000000000000000562745F74785F10
:10EB800070726F636573736F7200574553545F54AF
:10EB90004F504449522F7A65706879722F737562AD
:10EBA0007379732F626C7565746F6F74682F686FFB
:10EBB00073742F6863695F636F72652E6300657697
:10EBC000745F666C6167732026202831554C203CA9
:10EBD0003C202830292900415353455254494F4E77
:10EBE000204641494C205B25735D20402025733A27
:10EBF00025640A0062745F6863695F6576745F67A5
:10EC000065745F666C616773286864722D3E657613
:10EC100074292026202831554C203C3C20283129BD
:10EC20002900657272203D3D20300009436F6E74EB
:10EC3000726F6C6C657220756E726573706F6E7337
:10EC40006976652C20636F6D6D616E64206F7063F3
:10EC50006F6465203078253034782074696D656F75
:10EC600075742077697468206572722025640A00C3
:10EC7000425420525820575100627566000001FF2F
:10EC80000262745F6863695F69706330006E726608
:10EC90005F62745F68636900636C6F636B403530FB
:10ECA000303000656E74726F70795F62745F686394
:10ECB000690063727970746F4035303834343030A5
:10ECC00030006770696F4038343238303000677018
:10ECD000696F40383432353030006D626F784032C1
:10ECE000613030300000010203040506070B756136
:10ECF0007274403830303000000000010101000023
:10ED00000100000000203030303030303030303002
:10ED1000303030300001756E7265676973746572EA
:10ED20006564202573206275730A0067656E6572DD
:10ED30006963002573006D6574616C3A20656D65CB
:10ED40007267656E63793A20006D6574616C3A2074
:10ED5000616C6572743A2020202020006D6574611A
:10ED60006C3A20637269746963616C3A2020006DAB
:10ED70006574616C3A206572726F723A20202020AF
:10ED800020006D6574616C3A207761726E696E6700
:10ED90003A202020006D6574616C3A206E6F7469B2
:10EDA00063653A20202020006D6574616C3A20690B
:10EDB0006E666F3A202020202020006D6574616C03
:10EDC0003A2064656275673A202020202000257370
:10EDD0003A2066726565696E67206E6F6E2D656D8F
:10EDE000707479207669727471756575650D0A00A5
:10EDF000756E6578706563746564206275666665B6
:10EE0000722068656C6420636F756E7465720D0A9C
:10EE10000072785F76710074785F7671004E5300EF
:10EE200069646C65006D61696E00737973776F72E8
:10EE30006B7100286E756C6C29002A666C6F6174AA
:10EE40002A00000000000000000000000000000098
:10EE500000000000000000000000000000000000B2
:10EE600000000000000000000000000000000000A2
:10EE70000000000000000000000000000000000092
:10EE80000000000000000000000000000000000082
:10EE90000000000000000000000000000000000072
:10EEA0000000000000000000000000000000000062
:10EEB0000000000000000000000000000000000052
:10EEC000E528000000000000000000000000000035
:10EED0000000000000000000000000000000000032
:10EEE0000000000000000000000000000000000022
:10EEF0000000000000000000000000000000000012
:10EF00000000000000000000000000000000000001
:10EF100000000000000000000000000000000000F1
:10EF200000000000000000000000000000000000E1
:10EF300028DD000014010500000000009BA800006F
:10EF4000000000000000072000000100F0DC0000CD
:10EF500000000000F0DC00000100000002000000E2
:10EF600000000000000000000002000088030020F4
:10EF70003A000000740300203A0000006003002003
:10EF80003A0000009C0300203A0000004C030020DF
:10EF90003A000000B00300203A000000000000002A
:10EFA00071B00000000000000000000000D0005020
:10EFB0000000000000000000000000000000000051
:10EFC0000000000000000000000000000000000041
:10EFD0000000000000000000000000000000000031
:10EFE0000000000000000000000000000000000021
:10EFF0000000000000000000000000000000000011
:10F000000000000000000000000000000000000000
:10F0100000000000000000000000000000000000F0
:10F0200000000000000000000000000000000000E0
:10F0300000000000000000000000000000000000D0
:10F040004529000000000000000000000000000052
:10F050001922000000000000000000000000000075
:10F0600000000000000000008DEC00000000000027
:10F0700095B7000000000000053700000000000008
:10F0800028DD0000400200204002002000000000B7
:10F090000100000050020020500200200CDD0000A2
:10F0A000FFFF0000FFFF00000090D003FF00000002
:10F0B000FF0000002BED000000000000F54F0000F5
:10F0C0000000000000000000000000000000000040
:10F0D0000000000000000000000000000000000030
:10F0E00090020000A0020020A002002047D90000EA
:10F0F00043D900002BDA0000DD730000D17300005B
:10F10000C5730000000000002D74000004030020FF
:10F11000FC020020F402002000000000EC020020AD
:10F12000FD750000497500007D750000C575000083
:10F13000AC1C00203A00003AB01C00203A00003A13
:10F14000B41C00203A00003AB81C00203A00003AF3
:10F150000022002018030020D8020020D002002046
:10F16000CC020020C80200200000000000000000C7
:10F17000000000000000000000000000000000008F
:10F1800060440020001000000000000000000000AB
:10F190004C0300204C030020000000000000000091
:10F1A0000E0000006003002060030020000000004B
:10F1B000000000000E000000740300207403002013
:10F1C00000000000000000000E0000008803002086
:10F1D0008803002000000000000000000E00000076
:10F1E0009C0300209C0300200000000000000000A1
:10F1F0000E000000B0030020B0030020000000005B
:10F20000000000000E0000000000000000000000F0
:10F21000CC030020CC030020D4030020D403002022
:10F2200003000300000000000000000074E1000083
:10F23000F85C00200000000000000000F80300203F
:10F24000F803002000040020000400200100010059
:10F250000000000000000000DCE10000605F002012
:10F26000000000000000000024040020240400200E
:10F270002C0400202C0400200A000A0004000000D6
:10F28000BD1E000060E10000285B002000000000BF
:10F29000000000005004002050040020580400200A
:10F2A00058040020010001000000000000000000E0
:0CF2B00088E10000445E002015E015E03D
:00000001FF
